:020000040800F2
:10000000C02601205D030008A10900082509000899
:100010009D090008B7070008D50B00080000000084
:10002000000000000000000000000000690200085D
:100030006908000800000000C5020008590A00080D
:1000400077030008770300087703000877030008A8
:100050007703000877030008770300087703000898
:100060007703000877030008770300087703000888
:100070007703000877030008770300087703000878
:100080007703000877030008770300087703000868
:10009000810B000877030008BD07000877030008FC
:1000A00077030008D90A00087703000877030008DF
:1000B000F50A00081D0B0008770300087703000805
:1000C0007703000877030008770300087703000828
:1000D0007703000877030008770300087703000818
:1000E0007703000877030008770300087703000808
:1000F00077030008770300087703000877030008F8
:1001000077030008770300087703000877030008E7
:1001100077030008450B0008770300087703000801
:1001200077030008770300087703000877030008C7
:1001300077030008770300087703000877030008B7
:1001400000000000000000000000000000000000AF
:1001500077030008E9070008770300083D08000856
:100160007703000877030008770300087703000887
:1001700077030008790B0008770300086B08000874
:100180007703000800F002F800F05EF80AA090E89B
:10019000000C82448344AAF10107DA4501D100F042
:1001A00053F8AFF2090EBAE80F0013F0010F18BFB1
:1001B000FB1A43F00103184788F70000A8F7000076
:1001C0000A444FF0000C10F8013B13F0070408BF7D
:1001D00010F8014B1D1108BF10F8015B641E05D01B
:1001E00010F8016B641E01F8016BF9D113F0080FD0
:1001F0001EBF10F8014BAD1C0C1B09D16D1E58BF62
:1002000001F801CBFAD505E014F8016B01F8016B98
:100210006D1EF9D59142D6D370470000002300240B
:1002200000250026103A28BF78C1FBD8520728BF06
:1002300030C148BF0B6070471FB50FF077F900F071
:10024000C2F81FBD10B510BD00F050FA1146FFF7FF
:10025000F3FF05F0BFFC00F06EFA03B4FFF7F2FF06
:1002600003BC00F031FA00002C4B19680868B0E8B4
:10027000F04F80F30988BFF36F8F4FF0000080F3D9
:10028000118870470000000008480068006880F38B
:1002900008884FF0000080F3148862B661B6BFF39F
:1002A0004F8FBFF36F8F00DF00BF00BF08ED00E08E
:1002B000DFF80C00016841F470010160704700BF75
:1002C00088ED00E0EFF30980BFF36F8F134B1A68DE
:1002D0001EF0100F08BF20ED108A20E9F04F1060CB
:1002E00009B44FF0500080F31188BFF34F8FBFF374
:1002F0006F8F0CF069FB4FF0000080F3118809BC90
:1003000019680868B0E8F04F1EF0100F08BFB0EC95
:10031000108A80F30988BFF36F8F7047FC000020BC
:10032000EFF30580704700000B49D1F800C04A6820
:100330005CF8043B1068184442F8040B8C4528BF55
:10034000A1F1DC0C8A4228BFA1F1DC02C1F800C097
:100350004A6020F00040704758200120094880473B
:1003600009480047FEE7FEE7FEE7FEE7FEE7FEE797
:10037000FEE7FEE7FEE7FEE704480549054A064BAF
:1003800070470000690A000885010008C0200120AC
:10039000C0260120C0220120C02201200B4910B537
:1003A000A1F17C020A4CC2E93712372106E000EBCA
:1003B000104342F82130074B00FB03400B1EA1F114
:1003C0000101F4DC10BD0120E8E70000F81F012066
:1003D000E119D666CD0D01000EB5054614460E4650
:1003E00013A000F02DF9284600F02AF916A000F01D
:1003F00027F9304600F024F915A000F021F900217A
:100400008DF80B100A210DF10A008DF80A1008E092
:1004100094FBF1F201FB124294FBF1F4303200F84C
:10042000012D002CF4DC00F00BF900F0FEF80000C8
:100430002A2A2A20617373657274696F6E2066615F
:10044000696C65643A2000002C2066696C652000A8
:100450002C206C696E65200040EA010310B59B07F3
:100460000FD1042A0DD310C808C9121F9C42F8D01E
:1004700020BA19BA884201D9012010BD4FF0FF30CF
:1004800010BD1AB1D30703D0521C07E0002010BDE5
:1004900010F8013B11F8014B1B1B07D110F8013B71
:1004A00011F8014B1B1B01D1921EF1D1184610BD52
:1004B00040EA0103024630B59B0710D14FF00134EA
:1004C00000E008C208C91D1B9D4315EAC41FF8D0EF
:1004D00013F0FF0102F8011B0DD01B0AF8E711F819
:1004E000013B002B02F8013B05D011F8013B002B2A
:1004F00002F8013BF3D130BD032A40F2308010F006
:10050000030C00F0158011F8013BBCF1020F6244AE
:1005100098BF11F801CB00F8013B38BF11F8013B3F
:10052000A2F1040298BF00F801CB38BF00F8013BEC
:1005300011F0030300F08E80083AC0F0088051F8F3
:10054000043B083A51F804CBA0E80810F5E7121D67
:100550005CBF51F8043B40F8043BAFF30080D20786
:1005600024BF11F8013B11F801CB48BF11F8012B52
:1005700024BF00F8013B00F801CB48BF00F8012B75
:10058000704702F0FF0343EA032242EA024200F00E
:1005900002B84FF000020429C0F0128010F0030CE2
:1005A00000F01B80CCF1040CBCF1020F18BF00F866
:1005B000012BA8BF20F8022BA1EB0C0100F00DB815
:1005C0005FEAC17C24BF00F8012B00F8012B48BF73
:1005D00000F8012B70474FF0000200B51346944617
:1005E0009646203922BFA0E80C50A0E80C50B1F18B
:1005F0002001BFF4F7AF090728BFA0E80C5048BF9F
:100600000CC05DF804EB890028BF40F8042B08BF3C
:10061000704748BF20F8022B11F0804F18BF00F838
:10062000012B704770477047704710B5002000F0ED
:1006300055F8FFF707FEBDE81040012000F044B870
:1006400010B5044602E0641C00F036F8207800285B
:10065000F9D110BD10B5203AC0F00B80B1E81850A8
:10066000203AA0E81850B1E81850A0E81850BFF49C
:10067000F5AF5FEA027C24BFB1E81850A0E818503B
:1006800044BF18C918C0BDE810405FEA827C24BF8F
:1006900051F8043B40F8043B08BF7047D20728BF1D
:1006A00031F8023B48BF11F8012B28BF20F8023B6C
:1006B00048BF00F8012B704708B569468DF8000067
:1006C0000320ABBE08BD000001491820ABBEFEE709
:1006D00026000200004870476020012010B500F09D
:1006E00039F8BDE8104000F02FB870477546FFF7A5
:1006F000F1FFAE4605006946534620F007008546E7
:1007000018B020B5FFF738FEBDE820404FF00006D6
:100710004FF000074FF000084FF0000B21F00701E9
:10072000AC46ACE8C009ACE8C009ACE8C009ACE82C
:10073000C0098D46704710B50446AFF300802046CF
:10074000BDE81040FFF789BD002801D0FFF7BCBF0E
:100750007047000010B5002102A000F013F801203E
:1007600010BD0000534947414252543A2041626E45
:100770006F726D616C207465726D696E6174696F02
:100780006E00000070B505460C460A2000E06D1CA6
:10079000FFF792FF35B128780028F8D102E0641CF9
:1007A000FFF78AFF14B120780028F8D1BDE8704027
:1007B0000A20FFF781BF00BFFEE7000008B5002058
:1007C00000900421074800F088FD50B1054818301A
:1007D000006800F0700000900421024800F0BEFCA8
:1007E00000BF08BD0064004000B587B0002006903F
:1007F00009210F4800F0F0FCC0B101AA00210C480B
:1008000000F0EDFD002306AA01A90A4800680EF0D9
:1008100035F80698012809D1069838B14FF0805074
:1008200005490860BFF34F8FBFF36F8F07B000BD5E
:10083000006800402C00002004ED00E008B5002016
:1008400000900421074800F048FD50B105481830D9
:10085000006800F0700000900421024800F07EFC67
:1008600000BF08BD00680040704710B5402002F08E
:1008700037FF20B1402002F0A9FE03F047FA4FF401
:10088000803002F0A3FE10BD10B50BF0A5FD10BD29
:1008900010B50BF0CBFD10BD70B50346154626E034
:1008A00000BF502484F31188BFF34F8FBFF36F8FC5
:1008B00000BFDC889E88B4420CD0DE881C68A05D36
:1008C000DC88641CDC80DC88B4F5847F07DD0024D0
:1008D000DC8004E0002484F3118800BF09E0087084
:1008E000491C521E002484F3118800BF00BF002A57
:1008F000D6D100BFA81A70BD70B50546074885421D
:100900000AD1074C20680BF0E3FA207100231A4645
:10091000211DE0680DF0B2FF70BD000000500040E6
:100920003404002000BFFEE710B5FFF7F9FC08B162
:10093000012010BD0020FCE708B54FF0FF3000900B
:1009400014480068C068C0F3401090B120211148DD
:1009500000680BF0D3FA01280BD10E4800680BF0A9
:10096000B7FA0090012269460B4800F03AF806F009
:100970008BFE08480068C068C0F3C01040B18021F9
:10098000044800680BF0BAFA012801D106F084FE91
:1009900008BD0000080400200C04002000BFFEE792
:1009A0007047F0B503460C4603F00701C1F107009C
:1009B000042801D9042001E0C1F107000646081D02
:1009C000072801D2002000E0C81E05460120B040E3
:1009D000401E2040A8400127AF407F1E17403843EB
:1009E000F0BD30B500BF502383F31188BFF34F8FA4
:1009F000BFF36F8F00BF19E00B78858804686355DB
:100A000083885B1C83808388B3F5847F01DD0023AA
:100A100083808388C488A34208D1C3885B1CC380B9
:100A2000C388B3F5847F01DD0023C380131EA2F1C8
:100A30000102E1D100BF83F3118800BF30BD000087
:100A400010B500BF0348007808B900F0C5F800BF32
:100A500010BD0000041F012010B50EF089FA012816
:100A600001D00DF0CDFC10BD1848006840F47000B6
:100A7000164908601648006820F00100401C14491F
:100A8000086000BF12480068C0F340000028F9D099
:100A90000F48406820F003000D49486000BF0C4833
:100AA0004068C0F381000028F9D10948006809496D
:100AB0000840074908600020486008634FF41F00A1
:100AC0008860C803014980390860704788ED00E0FC
:100AD00000100240FFFFF2FE10B5012104480AF0A9
:100AE000A6FF18B1012102480AF070FF10BD0000F6
:100AF000002C014010B5402108060AF098FF60B1B3
:100B0000402108060AF062FF4FF080400AF062FFC1
:100B100000214FF080400AF01BFF10BD10B54021AE
:100B200007480AF084FF50B1402105480AF04EFF03
:100B300003480AF04FFF002101480AF009FF10BDE9
:100B40000004004010B50A480A49086008460068D9
:100B5000C068C0F3401048B12021064800680BF07F
:100B6000CDF9012802D10248FFF7C6FE10BD0000F2
:100B7000005000406004002010B5FFF7DDFE10BDFE
:100B800000B587B00020069009210F4800F024FB33
:100B9000C0B101AA00210C4800F021FC002306AAE4
:100BA00001A90A4800680DF069FE0698012809D1DC
:100BB000069838B14FF0805005490860BFF34F8F59
:100BC000BFF36F8F07B000BD006400402800002015
:100BD00004ED00E000BFFEE710B5124C02202061DA
:100BE000606111A0A0611349E1614FF400612162CD
:100BF0000021A1626162E1620BA0A0640E49E16480
:100C0000102121650021A1656165E1650BA1E01D51
:100C1000FFF74EFC0AA12046FFF74AFC2020A071F6
:100C200010BD0000041F01205465726D696E616C77
:100C300000000000F4160120F41E0120525454005C
:100C4000534547474552000002480068C0F3022060
:100C5000704700000CED00E010B5002804DB0A0727
:100C6000130E054A135406E00A07140E034A00F057
:100C70000F031B1FD45410BD00E400E018ED00E08A
:100C800010B5002000F01EF8012000F01BF8022033
:100C900000F018F8FFF7D4FE10BD0000022800DDB8
:100CA0007047064931F8101031B1044931F810107D
:100CB000034A52F82020116100BFF1E79C00002098
:100CC000900000201CB504460F4951F82400012172
:100CD00000F042FE684603F037FE01208DF8070061
:100CE00000208DF8040010208DF80600074830F829
:100CF0001400009004208DF80500054951F82400E7
:100D0000694603F02CFE1CBDA40000209C000020BE
:100D100090000020022800DD7047064931F81010CD
:100D200031B1044931F81010034A52F820205161C2
:100D300000BFF1E79C00002090000020022800DDA9
:100D40007047094931F8101059B1084951F820107D
:100D5000C968054A32F810205140044A52F8202050
:100D6000D16000BFECE700009C0000209000002054
:100D700086B032E04FF0FF3201A9184B18680DF031
:100D80008FFE012829D10199B1F5A27F14D0A1F2DB
:100D9000423129B1032915D0B1F5817F1CD105E07D
:100DA0009DF812100E4AD268518115E09DF814107A
:100DB0000B4AD26811830FE09DF80F10084AD268E1
:100DC000918109E09DF814209DF8151042EA012157
:100DD000034AD268518300BF00BFCBE72800002040
:100DE000D003002086B050E04FF0FF3201A9274B1E
:100DF00018680DF055FE012847D1019901291FD02F
:100E000002292FD0B1F5806F3ED19DF80F209DF8BB
:100E1000101042EA01211E4AD26891839DF81120E8
:100E20009DF8121042EA0121194AD268D1839DF837
:100E300013209DF8141042EA0121164A118023E084
:100E40009DF8141049B99DF812209DF8131042EA3C
:100E500001210F4AD268118003E000210C4AD268B8
:100E6000118011E09DF8141049B99DF812209DF8E9
:100E7000131042EA0121064AD268518003E00021A2
:100E8000034AD268518000BF00BFADE72C000020AC
:100E9000D00300204400002030B50246002000238B
:100EA000146824F002041460146824F00104641C23
:100EB000146000E05B1C546804F001041CB94FF698
:100EC000FF74A342F6D1546804F00104002C3FD013
:100ED0004D78146865F3C71414608D78146865F351
:100EE00086141460CD78146865F3451414600D7988
:100EF000146865F3041414604D79146865F3C30431
:100F000014608D79146865F3820414600C78D569D7
:100F100064F39E75D5610C786508D46965F3DF7458
:100F2000D461146824F001041460002300E05B1C09
:100F3000546804F001041CB14FF6FF74A342F6D1CB
:100F4000546804F001040CB1002002E0012000E02C
:100F5000002030BD30B5024600200023146824F084
:100F600002041460146824F00104641C146000E09E
:100F70005B1C546804F001041CB94FF6FF74A342D3
:100F8000F6D1546804F001045CB30C88641ED56982
:100F900064F30B05D5618D78D46965F31964D46168
:100FA000CD78D46965F31344D4610D79D46965F3C0
:100FB0001654D461146824F001041460002300E086
:100FC0005B1C546804F001041CB14FF6FF74A3428B
:100FD000F6D1546804F001040CB1002002E00120B5
:100FE00000E0002030BD002141708170C1700171AE
:100FF000417181710170704730B50022CC780123B6
:1010000003FA04F2D0F8003223F001035B1CC0F8AD
:101010000032D0F81C329343C0F81C320B7913B164
:10102000012B5AD12CE0D0F80C329343C0F80C328B
:101030008B891C04CD7800F5107343F83540CC78CB
:1010400053F834300C892343CD7800F5107444F8FC
:1010500035304B891C04CD7800F5107303EBC503C4
:101060005C60CC7800F5107303EBC4035B68CC883C
:101070002343CD7800F5107404EBC50463602DE0C4
:10108000D0F80C321343C0F80C32CB881C04CD7856
:1010900000F5107343F83540CC7853F834300C89A0
:1010A0002343CD7800F5107444F835304B891C0487
:1010B000CD7800F5107303EBC5035C60CC7800F5C8
:1010C000107303EBC4035B688C892343CD7800F570
:1010D000107404EBC504636000E000BF00BF4B78F0
:1010E00013B1012B0CD105E0D0F804329343C0F8C2
:1010F000043206E0D0F804321343C0F8043200E0B2
:1011000000BF00BF8B7813B1012B0CD105E0D0F8E4
:1011100014329343C0F8143206E0D0F8143213436B
:10112000C0F8143200E000BF00BF0B783BB1012BC8
:101130000BD1D0F81C321343C0F81C3206E0D0F8B3
:101140001C329343C0F81C3200E000BF00BFD0F84F
:10115000003223F00103C0F8003230BD122935D22D
:10116000DFE801F034090A0B0F0C14171B341F229F
:101170003425282B2E3100BF00BF00BF042242605F
:1011800025E0042242600022826120E00122826088
:101190001DE04FF48072826019E04FF4803282606B
:1011A00015E00822C26012E01022C2600FE008229F
:1011B00002610CE01022026109E00822426006E0B0
:1011C0001022426003E0034A826000E000BF00BFDB
:1011D00070470000010101000246002012296FD271
:1011E000DFE801F06E090D11151D2125292D353976
:1011F0003D45494D515D936903F0010062E09369FB
:10120000C3F340005EE09369C3F380005AE0936942
:10121000C3F302130BB1012000E0002052E0536839
:10122000C3F380004EE0936803F001004AE0936846
:10123000C3F3002046E09368C3F3004042E0D36864
:1012400003F003030BB1012000E000203AE0D36873
:10125000C3F3C00036E0D368C3F3001032E0136973
:1012600003F003030BB1012000E000202AE0136922
:10127000C3F3C00026E01369C3F3001022E05368F3
:10128000C3F3C0001EE05368C3F340031BB95368A7
:10129000C3F300130BB1012000E0002012E09368BB
:1012A000C3F380633BB99368C3F3C0631BB993680E
:1012B000C3F300730BB1012000E0002002E0FFE760
:1012C000002000BF00BF70471AB143690B43436160
:1012D00002E043698B4343617047F0B504460D4615
:1012E00000260027122D6CD2DFE805F06B091623CB
:1012F000303D414243474B4F53575B5F63676069E3
:10130000C0F3C03028B16069C0F3002008B10120EB
:1013100000E00020074656E06069C0F3C03028B105
:101320006069C0F3402008B1012000E000200746BA
:1013300049E06069C0F3C03028B16069C0F3802023
:1013400008B1012000E0002007463CE06069C0F3DE
:10135000C03028B16069C0F3C02008B1012000E0AE
:10136000002007462FE06069C0F3C0372BE000BFC4
:1013700000BF606900F0010725E06069C0F3400725
:1013800021E06069C0F380071DE06069C0F3C00719
:1013900019E06069C0F3001715E06069C0F34017F9
:1013A00011E06069C0F380170DE06069C0F3004789
:1013B00009E06069C0F3404705E0606900F001079B
:1013C00001E0002700BF00BF012F01D00020F0BDC9
:1013D00029462046FFF700FF06463046F7E730B5BE
:1013E00005460C46134605F5D87000EB041000685E
:1013F000C0F380001872187A10B1012813D107E0E9
:1014000005F5D87000EB04100068400D18600BE083
:1014100005F5D87000EB041000686FF0604101EA38
:10142000D000586000E000BF00BF05F5D87000EBA9
:1014300004100068C0F34000587205F5D87000EB46
:101440000410406800F00F00987205F5D87000EBAA
:1014500004104068000AD87405F5D87000EB041039
:101460008068D87205F5D87000EB04108068010A16
:10147000197305F5D87000EB04108068010C5973DE
:1014800005F5D87000EB04108068010E997305F51E
:10149000D87000EB0410C068D87305F5D87000EB65
:1014A0000410C068010A197405F5D87000EB041027
:1014B000C068010C597405F5D87000EB0410C068C1
:1014C000010E99742146284600F09DF830BD10B5F4
:1014D000024604209368C3F380630BB100200CE044
:1014E0009368C3F3C0630BB1012006E09368C3F3B4
:1014F00000730BB1022000E0042004287CD002F528
:10150000C07303EB00131B6803F0010402F5C07302
:1015100003EB00131C600C7A02F5C07303EB00139D
:101520001B6864F3820302F5C07404EB00142360AB
:101530000B7A13B1012B1CD10DE00C8802F5C0739E
:1015400003EB00131B6864F35F5302F5C07404EBF4
:10155000001423600EE002F5C07303EB00131B6858
:101560004C6843EAC40402F5C07303EB00131C602B
:1015700000E000BF00BF4C7A02F5C07303EB00131C
:101580001B6864F3410302F5C07404EB001423608C
:101590008B7A02F5C07404EB0014646863F30304EF
:1015A00002F5C07303EB00135C608B7B1C064B7B66
:1015B00044EA03440B7B44EA0323CC7A234302F539
:1015C000C07404EB0014A3608B7C1C064B7C44EAC3
:1015D00003440B7C44EA0323CC7B234302F5C07411
:1015E00004EB0014E36002F5C07303EB00131B6807
:1015F00023F001035B1C00E004E002F5C07404EB7F
:101600000014236010BD11B1012906D102E020228F
:10161000C26003E02022026100E000BF00BF70470B
:1016200070B586B0044600254FF44070019000204C
:1016300002908DF80C008DF80D0008208DF80E003A
:1016400020788DF80F0061788DF81010A1788DF852
:101650001110E1788DF8121021798DF8131061794D
:101660008DF8141077218DF8151088218DF816103B
:1016700001A90948FFF72BFF064604E06D1CB5F5EC
:10168000803F00D305E03146034800F007F8012809
:10169000F4D100BF06B070BD0068004002460020D3
:1016A00021B1012910D002292AD11BE0936803F04F
:1016B00001033BB19368C3F340030BB1012002E087
:1016C000002000E002201DE09368C3F300233BB13B
:1016D0009368C3F340230BB1012002E0002000E037
:1016E00002200FE09368C3F300433BB19368C3F358
:1016F00040430BB1012002E0002000E0022001E0A5
:10170000002000BF00BF70470349496860F307111C
:10171000014A5160704700000010024003494968C7
:1017200060F30A21014A5160704700000010024036
:101730000349496860F3CD21014A516070470000B8
:1017400000100240012807D10749496D21F03001FE
:101750003031054A516505E00349496D21F03001FA
:10176000014A51657047000000100240052827D249
:10177000DFE800F0030A11181F00134A126861F332
:101780000002114B1A601CE00F4A126861F310420C
:101790000D4B1A6015E00C4A126861F318620A4B8F
:1017A0001A600EE0084A126A61F30002064B1A62E0
:1017B00007E0054A526A61F30002034B5A6200E0F7
:1017C00000BF00BF70470000001002402DE9F0414B
:1017D000014600270022002590460023002400F047
:1017E00065F9064626B1012E12D0022E43D112E031
:1017F0003948406DC0F3402038B13748006BC0F322
:10180000406010B13548086001E03548086035E0B7
:101810003348086032E030484068C0F300482E4842
:101820004068C0F383422C484068C0F341750DB94D
:101830000F2A03D12801401C024400E0921CB8F199
:10184000000F03D127485043086013E02248406846
:10185000C0F3404058B12048406DC0F30137B81C78
:10186000DFF87CC0BCFBF0F05043086002E01C488D
:101870005043086002E01A48086000BF00BF1648E5
:101880004068C0F303131848C45C0868E04048602F
:1018900011484068C0F302231448C45C4868E04023
:1018A000C8600D484068C0F3C2231148C45C486852
:1018B000E040886008484068C0F30073064840680C
:1018C000C0F3813040EA83030A48C45C8868B0FBF7
:1018D000F4F00861BDE8F08100100240006CDC0209
:1018E00000127A0000093D0036F5000846F50008B0
:1018F0004EF5000856F5000810B501460020094BCA
:1019000003EB1142126801F01F040123A3401A40A7
:1019100001F01F040123A3409A4200D000E00120FF
:1019200010BD00000010024030B50024002500E08A
:10193000641C1120FFF7E0FF012802D0B4F5405FDE
:10194000F6D31120FFF7D8FF012801D0002500E0D1
:101950000125284630BD000010B501290DD10E4BE0
:1019600003EB1042126800F01F040123A3401A4346
:10197000094C04EB10431A600CE0074B03EB1042D8
:10198000126800F01F040123A3409A43024C04EBA9
:1019900010431A6010BD00000010024010B568B975
:1019A0001C4B5B6823F480331A4C636023461B6B2B
:1019B00023F0007303F10073236317E0154B5B689A
:1019C00023F4803303F58033124C6360012805D182
:1019D00023465B6823F40033636007E00D4B5B68CC
:1019E00023F4003303F500330A4C6360094B5B6852
:1019F00061F39543074C63600C09064B5B6864F325
:101A00005E73044C636023465B6862F3DF7363605C
:101A100010BD0000001002401348006820F00100D3
:101A2000401C1149086000BF0F480068C0F3400027
:101A30000028F9D00C48406820F003000A494860AB
:101A400000BF09484068C0F381000028F9D106486A
:101A5000006806490840044908600020486008639F
:101A60004FF41F008860704700100240FFFFF2FE35
:101A70000D49496860F301010B4A516000BF00BF86
:101A800000BF00BF00BF00BF00BF00BF00BF00BF5E
:101A900000BF00BF00BF00BF00BF00BF00BF00BF4E
:101AA00000BF00BF704700000010024002484068BD
:101AB000C0F3810070470000001002400A468368AE
:101AC0001B68136083681A6070470246906801685B
:101AD00021B1086893681860084670470020FCE749
:101AE00010B5002406480078012806D10548006892
:101AF000804700200249087000E00624204610BDFF
:101B00003A020020400200202DE9F05F06460D4613
:101B10004FF0000B2888052848D170784FEA00293B
:101B2000B07840EA090909F101001FFA80F9F0785C
:101B3000040230790443012C35DBB4F5FA6F32DA54
:101B4000374600202880012007F8010B2888401C18
:101B5000288004F0070040B12046E11704EB5171E2
:101B6000C910491C01F0FF0805E02046E11704EB0D
:101B70005171C1F3C70807F8018B2888401C2880E1
:101B8000002322464946384601F0ACF98246BAF1B4
:101B9000000F04D0504605F036FD834608E0288843
:101BA0004044288004E04FF0030B01E04FF0030BAA
:101BB0005846BDE8F09F2DE9F05F06460D464FF010
:101BC000000B2888052847D170784FEA0029B078A3
:101BD00040EA090909F101001FFA80F9F0780402CE
:101BE00030790443012C34DBB4F5FA6F31DA37462F
:101BF00000202880022007F8010B2888401C28803C
:101C000004F0070040B12046E11704EB5171C91000
:101C1000491C01F0FF0805E02046E11704EB517173
:101C2000C1F3C70807F8018B2888401C288022468A
:101C30004946384601F0F0F98246BAF1000F04D067
:101C4000504605F0E0FC834608E0288840442880A0
:101C500004E04FF0030B01E04FF0030B5846BDE8E2
:101C6000F09F2DE9F04705460C464FF0000A20880A
:101C7000052838D168784FEA0028A87840EA080893
:101C800008F101001FFA80F8E87806022879064377
:101C9000012E25DB7D2E23DC2F4600202080032013
:101CA00007F8010B2088401C20807006000E07F802
:101CB000010B2088401C20800023324641463846D4
:101CC00001F00EFA8146B9F1000F04D0484605F044
:101CD0009AFC824609E0208800EB4600208004E060
:101CE0004FF0030A01E04FF0030A5046BDE8F087C9
:101CF0002DE9F04705460C464FF0000A20880528DC
:101D000037D168784FEA0028A87840EA080808F137
:101D100001001FFA80F8E878060228790643012EB0
:101D200024DB7D2E22DA2F4600202080042007F8B5
:101D3000010B2088401C20807006000E07F8010B64
:101D40002088401C208032464146384601F022FA65
:101D50008146B9F1000F04D0484605F054FC824694
:101D600009E0208800EB4600208004E04FF0030AE1
:101D700001E04FF0030A5046BDE8F0872DE9FC5F13
:101D800004460D460020009028880A285DDB607814
:101D90004FEA002AA07840EA0A0A0AF101001FFA75
:101DA00080FAE07806022079064360794FEA002B3A
:101DB000A07940EA0B0B0BF101001FFA80FBE079E0
:101DC0000702207A0743607A0190012E3BDB7D2ECB
:101DD00039DC012F37DB792F35DC7900019881421E
:101DE00031D101233A46594604F10A0001F078F94D
:101DF0008146B9F1000F1ED1A0460020288017208F
:101E000008F8010B2888401C28807006000E08F88E
:101E1000010B2888401C288000233246514640464A
:101E200001F05EF98146B9F1000F04D12888022142
:101E300001FB06002880B9F1000F06D0484605F0E6
:101E4000E2FB009001E0032000900098BDE8FC9FB9
:101E500070B505460C46064802880649681CFEF720
:101E60004BFB03480088401C2080002070BD000010
:101E7000B603002031F900202DE9F84304460F464F
:101E80004FF000083888052829D160780502A0782D
:101E90000543681C85B22079F0B9E078FF2801D0AD
:101EA000E078C8B900208DF80100E078FF2803D160
:101EB00001208DF8000002E000208DF800000123D1
:101EC0001A462946684601F00DF806464EB13046DE
:101ED00005F099FB804604E04FF0030801E04FF065
:101EE00003084046BDE8F8832DE9F04104460F465B
:101EF0004FF000083888052812D160780502A078D4
:101F00000543681C85B201231A462946E01C01F0EE
:101F1000E7F8064636B1304605F075FB804601E02D
:101F20004FF003084046BDE8F0812DE9F05F05461B
:101F30000E464FF0000B3088052839DD687807021F
:101F4000A8780743781C87B2E8780402287904430C
:101F500095F805A004F0070040B12046E11704EB16
:101F60005171C910491C01F0FF0805E02046E11736
:101F700004EB5171C1F3C708012C16DBB4F5F66F01
:101F800013DCD04511D1012322463946A81D00F0AB
:101F9000A9FF8146B9F1000F04D0484605F033FB94
:101FA000834607E00520308004E04FF0030B01E09A
:101FB0004FF0030B5846BDE8F09F2DE9F04704466B
:101FC0000E464FF0000A3088062828DB60780702AA
:101FD000A0780743781C87B2E07805022079054392
:101FE00094F80590012D17DB782D15DC6806000E9E
:101FF000484511D101232A463946A01D01F070F849
:102000008046B8F1000F04D0404605F0FCFA824645
:1020100007E00520308004E04FF0030A01E04FF0B4
:10202000030A5046BDE8F0872DE9F04705460C4607
:1020300090469946089F00261CB1012C01DBF72C25
:1020400001DD02262EE019480470022D1CD118482B
:102050001849086018481949086019481949086062
:1020600019481A490860002019490860FF200F49E3
:1020700008700220174908700120174908700020D5
:1020800001F0C0F8064601E0022600BF00BF4EB9CD
:102090000BF0E8FF08B9032604E00E4805700120A4
:1020A0000D4908703046BDE8F08700003802002076
:1020B00091320008400200209332000844020020C0
:1020C0001932000848020020613200083C0200205A
:1020D0004C020020390200203A02002010B50024F2
:1020E00006480078012806D105480068804700208E
:1020F0000249087000E00624204610BDF3020020CB
:10210000F80200202DE9F84F054689464FF0000AF5
:102110000BF05EFF00B13EE0B9F80000022838DBAA
:1021200068460AF05FF800984078060200988078C8
:102130000643701C86B20098C078040200980079AB
:10214000044304F0070038B12046E11704EB517155
:10215000C910491CCFB205E02046E11704EB5171CC
:10216000C1F3C707012C11DB6878B8420ED10023F8
:1021700022463146A81C00F01FFC8046B8F1000F33
:1021800009D0404605F03FFA824604E04FF0030ACA
:1021900001E04FF0030A5046BDE8F88F2DE9F84FF3
:1021A000054689464FF0000A0BF012FF00B13DE0F2
:1021B000B9F80000022837DB68460AF013F80098E7
:1021C00040780602009880780643701C86B200981A
:1021D000C078040200980079044304F0070038B185
:1021E0002046E11704EB5171C910491CCFB205E03C
:1021F0002046E11704EB5171C1F3C707012C10DB36
:102200006878B8420DD122463146A81C00F074FC13
:102210008046B8F1000F09D0404605F0F4F9824637
:1022200004E04FF0030A01E04FF0030A5046BDE816
:10223000F88F2DE9F843054688464FF000090BF06A
:10224000C7FE00B12CE0B8F80000022826DB684683
:1022500009F0C8FF0098407806020098807806438D
:10226000701C86B20098C07804020098007904437C
:10227000012C10DB6000697888420CD100232246D3
:102280003146A81C00F0A2FC07464FB1384605F0C5
:10229000BAF9814604E04FF0030901E04FF0030969
:1022A0004846BDE8F8832DE9F843054688464FF0D7
:1022B00000090BF08DFE00B12BE0B8F800000228F9
:1022C00025DB684609F08EFF0098407806020098EA
:1022D00080780643701C86B20098C078040200988B
:1022E00000790443012C0FDB6000697888420BD130
:1022F00022463146A81C00F0C5FC07464FB13846BF
:1023000005F081F9814604E04FF0030901E04FF048
:1023100003094846BDE8F8832DE9F84F054689468C
:102320004FF0000B0BF054FE00B144E0B9F8000090
:10233000022840DB684609F055FF00984078060205
:10234000009880780643701C86B20098C078070217
:10235000009800790743009840794FEA00280098D8
:10236000807940EA080808F101001FFA80F8009817
:10237000C0794FEA002A0098007A40EA0A0A7800F9
:102380006978884215D101235246414600980A30A7
:1023900000F01CFC044634B900233A463146A81C20
:1023A00000F014FC044634B1204605F02CF98346B5
:1023B00001E04FF0030B5846BDE8F88F2DE9F843D4
:1023C00004460F464FF000083888052829D1607868
:1023D0000502A0780543681C85B22079F0B9E07841
:1023E000FF2801D0E078C8B900208DF80100E0781E
:1023F000FF2803D101208DF8000002E000208DF8B5
:10240000000001231A462946684600F0D5FA064620
:102410004EB1304605F0F7F8804604E04FF003086F
:1024200001E04FF003084046BDE8F8832DE9F04194
:1024300004460F464FF000083888052812D160780E
:102440000502A0780543681C85B201231A46294677
:10245000E01C00F0BBFB064636B1304605F0D3F871
:10246000804601E04FF003084046BDE8F0812DE9C9
:10247000F84F054689464FF0000BB9F800000528D3
:1024800003D00BF0A5FD002837D0684609F0AAFE5E
:1024900068780602A8780643701C86B2E8780402C1
:1024A00028790443009890F805A004F0070038B19B
:1024B0002046E11704EB5171C910491CCFB205E069
:1024C0002046E11704EB5171C1F3C707012C11DB62
:1024D00057450FD10123224631460098801D00F058
:1024E0006BFA8046B8F1000F09D0404605F08BF832
:1024F000834604E04FF0030B01E04FF0030B584616
:10250000BDE8F88F2DE9F84F82460F464FF00009DD
:102510003888052802D00BF05BFD38B3684609F017
:1025200061FE009840780402009880780443601CA3
:1025300084B20098C078050200980079054300989D
:1025400090F80580680040450DD101232A462146B8
:102550000098801D00F03AFB06464EB1304605F06B
:1025600052F8814604E04FF0030901E04FF00309FF
:102570004846BDE8F88F0000014800787047000029
:10258000F20200202DE9F04104460D4616461F4692
:102590004FF00008F4B91A481A4908601A481B4954
:1025A00008601B481B4908601B481C490860002044
:1025B0001B4908601B481C4908601C481C490860EE
:1025C0001C481D4908603A463146284600F038F953
:1025D000804602E04FF0020800BF00BFB8F1000FD4
:1025E0000AD10BF005FB10B94FF0030802E00120FF
:1025F0001249087009F0FCFD4046BDE8F08100007A
:102600007D290008F8020020A1290008FC02002012
:10261000E5280008F40200209528000800030020A7
:102620000403002019DE00080803002041DF000831
:102630000C030020ADDE000810030020F302002090
:102640002DE9F84300277548007830B173480078C9
:10265000032802D00620BDE8F88368460BF09AFAFA
:10266000002877D0BDF80000042829D004DC012818
:1026700007D002286FD10AE008286DD01028F9D1C0
:1026800090E003206549087009F074FEC2E0644AD6
:1026900064496548654B1B68984707464FB909F080
:1026A000EBFA61490978884203D104200BF0B2FAB1
:1026B00005E0012009F07CFE10200BF0ABFAA9E048
:1026C0005848006800785A49087001205949087034
:1026D00057480078C01120B152480068407808700F
:1026E0003FE000243AE0544810F8340000B937E0E5
:1026F000514810F834004E49097888422DD1012004
:1027000009F044FE0BF064FCB0B109F0DBFB444976
:10271000088001250DE0E8B209F044FE464800EBD0
:10272000C4003F4942683F480068904741490870EB
:102730006D1C102DEFDD09E03F4800EBC400384967
:1027400042683848006890473A490870002009F00C
:102750001DFE05E05FE05CE012E0641C102CC2DBB3
:1027600000BF3448007830B1022009F021FE10206B
:102770000BF050FA03E009F005FD09F0FBFD49E01C
:10278000284809F02FFD09F09DFB804609F074FAF6
:1027900081464246234801684846284B1B689847B3
:1027A000074637E0FFF7E8FE06461E4809F01AFD27
:1027B00026B1012E0FD0022E27D119E009F082FB9D
:1027C000804609F059FA8146424616480168484653
:1027D00009F0FCFC19E009F075FB804609F04CFAA1
:1027E000814642460F480168484609F0E3FC0CE088
:1027F00009F068FB804609F03FFA814642460948E5
:102800000168484609F0C8FC00BF00BF09F0B2FDEE
:1028100000E000BF00BF00201DE70000F302002021
:10282000A20300209C030020A0030020000300203E
:10283000A1030020A40300201C030020F4020020B8
:102840002DE9F04107460C4616464FF00008FEF70A
:102850001BF833460822214638460BF001FA10B91E
:102860004FF003080EE0B4F5964F01D9232503E09D
:1028700060000749B1FBF0F5A8B20BF09DFA08B96A
:102880004FF00308FEF704F84046BDE8F081000071
:10289000A07F17002DE9F04104460D46164600279B
:1028A000FDF7F2FF0D480088042810DB0B48018873
:1028B0000B4809F0EBFA50B9094800782070074836
:1028C0000088C01E30800648401C286000E00527B4
:1028D000FDF7DEFF3846BDE8F0810000B2030020BE
:1028E00031F800202DE9F04104460E4617464FF01E
:1028F0000008102C02DD0220BDE8F081FDF7C4FFC6
:1029000019480078012829D1701E18490860012053
:102910001749088015480068047008460088384444
:102920000880084601881148006809F0AFFA05469A
:102930000F490888411C0E4B19800E490D542A126C
:1029400019460888411C19800A490A5401200A497D
:1029500008700121002009F057FC01E04FF0050844
:10296000FDF796FF4046C7E7A9030020AC0300200F
:10297000B003002034F70020A803002010B5FDF7B5
:1029800083FF0020054908700021012009F03CFC6C
:1029900009F0C6FCFDF77CFF10BD0000A903002074
:1029A00010B5FDF771FF0021084609F02DFC09F074
:1029B0007DFCFDF76DFF10BD2DE9FF5F05460E465E
:1029C00014469A46002003902046E11704EB51710B
:1029D000C910491C1FFA81F809F04EF9401E4449FC
:1029E00001EBC0090020029040200190414800887E
:1029F00000904FF0010A701E86B20298864271DB89
:102A00003219DDE90110084482426BDC0099711A29
:102A100088B2C11700EB5171CF100099711A88B2BA
:102A2000C11700EB5171C910A0EBC1011FFA81FB66
:102A3000BAF1000F03D0BAF1010F51D126E00EE038
:102A400039467A1C97B201EB0900082259460BF06F
:102A5000DDFB05F8010BA8F101001FFA80F8B8F1C1
:102A6000000FEDDC6D1E2046E11704EB5171C9101B
:102A7000A4EBC1018CB22878C4F108018840287009
:102A80002878C4F108010841287029E00EE015F803
:102A9000013B39467A1C97B201EB090008225946DE
:102AA0000BF0C9FBA8F101001FFA80F8B8F1010F83
:102AB000EDDC2046E11704EB5171C910A4EBC10114
:102AC0008CB264B115F8013BE2B2394607F1010C52
:102AD0001FFA8CF701EB090059460BF0ACFB00BF65
:102AE00002E0FFE701200390039804B0BDE8F09FE7
:102AF00062FB0020E20300202DE9FE4F06460D4652
:102B00001446002002902046E11704EB5171C910D1
:102B1000491C1FFA81F909F0AFF8401E294901EB61
:102B2000C00A4FF0000B4020019027480088009019
:102B3000681E85B25D4540DB2919019858448142E1
:102B40003BDC0099691A88B2C11700EB5171CF10B4
:102B50000099691A88B2C11700EB5171C910A0EB36
:102B6000C1011FFA81F80EE016F8013B39467A1CC4
:102B700097B201EB0A00082241460BF05CFBA9F179
:102B800001001FFA80F9B9F1010FEDDC2046E117D1
:102B900004EB5171C910A4EBC1018CB27CB116F8E1
:102BA000013BE2B2394607F1010C1FFA8CF701EB49
:102BB0000A0041460BF03FFB01E001200290029821
:102BC000BDE8FE8FE2FA0020E00300202DE9FC5F63
:102BD00004460F4616460020019009F04DF8401EAD
:102BE00000EBC00101EB0010244901EBC0084FF0DD
:102BF000000A4FF0640B2248008800904FF0010952
:102C0000781E87B2574534DBB8190AEB0B018842AE
:102C10002FDC0098381A85B2B9F1000F03D0B9F152
:102C2000010F25D110E00CE038F81500001204F86F
:102C3000010B18F8150004F8010B681C85B2701E12
:102C400086B2002EF0DC13E00FE014F8011B08023E
:102C500028F8150014F8010B38F81510084328F867
:102C60001500681C85B2701E86B2002EEDDC00BF18
:102C700001E0012001900198BDE8FC9F620801205D
:102C8000E60300202DE9F84F04460D4617460020C4
:102C9000009008F0F1FF401E00EBC00101EB0010B6
:102CA000174901EBC0084FF000094FF0640A1548BE
:102CB000B0F800B0681E85B24D451BDBE81909EB82
:102CC0000A01884216DCA5EB0B0086B20FE014F86F
:102CD000011B080228F8160014F8010B38F816102A
:102CE000084328F81600701C86B2781E87B2002FA1
:102CF000EDDC01E0012000900098BDE8F88F0000B5
:102D0000E2FB0020E40300202DE9F84306460C46D0
:102D100015461F464FF00008102E02DD4FF0020846
:102D200022E038460BF05AF910B94FF005081BE0C5
:102D3000684609F057FA304609F034FB0320009941
:102D4000087020120099487000998C702812009920
:102D5000C87000990D71052009F030FB08200AF0B9
:102D600059FF00F005F880464046BDE8F8830000B2
:102D700038B50024601E002301224FF4F07100904A
:102D80000C4800680AF05AFE0546202D07D0402D59
:102D900006D0802D06D0B5F5807F07D104E005E090
:102DA000042403E0032401E0062400BF00BF204602
:102DB00038BD00000004002038B500253F480078E9
:102DC00008B1062038BD68460BF024F9002873D0FE
:102DD0009DF80000012806D0022805D0042818D04C
:102DE000082868D166E066E0354A36493648374BF0
:102DF0001B68984705465DB933480078344909781F
:102E0000884202D03048007810B904200BF03CF919
:102E100051E02C48006800782E49087001202E49A6
:102E20000870002417E02D4810F8340000B914E0B1
:102E30002A4810F834002749097888420AD12748DF
:102E400000EBC4001E4942681E48006890472249B2
:102E5000087002E0641C102CE5DB00BF1A48007803
:102E600030B31D480078C8B10020154908801948C2
:102E7000007840F08001124802880088401C104B06
:102E80001880104800688154134801781846028859
:102E90000088401C18800B4800688154084802884C
:102EA000084801680A4800780D4B1B68984705469A
:102EB00001E001E000BF00BF002083E73A020020EC
:102EC000EA020020E4020020E8020020480200207C
:102ED00038020020E9020020EC02002064020020F9
:102EE0003C0200202DE9FF5F05460E4614469A4637
:102EF000002003902046E11704EB5171C910491CD2
:102F00001FFA81F8DFF8089100200290402001901C
:102F1000404800880090701E86B20298864271DB9D
:102F20003219DDE90110084482426BDC0099711A04
:102F300088B2C11700EB5171CF100099711A88B295
:102F4000C11700EB5171C910A0EBC1011FFA81FB41
:102F5000BAF1000F03D0BAF1010F51D126E00EE013
:102F600039467A1C97B201EB0900082259460BF04A
:102F70004DF905F8010BA8F101001FFA80F8B8F12E
:102F8000000FEDDC6D1E2046E11704EB5171C910F6
:102F9000A4EBC1018CB22878C4F1080188402870E4
:102FA0002878C4F108010841287029E00EE015F8DE
:102FB000013B39467A1C97B201EB090008225946B9
:102FC0000BF039F9A8F101001FFA80F8B8F1010FF0
:102FD000EDDC2046E11704EB5171C910A4EBC101EF
:102FE0008CB264B115F8013BE2B2394607F1010C2D
:102FF0001FFA8CF701EB090059460BF01CF900BFD2
:1030000002E0FFE701200390039804B0BDE8F09FC1
:10301000C4030020C20300202DE9FE4F05460E46E2
:103020001446002002902046E11704EB5171C910AC
:10303000491C1FFA81F9284801904FF0000A4020EE
:1030400000902648B0F800B0701E86B256453DDBB1
:10305000311900985044814238DCA6EB0B0188B24C
:10306000C11700EB5171CF10A6EB0B0188B2C1174D
:1030700000EB5171C910A0EBC1011FFA81F80EE0FD
:1030800039467A1C97B2019A8818082241460BF0FB
:10309000BDF805F8010BA9F101001FFA80F9B9F19B
:1030A000000FEDDC6D1E2046E11704EB5171C910D5
:1030B000A4EBC1018CB22878C4F1080188402870C3
:1030C0002878C4F108010841287001E0012002902D
:1030D0000298BDE8FE8F0000BA030020B80300206C
:1030E0002DE9F04704460D461E460020274B0027D9
:1030F0004FF0640CDFF89890B9F80080A5F1010951
:103100001FFA89F5BD423EDB05EB020907EB0C0A0D
:10311000D14538DCA5EB08091FFA89F116B1012E5B
:1031200030D115E011E033F811904FEA292904F865
:10313000019B13F8119004F8019B01F101091FFA9A
:1031400089F1A2F101091FFA89F2002AEBDC19E0EA
:1031500015E014F801AB4FEA0A2923F8119014F88E
:10316000019B33F811A049EA0A0923F8119001F1F3
:1031700001091FFA89F1A2F101091FFA89F2002A57
:10318000E7DC00BF00E00120BDE8F0871AFA00206C
:10319000CE0300202DE9F04303460020174D002602
:1031A0006427DFF85C80B8F800C0A1F101081FFABD
:1031B00088F1B1421FDB01EB020806EB0709C845A5
:1031C00019DCA1EB0C081FFA88F411E035F8148023
:1031D0004FEA282803F8018B15F8148003F8018BB7
:1031E00004F101081FFA88F4A2F101081FFA88F21D
:1031F000002AEBDC00E00120BDE8F08352F900205A
:10320000CC03002070B50446002520460AF066FF76
:1032100000B90325284670BD2DE9FC4104460D4642
:1032200016464FF00508694601A80AF047FF90B11D
:103230000198807807020198C07807436FB9019818
:10324000C01D2860BDF80000C01F30804FF000088E
:10325000FF20207001E04FF005084046BDE8FC81EA
:103260002DE9F04781460E4614460027F51FE01D64
:103270001FFA80F8601C000A2871601C68714146C2
:1032800028460AF065FF00B905273846BDE8F087F3
:10329000704710B509F098F810BD0000034909689F
:1032A00060F3C711014A11607047000000800240BE
:1032B0000349096860F34611014A11607047000034
:1032C000008002400349096860F31041014A11601F
:1032D000704700000080024010B586B00024142121
:1032E00001A8FDF778F92148006964F385001F49BA
:1032F000086101A8FEF76AFA1D490298884205D3C1
:103300001C490298884201D2022426E019490298F9
:10331000884205D318490298884201D203241CE050
:1033200015490298884205D314490298884201D26F
:10333000002412E011490298884205D310490298EE
:10334000884201D2012408E00D490298884204D342
:103350000C490298884200D804240448006964F3A8
:1033600085000249086106B010BD000000800240DF
:10337000002D3101C00E16020087930300E1F50510
:1033800080D1F008001C4E0E00B50346587800F0BE
:103390002FF89878FFF78CFFD878FFF77FFF187920
:1033A00000F078FB587900F0AFFAD87900F0DCFA39
:1033B000187A00F04FFB987AFFF784FFD87A00F074
:1033C00099FA187B00F0AAFA587B00F08BFC00BD3C
:1033D00000210170C17081708172417081714172F0
:1033E000C17241710173C171017201714173704702
:1033F0000349096860F30411014A11607047000035
:103400000080024008B508490968C9084FF47A727B
:10341000B1FBF2F14143009100BF00BF00994A1E89
:1034200000920029F9D108BDF800002002783B493C
:10343000096862F35961394A11604279374909686C
:1034400062F38601354A116082783449096862F373
:103450005641324A116002793049096862F30D2100
:103460002E4A1160C2782D49096862F310412B4A37
:10347000116042782949096862F3D751274A1160DF
:1034800082792649096862F34101244A1160C279B0
:103490002249096862F38F31204A1160027A1F497C
:1034A000896962F39A611D4A9161427A1B4989696F
:1034B00062F35961194A9161827A1849896962F304
:1034C0001861164A9161C27A1449896962F35551AB
:1034D000124A9161027B1149896962F390310F4A66
:1034E0009161427B0D49896962F3C7110B4A916171
:1034F000827B0A49896962F38611084A9161C27B1D
:103500000649896962F3C401044A9161027C034956
:10351000896962F38201014A91617047009002401B
:1035200070B505461446002015B1012D45D120E0A7
:10353000234E3160002015E001EB40124FF480165D
:103540001660C0EBC01606EB460604EB86069660D6
:103550005E1E864204D901EB40162036D66000E09C
:10356000D160401C9842E7D3164E3669154E316142
:1035700023E0154E3160002018E001EB40124FF0BF
:103580000046166044F2F4565660C0EBC01606EBD7
:10359000460604EB860696605E1E864204D901EB61
:1035A00040162036D66000E0D160401C9842E4D33B
:1035B000044EF668034EF16000BF00BF70BD00000E
:1035C000E800002000900240EC0000200149486122
:1035D000704700000090024001460020024A5269F4
:1035E0000A4002B101207047009002400F2872D2B9
:1035F000DFE800F0080F161D242B323940474E55E6
:103600005C636A00354AD26961F30002334BDA61C8
:1036100061E0324AD26961F34102304BDA615AE02B
:103620002E4AD26961F382022C4BDA6153E02B4AB5
:10363000D26961F3C302294BDA614CE0274AD269AF
:1036400061F30412254BDA6145E0244AD26961F343
:103650004512224BDA613EE0204AD26961F38612BC
:103660001E4BDA6137E01D4AD26961F3C7121B4B6A
:10367000DA6130E0194AD26961F30822174BDA6146
:1036800029E0164AD26961F34922144BDA6122E03B
:10369000124AD26961F38A22104BDA611BE00F4AA9
:1036A000D26961F34D320D4BDA6114E00B4AD269F5
:1036B00061F38E32094BDA610DE0084AD26961F399
:1036C000CF32064BDA6106E0044AD26961F3104258
:1036D000024BDA6100BF00BF70470000009002405B
:1036E00001460020402925D00EDC082933D006DC15
:1036F00001291DD002292DD0042942D119E0102919
:103700002AD020293DD128E0B1F5806F29D008DCEE
:10371000802923D0B1F5807F21D0B1F5007F30D151
:103720001EE0B1F5005F1DD0B1F5804F29D102E058
:1037300000BF00BF00BF144A52690A404AB1124A92
:10374000D2690A402AB1104A526902F4803202B1A9
:10375000012017E000BF00BF00BF00BF00BF00BFD7
:1037600000BF00BF084A52690A404AB1064AD269FE
:103770000A402AB1044A526902F4004202B101200F
:1037800000E000BF00BF70470090024038B505461A
:103790000C46002000900A2D55D2DFE805F0050CFC
:1037A000131A2128383F464D2848806964F34100A8
:1037B0002649886147E02548806964F382002349EF
:1037C000886140E02148806964F386101F49886160
:1037D00039E01E48806964F3C7101C49886132E0F3
:1037E0001A48806964F34D30184988612BE0174806
:1037F000806964F314501549886108468069009017
:103800000120FFF7FFFD1149009888611BE00F4878
:10381000806964F355500D49886114E00B48806954
:1038200064F31860094988610DE00848806964F311
:1038300059600649886106E00448806964F39A602B
:103840000249886100BF00BF38BD000000900240FF
:1038500000210170817141710172C17041738172E7
:1038600081730174C1714172012181700021C173A2
:10387000C17201210171002101734170704721B1B2
:10388000426822F00042426003E0426842F0004297
:10389000426070470448006800F0010008B1012050
:1038A00070470020FCE700000090024003480068D9
:1038B00020F00100401C0149086070470090024060
:1038C0000349096860F3CB21014A11607047000089
:1038D000008002400349096860F38E31014A11609B
:1038E000704700000080024001480068806870470F
:1038F000E80000200349096860F35341014A116060
:1039000070470000008002400349096860F38A2183
:10391000014A1160704700000080024003490968B5
:1039200060F39651014A1160704700000080024028
:103930000179427941EA02220A49096C62F30F01D6
:10394000084A1164C1780906827841EA0241427846
:1039500041EA022102781143024A526C014A516441
:1039600070470000008002400349096860F30C3191
:10397000014A1160704700000080024030B50346E4
:103980000C4600211648006963F3CF20144D2861CE
:103990002846006964F38A1028612846006920F0EF
:1039A000020028612846006920F00100401C2861BF
:1039B00000BF491C0A48406910800948006900F0AE
:1039C000010010B107488142F3D30648814201D17A
:1039D000002030BD0248406910800120F9E7000056
:1039E00000800240FFFF0F0030B503460C46002167
:1039F0001648406962F30F00144D6861284600695B
:103A000063F3CF2028612846006964F38A10286197
:103A10002846006920F00200801C286128460069C1
:103A200020F00100401C286100BF491C07480069C4
:103A300000F0010010B106488142F6D304488142EB
:103A400001D1002030BD0120FCE7000000800240D1
:103A5000FFFF0F000349096860F34D31014A11600F
:103A6000704700000080024038B5044600200090F6
:103A70000748006864F3820005490860084600684A
:103A800000900120FFF7BEFC01490098086038BD96
:103A9000008002400349096860F34921014A11602E
:103AA000704700000080024027480068006800F06E
:103AB000004008B10020704723480068008800F4E7
:103AC000807008B321484069401C2049486108467D
:103AD0004069012802D11C480068C8601A48006883
:103AE0001A490861184800680068C0F30D40001FBB
:103AF00008600846C0688068486013480068C0686D
:103B0000114908600120D6E70F480068008800F4DA
:103B1000007068B101200D4948610B480068C86019
:103B20000020086108480068C0680749086009E08B
:103B300006484069401C0549486103480068C06860
:103B4000014908600020B6E7EC000020185800206A
:103B500010B5012000F024F801210520FFF716FE22
:103B60000120FFF781FF01210420FFF70FFE012153
:103B70000020FFF70BFE10BD10B500210420FFF759
:103B800005FE00210846FFF701FE0020FFF76CFF4D
:103B900001210520FFF7FAFD002000F001F810BD1B
:103BA00038B50446002000900748006864F3C3005D
:103BB000054908600846006800900120FFF722FCD4
:103BC00001490098086038BD0080024070B5044685
:103BD0000025002641480068006800F0004008B158
:103BE000002070BD0CB90020FBE740F2F450844285
:103BF00008D9B4FBF0F5B4FBF0F100FB114010B1B3
:103C00006D1C00E00125012D1AD1344800680068C0
:103C100040F04050314909680860C4F30C002F4956
:103C2000096848602D480068006840F000402B4952
:103C30000968086029480068C068284908603EE0B3
:103C400000263AE025480068006820F040502349EB
:103C5000096808603EB921480068006840F080505B
:103C60001E490968086040F2F4501C490968486020
:103C7000681EB04213D119480068006840F0005037
:103C8000164909680860681EC0EBC01000EB4000D0
:103C9000A4EB8000C0F30C001049096848600F488D
:103CA0000068006840F000400C49096808600B4853
:103CB0000068C06809490860761CAE42C2D304207F
:103CC000FFF78AFC38B10420FFF780FC0448406805
:103CD000002003494860012083E70000E80000203D
:103CE000009002400349096860F3D751014A11600E
:103CF0007047000000800240044606E0204600F0C5
:103D000024FD4FF4FA7008F08DFCF7E708B50020A9
:103D100000906946074800680AF040FE009838B1F4
:103D20004FF0805004490860BFF34F8FBFF36F8F8F
:103D300008BD00007C00002004ED00E0064635468A
:103D400000BF4FF0FF310B4800680AF05DFF01280B
:103D5000F7D100BF284601F0F7FD04463CB12946E3
:103D600020462A69904710B1204602F0A9FD002C98
:103D7000F0D1E6E77C00002070B50546002411E094
:103D800004EB4400094901EBC000067D4EB104EB91
:103D9000440001EBC0008068A84202D1204600F038
:103DA000BBF8641C0A2CEBDB70BD000044F600205D
:103DB0002DE9FE4F0546884616464FF00A09CA46C9
:103DC0000A270024BB46002002900190009000BF0B
:103DD00062E004EB44004F4A02EBC000017D0A2F71
:103DE00002D109B9274655E0002953D0A5B104EB0B
:103DF0004402484B03EBC2022868526890420BD140
:103E00003EB104EB44001A4602EBC0008068B042A9
:103E100002D12046BDE8FE8F012928D104EB4400E1
:103E20003C4A52F8300080B104EB440002EBC00081
:103E3000428A029882422DDBA34604EB4400354AB5
:103E400002EBC000408A029024E004EB4400314AB7
:103E500002EBC000428A019882421BDBA14604EBC0
:103E600044002C4A02EBC000408A019012E0022973
:103E700010DB04EB4400274A02EBC000428A0098A2
:103E8000824207DBA24604EB4400224A02EBC00058
:103E9000408A0090601C04B20A2C9ADB08F00200F1
:103EA00020B90A2F05D108F0010010B94FF0FF30FA
:103EB000B0E70A2F01DA3C4614E0BAF10A0F01DA42
:103EC00054460CE0B9F10A0F01DA4C4607E0BBF1A9
:103ED0000A0F01DA5C4602E04FF0FF309AE7204615
:103EE00000F01AF835B104EB44010A4A02EBC101B3
:103EF00028684860002004EB4401064A02EBC10137
:103F0000488204EB4400114601EBC0008660204665
:103F100080E7000044F6002010B5044604EB44009E
:103F20000C4951F8300060B104EB4401094A52F8E1
:103F3000310002F0C5FC002004EB4401054A42F8C0
:103F40003100002004EB4401024A02EBC101087574
:103F500010BD000044F60020F0B587B007460D46BE
:103F600000BF0DB907B0F0BD00BF7C682088B0F578
:103F7000807F08D12079062805D16079042802D1F4
:103F80006088082803D0384602F09AFCEAE7D4F8A3
:103F90000E000690A0690590686808B9002607E041
:103FA00005986968884201D1012000E0002006469A
:103FB0000EB1012000E00220034604F1080206A928
:103FC000284600F0A7FAE088B0F5807F03D0B0F56E
:103FD000007F15D113E086B1022206AB04F1080080
:103FE000291DCDE90232CDE9001005F12603024674
:103FF0002231284600F0B6F900E000BF01E000E001
:1040000000BF00BF384602F05BFC00BFAAE700001B
:104010002DE9FE430446894615462F462146286869
:1040200000F084FE10B1DFF8248184E0287800F0ED
:10403000F000E02816D101208DF8040000208DF852
:1040400005005E208DF80600687800F07F008DF88E
:104050000700A8788DF80800E8788DF809000DF1C0
:10406000040867E02868A1680840D4E901121140FB
:1040700088420ED0288880B24FF6A961884208D0C5
:10408000E06810B104F10C0703E06FF00300BDE835
:10409000FE832F48007800EB40002E4901EBC00062
:1040A000007D02281ADB2A48007800EB400001EB73
:1040B000C0008068A04211D12549097801EB410177
:1040C000244A02EBC10138684968884206D1204879
:1040D00002784946204600F03FF8D8E7002621E064
:1040E00006EB46001B4901EBC000007D022817DBF0
:1040F00006EB460001EBC0008068A04210D106EB41
:104100004601144A02EBC10138684968884207D168
:104110000F48067032464946204600F01DF8B6E7C3
:10412000701CC6B20A2EDBDB4A463946204600F038
:104130006DF8ACE700BF4FF40060434604F126027F
:1041400049460090204600F0A5FAA0E76EF5000869
:104150002C02002044F60020F8B505460E46144611
:1041600004EB4400284901EBC000007D022839D14E
:1041700004EB440001EBC000408AB0F58E7F11DDF6
:1041800004EB44000A4602EBC000011D284600F083
:1041900031F938BB032004EB44011B4A02EBC10197
:1041A00008751FE004EB4400174901EBC000408A8A
:1041B000B0F5877F16DB04EB44000B4603EBC00031
:1041C00000F10C0204EB440003EBC000011D284683
:1041D00000F01CF930B9032004EB44010A4A02EB59
:1041E000C10108754FF40060009004EB44000649DB
:1041F00001EBC00000F10C0305F126023146284610
:1042000000F048FAF8BD000044F600202DE9FE4F0A
:1042100080460D46164608F1260A4FF0FF30029000
:10422000002001904146286800F080FD38B92878C8
:1042300000F0F000E02802D00DB1286818B96FF046
:104240000F00BDE8FE8F424601212846FFF7B0FD72
:104250008146B9F1000F02DA4FFA89F0F1E709F06F
:10426000FF0404EB44003D4901EBC000007D70B940
:104270000120019004EB4401384A02EBC1010875AA
:1042800004EB4400114601EBC000C0F8088001981F
:1042900000B93EB92946404600F0ACF802900EB98C
:1042A0000298CEE704EB44002C4901EBC000007DEE
:1042B000022811DB2A4804704FF40060009004EBE0
:1042C000440001EBC00000F10C0352463146404669
:1042D00000F0E0F902903FE004EB44001F4901EBDD
:1042E000C000007D012837D14FF0000B374607E0B2
:1042F000387B00F0400010B14FF0010B02E03F6846
:10430000002FF5D100BFBBF1000F07D032464FF4AC
:1043100020710E2002F028FA074603E0374638469F
:1043200002F0A0FBA7B104EB44000C4951F83000A7
:1043300030B104EB4401094A52F8310002F0C0FAEE
:1043400004EB4400054941F830700020029002E07F
:104350004FF0FF30029000BF029872E744F6002051
:104360002C0200202DE9FC5F81460E461746984638
:10437000DDE90CAB002001904FF420721C210E20CF
:1043800002F000F905461DB94FF0FF30BDE8FC9F73
:104390006C680F9801F0F1FBE080D8F80000A06095
:1043A000B8F80400A081DBF80000C4F81200BBF8E4
:1043B0000400E082DAF80000C4F80E000E980068ED
:1043C000A0614FF48070208008206080062020715A
:1043D0000420607140F606003B46324629460090B4
:1043E000484600F057F9284602F06AFA002501987D
:1043F000CCE7000070B504460D46034A2946204626
:1044000000F004F870BD00006EF500087FB50446AA
:104410000D4616460121074A201D04F126038DE8AA
:1044200025000391324619462046FFF79BFF04B052
:1044300070BD000074F5000870B5002464E004EB62
:104440004400334901EBC000057D002D5BD004EB37
:10445000440001EBC000408A401C04EB44012C4A9C
:1044600002EBC101488204EB4400114601EBC0009D
:10447000408AB0F5967F0DDA04EB440001EBC000F2
:10448000007D01280AD104EB440001EBC000408A02
:10449000052803DB2046FFF73FFD34E004EB440032
:1044A0001B4901EBC000007D032807D1042004EB69
:1044B0004401174A02EBC101087524E004EB4400F3
:1044C000134901EBC000007D042807D1022004EB52
:1044D00044010F4A02EBC101087514E004EB4400EB
:1044E0000B4901EBC000007D01280CD104EB440214
:1044F0000B4603EBC202111D04EB440203EBC202A4
:104500009068FFF777FF641C0A2C98DB70BD0000F1
:1045100044F600202DE9F84306460D461746984616
:104520005DB1286848B13146286800F0FFFB20B92A
:10453000287800F0F000E02803D16FF00F00BDE80C
:10454000F883324641462846FFF732FC0446002CE9
:1045500001DA60B2F3E7022004EB44011B4A02EBEC
:10456000C101087504EB4400114601EBC0008660F0
:1045700004EB440001EBC0003968C160B9880182D6
:10458000002004EB440102EBC101488204EB44002B
:10459000114651F83000B0B104EB440051F83090AE
:1045A000002004EB440142F831004FF400603B4628
:1045B00006F1260249460090304600F06BF8484666
:1045C00002F07EF900BF0020B9E7000044F60020A9
:1045D0002DE9F04104460E464FF00E0860890E2882
:1045E00000DC4FE0E07B18B996F83000401CE07327
:1045F0006568AF89287800F00100B0B128780128FB
:1046000009D1687888B9A8785E280ED1607B40F01F
:104610001000607309E006221D492846FBF71CFFC5
:1046200018B9607B40F008006073082F03D0B7F51D
:10463000C16F22D110E096F82D0000F0080000B9FB
:1046400020E04146204602F014FA00B11AE031465B
:10465000204600F07BFC11E096F82D0000F00800E9
:1046600000B90FE04146204602F003FA00B109E02C
:1046700031462046FFF770FC00E003E000BF002059
:10468000BDE8F081204602F01BF90020F8E70000A9
:104690006EF500082DE9F04706460D461746984688
:1046A000DDF82090484601F068FA82460E2128463F
:1046B00001F030FF00B113E06C68A4F80CA0D8F84A
:1046C00000002060B8F80400A0803868C4F8060034
:1046D000B888608129463046B2699047BDE8F087C6
:1046E0006FF00100FAE7000070B50446082001F001
:1046F00037FB054615B94FF0FF3070BD25626120CC
:1047000084F82E0074212F20015506486061064868
:10471000A06104F126002860204601F08FF80020F7
:10472000EBE70000114000083D5A000810B50446B0
:1047300094F82D00C0F3800018B1204601F058FE17
:1047400002E0204601F0F8FD10BD70B504460026D9
:10475000254601F063F8064695F82D00C0F3800069
:1047600020B91EB1284601F023FE08E095F82D007F
:10477000C0F3800018B116B9284601F0FDFD70BDE8
:1047800010B5044694F82D00C0F3800060B1094BC9
:104790005A7A9979187808F04BFC4FF4967008F023
:1047A000D7FAFFF7D5F901E0FFF7E6F92046FFF762
:1047B000BDFF10BD3058002010B50022042108466E
:1047C00009F077FE0849086000221421042009F04E
:1047D00070FE0649086000221421042009F069FED9
:1047E0000349086010BD0000300000202C000020AC
:1047F000280000201CB5294800210B468022CDE965
:10480000001027A127480AF023FB274800210B4668
:104810008022CDE9001025A126480AF019FB264880
:10482000072100234FF48072CDE9001023A1254811
:104830000AF00EFB2448012100238022CDE900105C
:1048400022A124480AF004FB2348042100238022EB
:10485000CDE9001021A122480AF0FAFA21480221EC
:104860000023CA01CDE900101FA121480AF0F0FA87
:10487000204806210023CA01CDE900101EA12048CE
:104880000AF0E6FA1F48052100234FF44072CDE9F3
:1048900000101DA11E480AF0DBFA1CBD000000201C
:1048A00072756E00357A000820000020737065650F
:1048B000640000007DBA0008080000206D62746387
:1048C0007000000079600008040000207273343822
:1048D00035000000917900081C000020696F00007D
:1048E000794C00080C0000206D62727475000000A5
:1048F0005D6000081400002063616E325F6D00008F
:10490000E50D00081000002063616E315F6D00004E
:10491000710D000870B50024002500BF0DE0094AA4
:1049200002EBC402928891B2064A52F8340000F0B9
:104930006AF8A0400543601CC4B2072CEFD3284698
:1049400070BD0000B00000204FF6FF710160002133
:1049500081710171042141710121C1717047F0B56C
:104960000A461588ABB29579032D01D100241AE0CF
:10497000957965B9557905F00F045579182D01D150
:10498000036110E05579282D0DD143610BE0957935
:1049900005F00805167906F004063543D67906F0C9
:1049A000030645EA0604DDB2A5B1002110E00125A9
:1049B0008D401D405DB105688F000F26BE40B54398
:1049C000056005688E0004FA06F635430560491C4B
:1049D0000829ECD3FF2B15DD1B12002110E0012567
:1049E0008D401D405DB145688F000F26BE40B54328
:1049F000456045688E0004FA06F635434560491C5B
:104A00000829ECD3F0BD0246002093680B408B428E
:104A100000D000E001207047F0B50C46104F07EBC6
:104A20001062C0F30741C0F30725C6B2C5F12007E5
:104A3000A7EB010C4FF0FF3707FA0CF3C5F1200785
:104A40007F1AFB40CB408B4017689F4317602CB107
:104A500006FA01FC176847EA0C071760F0BD000072
:104A60000000014070B505460C4622460321284649
:104A700000F0C0F870BD00002DE9FF5F05468A46D2
:104A80005B4880680390039800780007860E142E18
:104A900000DAA3E06889042800D29FE068680478FF
:104AA00014B1082C7ED100E092E0DFF8449109F1C6
:104AB00014094F48007D00F0F000E02800D191E09B
:104AC0004B4A1168506900F031F900B18AE0288939
:104AD000082800D282E006F10E01284601F01AFDF6
:104AE00080B3288930441FFA80FB2889584500DDAF
:104AF00078E04FF4207259460E2001F043FD07463E
:104B000007B96FE0798906F10800814203D238467F
:104B100001F0D6FE66E0324678680399FBF7ECFCBC
:104B20003146384601F0A5FF18B1384601F0C8FEFD
:104B300058E02946384601F02DFE20B1384601F0F4
:104B4000BFFE4FE004E0284601F0BAFE3D4606E015
:104B500006F10E01284601F08CFF00B142E0D5F8C5
:104B600004803146284601F0D5FCF0B96F68D9F8C9
:104B70000000F8601E4800693861002088F80000D5
:104B8000A8F80200FF20387200207881012000215F
:104B9000FF230A46CDE9010A00914946284600F064
:104BA000BDFA00E002E0834600BF11E0032C0ED006
:104BB0000B2C0CD00C2C0AD0042C08D0052C06D0C1
:104BC0000D2C04D00E2C02D0112C00D000BF00BF41
:104BD00000BF284601F074FEBDE8FF9F284601F0A3
:104BE0006FFEF9E7284601F06BFE00BFF4E7000016
:104BF0003CBF00202DE9FF470746884691464FF409
:104C000020722421222001F0BDFC05460DB9BDE82B
:104C1000FF87D7F804A06C6884F8008084F80190BE
:104C20000020A080E08079686A6802F108001C22F8
:104C3000FBF762FCDAF80C00039003A800F0EEFB2F
:104C400006465EB10020608001200021FF2303AAF8
:104C5000CDE901060091284600F060FA284601F0EF
:104C60002FFE00BFD3E770B505460C4622460B2148
:104C70002846FFF7BFFF70BD00260027002400254F
:104C80004FE0052D43D2DFE805F0031D273814005F
:104C90002448C068008CB84202D00024012507E0F7
:104CA0002048C068008C20490988884200D004252B
:104CB0002DE01D4800881B49C96808841A480788E8
:104CC000002524E01749C96801F12000FCF7A8FC81
:104CD000601CC4B202251AE01248C068008C124958
:104CE0000988884203D110480788002504E00A2C6F
:104CF00001DA012500E0032509E04DF6AD60094920
:104D0000C9680884074608490880002500BF00BF1D
:104D1000FFF700FE06460349C9680E81142007F01C
:104D200081FCAEE7D00300204400002018B5024605
:104D30000092D04300B10AB9012018BD91F82D00AE
:104D400000F0020008B90020F7E74868904201D15E
:104D50000020F2E700988B681840D1E90134234025
:104D6000984208D1886822EA00008C68E3439842A0
:104D700001D10120E1E70020DFE700002DE9F74F36
:104D80008CB004460F464FF00008B98CA1F1140016
:104D9000C11700EB5171C1F3CF0A14200590606870
:104DA0000990DDF8249099F8000000F00F0014211C
:104DB000B1EB800F04D06FF005000FB0BDE8F08FAD
:104DC00000BF6089142802DA6FF00500F5E700BF24
:104DD000B9F8060000F0D1FE04900498C0F30C006E
:104DE0000790049800F400500390208914381FFAAB
:104DF00080FBA0E04FF6FF7000EACA00584501DDD5
:104E0000584603E04FF6FF7000EACA0008904FF4DE
:104E1000207214210E2001F0B5FB054605B990E083
:104E2000142268680999FBF767FBD5F80490089885
:104E30000A9045E061890598081A80B202900299AB
:104E40000A98884201DA0A9800E002988046B8F190
:104E5000000F03D100200590246831E000F028FB0A
:104E600006461EB9284601F02BFD6AE061680598E8
:104E70000844334641224146CDE90008002001F0B4
:104E800029FC0B900B9830B9304600F016FB2846F1
:104E900001F016FD55E0204601F0E4FD74612A485A
:104EA000306128460B9901F03EFC0A98A0EB0800FF
:104EB00080B20A900A9810B100200590246800BFC3
:104EC0000A980028B6D10598404480B20590B88C65
:104ED0001438584501DB012000E0002006900798B7
:104EE000C0F30C000490069808B1039818B1049818
:104EF00040F400500490049800F03FFEA9F806002A
:104F00000899143188B200F038FEA9F80200002098
:104F1000A9F80A007B69294638460E9A9847284620
:104F200001F0CEFC0898ABEB00001FFA80FB07985D
:104F3000504480B20790BBF1000F7FF45BAF0020BC
:104F40003BE74FF0FF3038E7055800082DE9F04700
:104F500007460E467D6828780421B1EB201F05D056
:104F6000384601F0ADFC0020BDE8F0872878000746
:104F70004FEA9068688800F000FE8146398949450B
:104F800003DD4946384601F033FD7889404505DBAD
:104F90003889484502DBB8F1140F04DA384601F0CD
:104FA0008FFC0020E0E728694D494861E868086106
:104FB0000846007D00F0F000E0280AD196F82D00A8
:104FC00000F0010018B1706808B134461CE00024FC
:104FD0001AE0304600F088F808B1344614E00024A6
:104FE0003F48007D7F280FD03E48046809E0B44266
:104FF00000D105E0204600F077F800B103E000BFE3
:105000002468002CF3D100BF354908693146FFF709
:105010008DFE28B93248007C00F0F000E02804D171
:10502000384601F04DFC00209EE724B9384601F0D7
:1050300047FC002098E7E8884FF63F71084038B1F8
:10504000384600F0EDF807460FB900208CE77D6880
:10505000234804604660856028780007800E204958
:1050600088814146384601F004FD687A01280DD058
:10507000062806D011280ED13146384606F00EFE1D
:1050800022E03146384603F003FB1DE03146384646
:10509000FFF7F2FC18E0124948692146FFF746FE87
:1050A00070B90F48007D00F0F000E02808D00FFA3A
:1050B00088F1384601F05DFC02213846FFF7D2FC4A
:1050C000384601F0FDFB00BF00BF00200449086026
:1050D0004860886088810861486100BF44E700003B
:1050E0003CBF0020C401002010B5044694F82D00F8
:1050F00000F0010070B1606860B107484069616804
:10510000884205D0044948692146FFF70FFE08B1DF
:10511000012010BD0020FCE73CBF00202DE9FE4F20
:1051200007460C4615469846DDE90C9A0E9EA346A6
:1051300025B10CB1206808B906F1040B43462A4694
:1051400059463846CDE9009A029600F003F8BDE8CA
:10515000FE8F00002DE9F84F05460F4690469A460F
:10516000DDF828B00C9EB8F1000F38D04FF01409CC
:105170001421284601F0CEF918B16FF00100BDE806
:10518000F88F6C6884F808A00B986072D8F800005B
:10519000206148464FEAE97109EB9171C1F387013B
:1051A00041F04001217084F801B0288900F0E5FC4D
:1051B00060800020E0801848008800F0DEFCA080BD
:1051C00015480088401C144908801FB9134800681E
:1051D000E06001E03868E0600020608109E06889F3
:1051E000142802DA6FF00100C9E76C6820690090AA
:1051F000E846B08C48B12889B18C884205DD42462A
:1052000031462846FFF7BAFDB9E7424629463046FF
:1052100073699847B3E700002E020020B8F6000833
:105220002DE9F14F84B004984568287800F00F000C
:105230001421B1EB800F00D0E7E0E88800F09DFC7E
:10524000C0F30C004FF6FF7101EAC00A688800F055
:1052500094FC074628780007810E02910299B94212
:1052600000DDD2E00298381A87B2049801F073FA90
:1052700006466848018888190A280ADD314628460A
:1052800000F062FA20B16348008830440A2800DD4B
:10529000BBE06148046811E06069E968884209D1AF
:1052A000A0692969884205D1A089A988884201D1CD
:1052B000012000E0002000B102E02468002CEBD1C6
:1052C00000BF34B93146284600F0D0F9044694B9FD
:1052D0009BE0E88800F051FCC0F30C0058B9E0896D
:1052E00000F04BFCC0F30C0028B11422294604F155
:1052F0000800FBF701F9E888012121EA501001902C
:10530000019850B10AEB070188B2504503DB4FF614
:10531000EB71884200DD71E000BF2046019A0499DC
:1053200000F0D2F883460BF1010000B966E039487D
:105330000088304437490880019840B10AEB0701E2
:1053400088B2A083A17F41F00101A17700BFBBF12A
:10535000010F51D1A08B143080B20090606840687A
:10536000D0F8009060684568142204F108012846CE
:10537000FBF7C2F8009800F000FC68800020E8808D
:105380006881606804900DE0D9F80400039014214E
:10539000484601F06EFB4946049801F0C4F90398B1
:1053A000D0F80090B9F1000FEED11B48006884429C
:1053B00002D14FF000080EE01748D0F8008006E058
:1053C000D8F80000A04200D104E0D8F80080B8F17D
:1053D000000FF5D100BF4146204600F033F9049894
:1053E00001F0B9F906460B480088801B094908807E
:1053F000049805B0BDE8F08F0020FAE7606818B99E
:105400000021204600F01EF900BF049801F058FA70
:105410000020EEE7340200203002002010B50246E2
:105420002148016821E091F82D0000F00100D8B179
:1054300091F82D00C0F38000B0B14868A0B11068A9
:105440008B681840D1E901342340984201D10846C5
:1054500010BD91F82D0000F0020028B91068CB684B
:10546000984201D10846F3E709680029DBD10F48CB
:105470000068A0B10D48006890F82D0000F0010010
:1054800068B10A48006890F82D00C0F3800030B180
:1054900006480068406810B110787F2801D10020CC
:1054A000D6E702480068D3E7C4010020C801002005
:1054B00010B5052000F0ACFD10BD10B50446214626
:1054C000052000F06BFD10BD2DE9F74F84B00746B5
:1054D0008846002501200190D8F804000290029926
:1054E000488800F04AFB8346029800780007800E47
:1054F00003900398584503DD681E07B0BDE8F08FA0
:105500000398ABEB00001FFA80FB0299C88800F0FB
:1055100034FBC0F30C004FF6FF7101EAC00AD8F863
:10552000044000202060A4F804A00AEB0B00E080F7
:10553000E088504502DA4FF0FF30DEE7D7F80490FC
:105540003EE0D9F80460A088B188884220DAC4F827
:1055500000909DB1A088E988884203DBE088B1888B
:10556000884202DD4FF0FF30C7E7C5F80080E888C9
:10557000A18888420BD00020019008E0E088B18823
:10558000884202DD4FF0FF30B7E7C7F804801AE029
:10559000A088B188884202D14FF0FF30ADE7A088E3
:1055A000F188884202DA4FF0FF30A6E72DB1E88893
:1055B000B188884201D000200190D6F8009035468D
:1055C000B9F1000FBDD100BFB9F1000F0BD145B14A
:1055D000C5F80080E888A188884204D000200190A6
:1055E00001E0C7F80480069818B9B87F00F0010000
:1055F00028B30198E8B1786818B178684068808865
:1056000010B10020019014E02546D4F800900BE082
:10561000D9F80440E888A188884202D0002001908F
:1056200005E02546D4F80090B9F1000FF0D100BF95
:1056300000BF019808B101205FE700205DE700206E
:105640005BE7000070B504460D4607480068A042BD
:1056500003D105492068086001E0206828602146E0
:10566000042000F09BFC70BD3002002070B50546A0
:105670000E46042000F0CCFC044664B931462846AE
:1056800000F062F8B04203DB042000F0C1FC0446E5
:105690000CB9002070BD20212046FAF79CFF0F2096
:1056A000E077064800682060044804601422294618
:1056B00004F10800FAF720FF2046EBE73002002053
:1056C0002DE9F0470446894600266068D0F804803A
:1056D000B8F80400B0B96568D8F80000606014221A
:1056E00004F108016868FAF707FF01212846FFF76F
:1056F000BAFA284601F02FF80746F01986B2284674
:1057000001F0DEF865680EE0D5F80480AA46D8F806
:105710000050504601F01FF80746F01986B2504677
:1057200001F0CEF800BF002DEED149462046FFF72C
:1057300089FF04480088801B024908803046BDE884
:10574000F0870000340200202DE9F84F0546894615
:10575000002700BF0026B2460020009083461B4869
:10576000046821E06069E968884207D1A069296975
:10577000884203D1A089A988884201D0012000E095
:10578000002068B10BF1010B1EB92646CDF800A030
:1057900006E0E07FF17F884202DC2646CDF800A0DB
:1057A000206800B1A2462468002CDBD12EB130461F
:1057B0000099FFF785FF804647444F4502DABBF169
:1057C000010FC7DC3846BDE8F88F0000300200202A
:1057D00070B500250A4804680FE0E07F002805DD69
:1057E000E07F401EE0772546246806E026462468D0
:1057F00029463046FFF764FF00BF002CEDD170BD95
:105800003002002070B504462546686910B1686909
:1058100001F056F82846FFF750FE70BD38B56A46CD
:1058200001210320FEF7AAF808B9002038BDBDF811
:105830000000C0F380042046F8E7000038B50446B5
:105840000025062084F82C003348007884F82600D0
:1058500031484178272001552F488178282001556B
:105860002D48C178292001552B4801792A2001555E
:10587000294841792B20015540F2DC50A08494F84E
:105880002D0040F00E0084F82D000423234A244903
:105890000020FDF745FE0623224A23490120FDF79B
:1058A0003FFE00BF06E0204901EB45100121FDF756
:1058B000E6FF6D1C062DF6D300250AE0184800EB24
:1058C0004510006840F44000154901EB451108609F
:1058D0006D1C042DF2D3002014494861144800685F
:1058E00028B900210A2008F0A5FD114908601148D7
:1058F000006828B900210A2008F09CFD0D490860C5
:105900000A204FF4007322460B4900900BA002F0CE
:1059100077F9FEF71DF938BD7400002048400020DB
:10592000101C0020901C0020501B00201858002044
:105930007C000020800000203D3D00086574685F09
:105940007278706B740000002DE9F84F4FF0000B77
:10595000DA460027002000908046FEF7A5F80128CF
:1059600002D00020BDE8F88F3248D0F800B0D0F85F
:105970000490BBF1000F07D01FFA8BF14FF4C172F6
:10598000002000F0FFFD8046B8F1000F2FD029481D
:10599000C6680024454628E06F894FF0000A15E0EC
:1059A00040F2F4531A1B09EB04016B6803EB0A0085
:1059B000FAF7A2FDF668D6F8089040F2F450001B02
:1059C0003F1A40F2F450001B82440024381940F280
:1059D000F4518842E4D809EB04016A6802EB0A003A
:1059E0003A46FAF789FD3C442D68002DD4D1114880
:1059F000C6680020009007E0306840F0004030604A
:105A0000F6680098401C00900A484169009881425D
:105A1000F2D80020074948618020FDF7DDFD38B14C
:105A20008020FDF7D3FD044880680020024988608B
:105A3000404697E718580020009002402DE9F84FA3
:105A40008B464FF000090024A24600262E48D0F8CD
:105A50000080FDF749FF00905D463FE0D8F8000068
:105A600000F0004010B16FF007073EE06E894FF084
:105A7000000A23E040F2F4531A1B6B6803EB0A019F
:105A8000009B1819FAF738FDD8F80C80D8F80000F8
:105A900000F0004010B16FF0070726E0D8F80800CA
:105AA000009040F2F450001B361A40F2F450001BF4
:105AB000824440F2F450001B81440024301940F22B
:105AC000F4518842D6D86A6802EB0A01009A10198C
:105AD0003246FAF711FD3444B1442D68002DBDD192
:105AE0004846FEF773F8002700BF0420FDF774FD59
:105AF00038B10420FDF76AFD0448406800200349DE
:105B000048603846BDE8F88FE80000200090024069
:105B10002DE9F041044625466868804702F06CF89C
:105B200006460D49286809684718B81BB0F1004FB0
:105B300001D3012000E0002030B1296888192246F5
:105B4000064902F089F804E022460449384602F08A
:105B500083F8BDE8F08100001C020020115B000802
:105B60000146080601F47F4240EA022001F47F0268
:105B700040EA122040EA1160704701460806000C16
:105B800040EA1120704710B5002401F0F3FF00F047
:105B900089F800F017FA00F063FB06F073F802F0E2
:105BA0006BFD02F09FF810BD10B50446207808493F
:105BB000087060784870A0788870E078C8702079A4
:105BC0000871607948712046FDF7B2FE10BD0000F3
:105BD0007400002007F098FC07F04AFC07F0B0F8CA
:105BE00007F0E0FB07F0FCFC07F020FD07F068FD84
:105BF00007F0E0F806F05CFF07F014F807F0BEFAD3
:105C0000FBF73EF807F054FE07F0ACFA03E04FF460
:105C1000FA7007F09DF8FAE770B5054605B970BD52
:105C200005F0030010B100BF00BFF8E7A5F10804BC
:105C300018480068844205D305F10C00164909682C
:105C4000884202D900BF00BFE9E7144801F0B3FF62
:105C5000207928B9114801F0C6FF00BF00BFDEE778
:105C6000204600F051F828B90C4801F0BCFF00BFF5
:105C700000BFD4E70020207109480068844201D2A7
:105C800007480460204600F013FF044801F0ABFF12
:105C900000BFC4E7800100208401002088010020AB
:105CA0008C01002010B5134820F003001249086051
:105CB000084604684FF4C86020800020608020718E
:105CC0004FF4C86001F076FD0C49086001200968B6
:105CD00008714FF4C86009490968088007490968D4
:105CE00048800548006806490860064801F06EFFD4
:105CF00010BD000057BF002080010020840100205B
:105D00008C010020880100202DE9F0410446204646
:105D100000F0ACF80546208801F04CFD064660888E
:105D200001F048FD07462088B0F5C86F10D860889C
:105D3000B0F5C86F0CD86088A84202D03888A84255
:105D400006D106480068864205D07088A84202D075
:105D50000020BDE8F0810120FBE700008401002065
:105D60002DE9F0478046B8F1000F02D10020BDE8D0
:105D7000F08708F1030020F0030085B20C2D00D25B
:105D80000C25B5F5C86F01D8454501DA0020EEE7CE
:105D9000334801F010FF3348006800F067F806460A
:105DA00054E0304601F006FD04462079002849D130
:105DB000218806F10800081AA84243D3218806F179
:105DC0000800091A05F1140081421BD306F10800EE
:105DD00028441FFA80F9484601F0ECFC07460021F0
:105DE0003971218839807E80A4F8009001202071CB
:105DF0003888B0F5C86F07D0388801F0DBFCA0F810
:105E0000029001E00120207116480068844213D1FD
:105E10001448D0F800A004E0BAF8000001F0CAFC71
:105E200082469AF8040018B10F4800688245F3D101
:105E30000C48C0F800A000BF094801F0D4FE04F1EE
:105E4000080094E7304601F0B5FC0688C5F5C86047
:105E5000B042A6D8024801F0C6FE002087E7000045
:105E6000880100208C0100208401002001460248A6
:105E70000088081A80B27047800100202DE9F84F91
:105E800081468B460BF1030020F0030085B20C2DF8
:105E900000D20C25B5F5C86F01D85D4502DA0020A7
:105EA000BDE8F88F39480068814503D33848006859
:105EB000814503D300BF00BF4846F1E7A9F10808B8
:105EC0004046FFF7D3FF0646B8F80010881B083895
:105ED0001FFA80FA554501DD0020E1E7554501D163
:105EE0004846DDE72B4801F066FEB8F8000001F0F7
:105EF00061FC0446207910BB2088009006F1080060
:105F0000284487B224480068A04204D1384601F0F2
:105F100051FC21490860384601F04CFC0446002041
:105F20002071009820806680A8F800702088B0F565
:105F3000C86F03D0208801F03DFC478021E005F1C7
:105F4000140050451DD806F10800284487B2384691
:105F500001F030FC044610480068844201D20E482B
:105F6000046000202071B8F8000020806680A8F846
:105F700000702088B0F5C86F03D0208801F01AFCAB
:105F80004780044801F02FFE484689E78001002041
:105F900084010020880100208C01002070B5044697
:105FA0000D4600BF0D2C00DB70BD00BF05B9FBE73F
:105FB000034951F824002946FBF780FD00BFF3E7B1
:105FC00018F6000810B5002406E0054951F8240031
:105FD00000F008F8601C84B20D2CF6D310BD000050
:105FE00018F6000810B50023846823604368DB1CA2
:105FF00023F00301002207E083681B680B608368BD
:10600000196003881944521C43889342F4DC10BD84
:1060100070B5044600BF0D2C01DB002070BD00BF31
:10602000034951F82400FBF750FD05462846F5E7E3
:1060300018F6000838B500204FF416530246012127
:1060400000900220FBF7F0FF04461CB9FBF748FD67
:10605000044600BF04B138BD00BFFCE700234FF485
:10606000165219461846FCF78DFAFCF737F801E08E
:10607000FCF7E6FAFCE70000FFF7DCFF0020084928
:10608000C96808800649C96848800549C968888088
:106090000349C968C88001E0FCF78EFEFCE70000F8
:1060A000D00300202DE9F04704460D4616461F4652
:1060B000DDE9098ADDF8209000BF14B90020BDE8B1
:1060C000F08700BF00BFB8F1000F01D10020F6E754
:1060D00000BF05B92A4D06B9294E07B9284F00203F
:1060E0006060A060E060274860610020A08484F8C0
:1060F0002D00E061C4F820902348007884F8300037
:10610000C4F810A03B4632462946204600F0DEF88F
:106110002046C04708B10020D1E700BF94F83020E6
:10612000FF2A02D1002284F830200021174A10688B
:106130000DE0491C90F8302094F830309A4205D197
:1061400094F83020521C84F8302002E000680028C7
:10615000EFD100BF0028E1D194F83000FE2803D130
:1061600000200949087004E094F83000401C0649FA
:1061700008700648006820600448046020469EE7D6
:10618000B8F60008C3620008CC010020C40100205A
:1061900070B504460D462946204602F001FF294607
:1061A000204605F05BFE70BD10B503460868DC684C
:1061B000A04201D1012000E0002030B909B900203F
:1061C00000E00868D860012010BD0020FCE7F8B5A9
:1061D00005460C46164620686968884201D10120B0
:1061E00000E0002090B9206800906868306069463F
:1061F0003046FFF7CDFF0CB9002000E02068686052
:106200000121284600F03FF80120F8BD0020FCE7FE
:1062100010B5034608689C68A04201D1012000E047
:10622000002030B909B9002000E00868986001201A
:1062300010BD0020FCE7000002466AB10748016873
:1062400008E091F83000401CC0B2904201D10846ED
:10625000704709680029F4D10020F9E7C401002043
:10626000704770B505460C4694F82D0000F01800F4
:1062700020B121462846FEF7ABF970BD21462846DD
:10628000FEF764FEF9E770B504460D4694F82D005C
:1062900000F0040020B194F82D0000F0010000B9D6
:1062A00070BD05F0010050B1606840B194F82D0058
:1062B00000F0080018B1211D2046FEF79BF800BF32
:1062C000EEE703466FF00B00704700002DE9F84F32
:1062D00080460C4615461E464FF00009CA4604B9D2
:1062E000114C05B9104D06B90F4E0CB1206808B914
:1062F000012000E00020074627B16A4621464046BB
:10630000FFF765FF4A4629464046FFF781FF5246A0
:1063100031464046FFF748FF27B96A4621464046C6
:10632000FFF755FFBDE8F88FB8F60008014908608F
:1063300070470000C801002010B5044600BF04B932
:1063400010BD00BF94F82D0000F0010078B100BF2F
:1063500094F82D0000F0FE0084F82D0000BF94F8A2
:106360002D0000F0080010B12046FDF705FD00BF2C
:10637000E6E700B1C161704710B5044600BF04B93B
:1063800010BD00BF94F82D0000F0040070B100BFF4
:1063900094F82D0000F0FB0084F82D0000BF00BF32
:1063A000E06910B12046E169884700BF00BFE7E718
:1063B00010B5044600BF04B910BD00BF94F82D000D
:1063C00000F0040090B900BF94F82D0040F00400E4
:1063D00084F82D0000BF03212046FFF754FF00BFC3
:1063E000E06910B12046E169884700BF00BFE3E7DC
:1063F00010B5044600BF04B910BD00BF94F82D00CD
:1064000000F0010058B900BF94F82D0040F00100E1
:1064100084F82D0000BF03212046FFF734FF00BFA2
:10642000EAE700002DE9F0470B4614464FF0000C58
:1064300000BF2C4A1268C2F302211D4626460A46B6
:10644000C2F10709B9F1040F02D94FF0040901E0C4
:10645000C2F10709C84602F10409B9F1070F02D2D7
:106460004FF0000901E0A2F103094F464FF0010986
:1064700009FA08F9A9F1010909EA050909FA07F970
:106480004FF0010A0AFA07FAAAF1010A0AEA060A13
:1064900049EA0A09CC4601466246002904DB150791
:1064A0002E0E114D6E5407E015072F0E0D4D0C35B5
:1064B00001F00F06361FAF5500BF014600290DDB66
:1064C00000BF00BF01F01F050122AA404D09AD0029
:1064D00005F1E025C5F8002100BF00BF00BFBDE801
:1064E000F08700000CED00E000E400E000BF00F0E9
:1064F0000702064B19684FF6FF031940044B0B4384
:1065000043EA0221014B196000BF70470CED00E027
:106510000000FA0570B504460D46002229462046C3
:1065200000F001F870BD70B50346154613B1B1F522
:10653000803F01D3012070BD09B90020FBE78AB27A
:106540001889104480B2904201DA0120F3E71E7BE3
:1065500006F0800038B15868441A03F110008442F4
:1065600007D20120E7E715B15868441A01E001207D
:10657000E1E75C60588910445881188910441881FB
:106580000020D8E72DE9FE4F82460D46904657463B
:10659000B8F1010F0AD0B8F1410F06D0B8F5C17FAC
:1065A0000BD0B8F5207F78D148E000BF424629469D
:1065B000002000F077F8044671E0002400200290EB
:1065C000A94600BF0C20FFF723FD064646B900F0A0
:1065D000F9F914B1204600F073F90020BDE8FE8FF0
:1065E000F81C20F00300C0F5147080B2484501DDAE
:1065F000484605E0F81C20F00300C0F5147080B296
:1066000083460020CDE9008006F110003844C01C0C
:1066100020F003015B464A46304600F0C4F90CB94D
:10662000344601E0029806600296A9EB0B001FFABF
:1066300080F90027B9F1000FC4DC30E0F81C20F02D
:106640000301E81C20F00300084486B206F11000A4
:106650001FFA80F9E81C20F00300B04204D8E81CBF
:1066600020F00300484501D90020B7E74846FFF76E
:1066700077FB04460CB90020B0E70020CDE900808C
:1066800004F110003844C01C20F003012B462A46B8
:10669000204600F088F902E0FFE700209EE700BFF7
:1066A00020469BE72DE9FC4105460C4616460B208B
:1066B000FFF7AEFC074617B90020BDE8FC810020BB
:1066C000234622462946CDE90060384600F06BF9A2
:1066D0003846F2E72DE9FC5F05460C46174698461A
:1066E000DDE90C9BAA460AF1030020F003002044D8
:1066F000584502D90020BDE8FC9FB9F1000F06D033
:106700000AF1030020F0030000EB090600E0002678
:106710000220234622463146CDE90070404600F073
:1067200042F94046E7E710B5024600BF02B101B9A1
:1067300010BD00BF104604E003890C892344038187
:1067400000680368002BF7D103890C892344038177
:10675000016000BFECE70146002002E0421C90B25D
:1067600009680029FAD170472DE9F04107460D4626
:10677000144621892A463846FFF704FF064616B913
:106780000020BDE8F0812146304600F003F8804645
:106790003046F6E72DE9F04105460C460026002775
:1067A00000BF25B11CB128892189884203DA6FF026
:1067B0000F00BDE8F08100BF00BF6889801B6189C0
:1067C000C91B884203D36089A0EB070802E06889EF
:1067D000A0EB06086268D1196A6890194246F9F779
:1067E0008BFE464447446089B84201D8002724689C
:1067F0006889B04208D100262D6800BF1DB914B1C8
:106800006FF00F00D5E700BF54B16089218988423D
:1068100006D100BF206810B16FF00500C9E700BFC6
:1068200055B168892989884206D100BF286810B10E
:106830006FF00500BDE700BF002CBED10020B8E717
:106840002DE9F05F8046894616461D464FF0000A46
:10685000D34600BFB8F1000F02D10020BDE8F09F81
:1068600000BF00BFB9F1000F01D10020F6E700BF63
:10687000444620E035B16089A84203DC6089281ACB
:1068800085B217E06089401B87B2B74200DD37460A
:106890006268511909EB0A003A46F9F72DFE0BEB35
:1068A00007001FFA80FB0AEB07001FFA80FAF01BB3
:1068B00086B2002524680EB1002CDBD15846CDE706
:1068C0002DE9F047044614B90020BDE8F087002602
:1068D0002DE0A07B401EC0B2A0738046B8F1000F2F
:1068E00023D12768207B00F00F05607B00F00200B9
:1068F00028B1A1462046D9F81010884711E0022D92
:1069000004D121460C20FFF749FB0AE0012D04D1F8
:1069100021460B20FFF742FB03E015B92046FFF7A5
:106920007BF9701CC6B23C4600E0002400BF002C7E
:10693000CFD13046C9E7000010B500BF002008499C
:10694000087000BF0748046806E0606F18B1204671
:1069500001F049FE10BDE468002CF6D100BFF9E754
:10696000CD010020E001002010B50446FFF7E4FF50
:1069700010BD70B504460D4601222946204600F0A0
:1069800001F870BD70B505460C461646002C04DAB9
:106990006142284600F06DF870BD32462146284617
:1069A000FFF7C1FDF8E770B5DDE904450026066094
:1069B000416002814381047345730126867300267A
:1069C000C67370BD10B508480478012006490870E8
:1069D0004CB900BF0021054804F06CFF10B1002045
:1069E0000149087000BF10BDCD0100206969000891
:1069F0002DE9F04106460F463089B84201DCBDE87A
:106A0000F0813089C01B1FFA80F83D46344607E00C
:106A10006089281A85B22089A0EB080020812468AB
:106A20006089A842F4DB207B00F00F0070B9608918
:106A3000A8420BD0607B00F0020038B9A088001B90
:106A4000284481B22046FFF719FA0446658160891F
:106A50002081206810B12068FFF732FF00202060FD
:106A600000BFCCE720B100BF817B491C817300BF10
:106A7000704710B5024612B1B1F5803F01D3012035
:106A800010BD09B90020FBE78BB200BF50899842C6
:106A900001DA0120F4E700BF5468506808445060F0
:106AA0005089C01A50811089C01A10810020E7E770
:106AB0002DE9F0410446208800F07CFE0546AC42FA
:106AC00019D02879B8B91B480068854213D01A48F4
:106AD0000068A84201D118480460288820802888CE
:106AE000B0F5C86F07D02046FFF7C0F907462888E1
:106AF00000F060FE4780608800F05CFE0646A6421B
:106B000015D0307998B90C480068A04201D10A48E4
:106B10000660208830802088B0F5C86F07D03046E6
:106B2000FFF7A4F90746208800F044FE4780BDE83F
:106B3000F0810000840100208C0100202DE9F0414B
:106B400005460E461648076816480068001D05F001
:106B5000A0FA681C38B936B112480168091D1248FC
:106B600005F004FB1AE07C190E4800684460BC4242
:106B700007D20C480168091D0C48006805F0DCFAD2
:106B80000CE008480168091D0948006805F0D4FABE
:106B900008480068844201D206480460BDE8F081DC
:106BA00010010020FC000020105A002004010020E9
:106BB000000100202C01002010B5044605F00CFC5B
:106BC00024480068401C234908602348006840B9F5
:106BD000214804600846006801280DD100F042FAFF
:106BE0000AE01E48006838B91B480068C06AE16ABC
:106BF000884201D81848046019480068401C1849A8
:106C000008600846006860641649E06A09688842BE
:106C100002D91449E06A0860E16A01EB8101124A75
:106C200002EB8100211D05F0A1FA05F0FFFB0B48E6
:106C3000006868B108480068C06AE16A884207D203
:106C40004FF0805009490860BFF34F8FBFF36F8F3B
:106C500010BD00000C010020FC00002018010020E5
:106C600028010020140100208058002004ED00E0DD
:106C700008B505F0B1FB12480068E8B9114805F005
:106C80004BFA114805F048FA0E48104908600E48C2
:106C90000F49086000200F4B0F4A102100900A2076
:106CA00007F05BFC064908600846006820B10BA1AC
:106CB0000348006805F07AFC05F0B8FB08BD000049
:106CC00044010020245A0020385A00203C010020B2
:106CD000400100204C5A00209C5A0020546D7251F3
:106CE0000000000010B516E005F076FB0C48C06807
:106CF000C468201D05F0CDF90A480068401E094906
:106D0000086009480068401E0749086005F08EFBCE
:106D1000204600F05FF8044800680028E4D110BD68
:106D2000FC5900200C0100200801002070B5044629
:106D30000D46206C70B1216CE0680144E160D4E93B
:106D40000210884201D32168E1602846226CE16884
:106D5000F9F7D2FB70BD2DE9F04104460F46154608
:106D60004FF00008A66B206C48B9206800282CD191
:106D7000A06808F0B5F980460020A06025E07DB944
:106D80003946226C6068F9F7B7FB216C60680844EB
:106D90006060D4E90101884217D32068606014E084
:106DA0003946226CE068F9F7A7FB216CE068411ACC
:106DB000E1602168E068884203D2216CA068411A32
:106DC000E160022D01D106B1761E701CA063404621
:106DD000BDE8F08110B5044694F8590030B9206B35
:106DE00005F042FB204605F03FFB1AE094F85900FD
:106DF000012803D1204605F037FB12E094F8590032
:106E0000022801D1012000E0002050B900BF50202D
:106E100080F31188BFF34F8FBFF36F8F00BF00BFA8
:106E2000FEE710BD01464A6A22B10A6B1268C2F140
:106E3000100000E0002070470146084A12681268FE
:106E40000AB9012200E000220A600A6822B9034A56
:106E50001268D268106800E0002070473C010020F2
:106E600030B54FF4C843174800F007042CB1C01DDB
:106E700020F00700134C041B1B1B0246124C22601F
:106E80000024114D6C60D018083820F007000F4C1A
:106E9000206000240D4D2D686C600C4D2D682C6019
:106EA0001146441A4C60094C24680C60084D4C682B
:106EB0002C60084D4C682C604FF00044064D2C604F
:106EC00030BD00003C5B0020500100205801002034
:106ED000600100205C0100206C01002000BFFFF772
:106EE00001FF064800680128F9D94FF08050044995
:106EF0000860BFF34F8FBFF36F8FF0E7805800201B
:106F000004ED00E010B5044654B10020A0602060FC
:106F10000021E16000231A461946204607F0DAFBFB
:106F200010BD2DE9F04106460D4617469846069CD1
:106F30000DB9246000E02760E66325640121204646
:106F400007F07CFB84F84C80BDE8F0812DE9F05F10
:106F500082460E4690469B460A9F0C9C4FEA88014B
:106F6000A522206BF9F70DFBA8F10100216B01EBC5
:106F7000800929F0070909F0070008B9012000E09D
:106F8000002050B900BF502080F31188BFF34F8F0D
:106F9000BFF36F8F00BF00BFFEE786B1002507E09B
:106FA000715D04F134004155705D00B902E06D1C63
:106FB000102DF5D300BF00214320015502E0002031
:106FC00084F83400102F00D30F27E762E764002015
:106FD0002065201D05F0ADF804F1180005F0A9F8B2
:106FE0002461C7F11000A06164620020606584F82C
:106FF00058005A465146484600F0B4FC20600B98B1
:1070000008B10B980460BDE8F09F2DE9F0470646F3
:107010000D4617469846DDE908940DB1012000E0C1
:10702000002050B900BF502080F31188BFF34F8F6C
:10703000BFF36F8F00BF00BFFEE78CB1FFF718FEF4
:107040002660A561C4F81C80C4F82090201D05F0BE
:1070500070F82FB194F8280040F0040084F828005C
:10706000BDE8F08710B5002407E004EB84010F4A67
:1070700002EB810005F050F8641C102CF5D30C488D
:1070800005F04AF80B4805F047F80B4805F044F8BE
:107090000A4805F041F80A4805F03EF80448094955
:1070A000086004480849086010BD000080580020AE
:1070B000C0590020D4590020E8590020FC59002074
:1070C000105A0020000100200401002010B50146E4
:1070D000164800E0006803688B42FBD30246436811
:1070E00013448B4204D143684C68234443600146F7
:1070F0000A464B6813440468A34211D10C4C036840
:107100002468A34208D04B680468646823444B6039
:1071100003681B680B6005E0054B1B680B6001E012
:1071200003680B60884200D0016010BD5001002050
:10713000580100202DE9F04104460D4616461F4631
:107140004FF0000865602461B5420CD8F01BA169BE
:10715000884202D34FF0010811E0211D0948006860
:1071600004F0EAFF0BE0BE4204D2BD4202D34FF06E
:10717000010804E0211D0448006804F0DDFF4046DA
:10718000BDE8F081400100203C01002070B50546BB
:1071900005F022F9A86B08B9012400E0002405F0ED
:1071A00045F9204670BD70B5054605F015F9A86B88
:1071B000E96B884201D1012400E0002405F036F992
:1071C000204670BDF8B505460F461A480068C068ED
:1071D000C468201D04F05DFF94F8280000F004004E
:1071E000E8B1A06941192B463A462046FFF7A2FFB5
:1071F000D8B1002003462A4601460090204608F0F8
:1072000039F9064656B900BF502080F31188BFF304
:107210004F8FBFF36F8F00BF00BFFEE705E094F80C
:10722000280020F0010084F828002046216A8847C1
:10723000F8BD00003C010020F0B587B0A0E0039845
:10724000002811DA04AE56B900BF502080F311882F
:10725000BFF34F8FBFF36F8F00BF00BFFEE7D6E9CC
:107260000020B168904700BF03980028E6DB059C2A
:10727000606908B9012000E0002010B9201D04F069
:1072800008FF02A800F0DCF8054603980A2875D22A
:10729000DFE800F009050739416306083A4200BFFC
:1072A00000BF00BF00BF94F8280040F0010084F840
:1072B00028000498A269811803462A462046FFF751
:1072C00039FFF8B12046216A884794F8280000F079
:1072D0000400B8B1002000900498A169421800236E
:1072E0001946204608F0C6F8074657B900BF502097
:1072F00080F31188BFF34F8FBFF36F8F00BF00BFC4
:10730000FEE700BF3BE000BF94F8280020F001003A
:1073100084F8280033E000BF94F8280040F0010012
:1073200084F828000498A061A06908B1012000E059
:10733000002050B900BF502080F31188BFF34F8F59
:10734000BFF36F8F00BF00BFFEE7A06941192B4656
:107350002A462046FFF7EEFE11E094F8280000F0E0
:10736000020018B9204605F07FF805E094F82800DF
:1073700020F0010084F8280001E0FFE700BF00BF13
:10738000002203A90448006807F08AFB00287FF464
:1073900056AF07B0F0BD000044010020F8B5054627
:1073A0000C4605F009FB684600F04AF806460098CE
:1073B00020BB44B9B54206D807F082FF31462846C3
:1073C000FFF700FF1CE03CB10E480068006808B9F8
:1073D000012000E000200446A91B22460A4800685C
:1073E00005F0FAF807F06CFF50B94FF080500749EC
:1073F0000860BFF34F8FBFF36F8F01E007F060FFAE
:10740000F8BD0000400100204401002004ED00E030
:1074100009480068006808B9012000E0002020B198
:107420004FF0FF300549086005E003480068C06878
:107430000068024908607047000100202C0100200C
:1074400070B5044607F0A4FD05460748006885426C
:1074500004D200F00BF80120206001E00020206041
:1074600001480560284670BD4C0100202DE9F84315
:1074700034E025480068C068056823480068C06893
:10748000C468201D04F005FE2046216A884794F850
:10749000280000F0040008B3A0694619AE4207D9DD
:1074A00066602461211D1848006804F045FE15E05F
:1074B000002003462A4601460090204607F0DAFFE6
:1074C000074657B900BF502080F31188BFF34F8F94
:1074D000BFF36F8F00BF00BFFEE700BF0A48006820
:1074E000006808B9012000E000200028C1D006484B
:1074F000D0F8008005480068034908600348C0F8D8
:107500000080BDE8F88300003C010020400100201D
:107510000E480068401C08B9012000E0002050B966
:1075200000BF502080F31188BFF34F8FBFF36F8FE0
:1075300000BF00BFFEE700BF502080F31188BFF3FB
:107540004F8FBFF36F8F00BF00BFFEE74C000020DE
:1075500010B50346002022B903EA010434B101202A
:1075600004E003EA01048C4200D1012010BD08B5FB
:1075700000BF6846FFF760FC044620460099FFF70D
:107580000DFFFFF759FEF4E770B5044604F024FF41
:1075900094F9455010E0606A08B9012000E000202D
:1075A00038B904F1240007F03FFE18B105F074F873
:1075B00000E003E0681E45B2002DECDC00BFFF20B8
:1075C00084F8450004F032FF04F006FF94F94450BB
:1075D00010E0206908B9012000E0002048B904F15A
:1075E000100007F021FE08B105F056F8681E45B2FC
:1075F00000E001E0002DECDC00BFFF2084F8440037
:1076000004F014FF70BD014621B1012904D00729FF
:1076100006D103E0002005E0022003E0062001E09F
:10762000042000BF00BF704710B50446A4B1204637
:1076300000F05CFD10B1204600F082FC07480068B5
:10764000844202D100200549086005480068844250
:1076500002D100200249086010BD00002C04002067
:107660002804002070B504460E46254615B128466C
:10767000FFF7DAFF70BD000010B5024800688047D0
:1076800010BD00001003002010B5024800688047BC
:1076900010BD00000803002010B5024800688047B4
:1076A00010BD00000C0300202DE9F04107460C46F8
:1076B000154615B12846BDE8F0811048006890B91C
:1076C0000E4804600E49204603F028F80D49204674
:1076D00000F0ECFE2146204600F0ACFC00200A49F8
:1076E0000880002607E005480068FFF79DFF204658
:1076F000FFF79AFF00263046DDE700002C0400204B
:107700000D77000865760008300400202DE9F04769
:1077100081460F4614461D4615B12846BDE8F08740
:1077200024B93846FFF780FF0020F7E76189384623
:1077300003F015F860891D4909880844B0F5837F76
:1077400005DD3846FFF770FF4FF0000829E0628939
:10775000174BDFF858C0BCF800C003EB0C006168A1
:10776000F8F7CAFE60891149098808440F49088062
:1077700008460088072814DB0D48007906020C48EB
:1077800040790643B01D098888420ADC0749098808
:10779000884203D1022006F077FC02E03846FFF76A
:1077A00043FF2046FFF78CF84046B7E7300400203F
:1077B000EB150120014602480068084470470000AC
:1077C000800100202DE9F04104464FF0000805F04B
:1077D000F3F85148006808B9FFF742FB4F480068CA
:1077E000204000287ED13CB304F10800A04223D9F8
:1077F000083404F0070000B304F00700C0F10800EB
:107800002044A04216D904F00700C0F10800044447
:1078100004F0070008B9012000E0002068B900BFAB
:10782000502080F31188BFF34F8FBFF36F8F00BFDD
:1078300000BFFEE7002400E00024002C54D03848AC
:107840000068844250D8374E3046056801E02E4625
:107850002D686868A04202D228680028F7D12E4817
:107860000068854240D0306800F108082868306020
:107870006868001B102819D92F1907F0070008B9EC
:10788000012000E0002050B900BF502080F3118893
:10789000BFF34F8FBFF36F8F00BF00BFFEE7686875
:1078A000001B78606C603846FFF710FC1C49686864
:1078B0000968081A1A490860084600681A490968E0
:1078C000884203D21648006817490860134968685F
:1078D0000968084368600020286014480068401C5C
:1078E000124900E000E0086007F0EAFC08F0070039
:1078F00008B9012000E0002050B900BF502080F3FB
:107900001188BFF34F8FBFF36F8F00BF00BFFEE73B
:107910004046BDE8F0810000580100206C010020C5
:107920005C01002050010020600100206401002063
:107930000648006830B10549096801F15000096D39
:10794000491C01600148006870470000FC000020ED
:107950000349096860F30821014A1160704700007B
:1079600000700040001F4FF080730360001F21F083
:1079700001030360001F054B036014380260001F01
:107980006FF0020303602038704700001175000893
:1079900000244AE02046611CCCB214282ED10024D9
:1079A0006423012200210420FBF7AEF91F48C068C0
:1079B000B0F858021E49C9680882642301220021D8
:1079C0000520FBF7A1F91948C068B0F82003184951
:1079D000C96848826423022210210320FBF794F92E
:1079E0001248C068B0F8B0011149C96888820F48D0
:1079F000C068B0F8B2010E49C968C8826423022287
:107A000004210620FBF780F90848C068B0F8F003AD
:107A10000749C96888800548C068B0F8F20304497E
:107A2000C968C880322004F0FDFDB3E7E8030020F8
:107A3000D00300200CE04FF480510648F8F7CBFD4E
:107A400005F00AF80020F9F779F9C82004F0EAFDFA
:107A5000F1E700001C0B002008B50BE04FF0FF30F1
:107A600000231A46012100900348006805F0E6FF54
:107A7000FFF712FEF2E700001804002010B50446DC
:107A800000BF80210A48006804F038FA0028F8D0C6
:107A900021460748006804F01FFA00BF402104484F
:107AA000006804F02BFA0028F8D0012010BD000077
:107AB000080400202DE9F84F07468846914607F054
:107AC00067FA8246B8F1000F00D1E846B9F1000F1D
:107AD00012D04A464146386806F0E2FF012806D136
:107AE00007F056FA0646A6EB0A04254615E00020E4
:107AF000C8F80000451E10E000BF4FF0FF324146BD
:107B0000386806F0CDFF0128F7D107F041FA0646A4
:107B1000A6EB0A0404B9012425462846BDE8F88FDF
:107B20002DE9F04100F068F8074600BF0F480468EF
:107B30000CB9BDE8F0816068381AB0F1004F01D38C
:107B4000012000E0002000B1F3E708492068086048
:107B5000A568E66806496068086021460A20FEF7C5
:107B60001DFA0DB13046A847E0E7000018020020DA
:107B70001C020020704770B504460D464FF0FF36DA
:107B800000220421284606F094FC2060206800B101
:107B90000026304670BD73B5054600231A4601A97C
:107BA000286806F097FD012801D1002401E04FF07C
:107BB000FF3420467CBD10B5044600BF4FF0FF31B6
:107BC000206807F021F80128F8D110BD70B50446EF
:107BD0004FF0FF35012006F05BFC2060206800B10B
:107BE0000025284670BD10B5044600231A461946E4
:107BF000206806F06FFD10BD10B507F0C9F910BD83
:107C00002DE9FE4F05460E4617469846DDF83090A2
:107C100002A81FFA88F23B462946CDE9009030467B
:107C200007F016F98246BAF1010F01D1029C00E07B
:107C300000242046BDE8FE8F2DE9F04104460D46A4
:107C40001646FFF7D9FF071932462946384600F095
:107C500003F8BDE8F08100002DE9F04106460F462B
:107C600090460A20FEF7D4F904460CB9BDE8F0812D
:107C700000202060A760C4F80C8066601848006887
:107C800010B917480460F1E7154960680968496848
:107C9000401AB0F1004F01D3012000E0002028B1CC
:107CA0000F48006820600E48046017E00C48056823
:107CB00011E0286850B1606829684968401AB0F13D
:107CC000004F01D3012000E0002018B12868206097
:107CD0002C6002E02D68002DEBD100BF00BFC5E78E
:107CE0001802002010B5012408E0064901EBC40287
:107CF00051F834000449FFF79FFF641C032CF4D3B0
:107D000010BD00009CF60008115B000810B50E487D
:107D1000006810B94FF0FF3010BDFFF76DFF04464B
:107D2000094800684068001BB0F1004F01D30120F2
:107D300000E0002008B10020EEE703490968496827
:107D4000081B00BFE8E70000180200202DE9F047FB
:107D50000026002400250027A046A146F9F7A6FE2C
:107D60008246BAF1000F06D0BAF1010F15D0BAF170
:107D7000020F46D115E02D48406DC0F3402040B1C0
:107D80002A48006BC0F3406018B1294829490860AF
:107D900002E029482749086037E02748254908605C
:107DA00033E022484068C0F3004720484068C0F3F1
:107DB00083441E484068C0F341750DB90F2C03D1B0
:107DC0002801401C044400E0A41C27B91B48604360
:107DD0001849086014E015484068C0F3404058B1A5
:107DE0001248406DC0F30136B01C1349B1FBF0F0EE
:107DF00060431049086003E00F4860430D49086084
:107E000003E00D480B49086000BF00BF0748406809
:107E1000C0F303180A4810F808900648006820FAD2
:107E200009F004490860BDE8F08700000010024036
:107E3000006CDC02F800002000127A0000093D000E
:107E40005EF500082DE9FF5F04460E4600BF0CB941
:107E5000BDE8FF9F00BF207D0A2807D12146344896
:107E600001F045FC204600F073FB5FE04FF0000A94
:107E7000D346276DD4F82480D4F89050D4F81090CD
:107E8000207DE8B9E08A38B300BF2A480068A042E4
:107E900005D128480068C068264908600DE02549DA
:107EA000086806E0C168A14202D1E168C16002E051
:107EB000C0680028F6D100BF00BF0020E0600BE0E2
:107EC000B246B4F816B000BF21461B4801F00FFCC3
:107ED00001201A49087000BF206F10B1206F02F016
:107EE0009BFDE06E10B1E06E02F096FD606F10B188
:107EF000606F02F091FDBAF1000F0AD0208B211DB6
:107F000023464246CDE9001B02903946204602F046
:107F100035FD207D0390204600F01AFB00BF1DB107
:107F20006FF00C014846A84700BF00BF00BF8FE7B5
:107F3000E4010020D8010020E0010020E801002039
:107F400010B5044601212046FFF77CFF10BD28B183
:107F5000027D012A02D10246916100BF704770B5CF
:107F600005460C4616462046FFF7EAFF6FF00C0068
:107F700070BD000070B505460120FEF749F80446C3
:107F80001CBB00F05FFB00F0B5FE0120FEF740F8DF
:107F90000446CCB9092000F089FE0120FEF738F82C
:107FA000044684B9082000F081FE0120FEF730F875
:107FB00004463CB9284600F045FE0120FEF728F8AB
:107FC000044600BF00BF00BF00BF44B39C21204651
:107FD000F8F701FB0C3465724FF48660A4F8580082
:107FE0004000E083A083FF2004F8010C4FF40670EA
:107FF000E0840620A0866086C01FA0840120A087A0
:1080000008480068606108480078A0744FF48660F2
:10801000E0870648A0670648C4F888000C3C204664
:1080200070BD0000D4010020EA01002025A700084F
:1080300000DD6D0000B10161704700002DE9F047DF
:1080400005460C4617464FF0040904B9244C00BFFE
:108050001DB96FF00F00BDE8F08700BF00BF287D9D
:1080600010B16FF00500F6E700BF37B900F0D8FF98
:1080700007460FBB6FF00100EDE74FF0000819E075
:10808000184850F82800066810E0F08AB8420CD171
:1080900046B1306830B12CB1206818B13068216821
:1080A000884202D16FF00700D5E7F668002EECD1C8
:1080B00008F10108C845E3DB34B1206820B10CB9F0
:1080C000002000E020682860EF8200BF06480068BA
:1080D000E8600548056002F0D5FF00BF0020BAE760
:1080E000B8F600088CF60008D801002010B5044648
:1080F00000BF14B96FF00F0010BD00BF207D012834
:1081000005D000BF608B40F01000608300BF0121EC
:10811000204600F001F8EFE73EB504460D46002D7D
:1081200047D0207D042802D0207D072841D1A06FB0
:1081300018B9208DB0F5066F3BD0208BE18A221D47
:10814000CDE90021029023462046626A216D02F0AB
:1081500015FC204601F0A1FA00BF00BF39480068B5
:10816000A04205D137480068C068364908600DE074
:108170003449086806E0C168A14202D1E168C160E3
:1081800002E0C0680028F6D100BF00BF0020E06018
:1081900000BF01202C49087000BF2C480068A04295
:1081A00002D102F0F3FF02E0204600F0D1F90020F6
:1081B0003EBD207D20B1012824D002283AD12CE0F8
:1081C000E08AD8B100BF22480068A04205D120480B
:1081D0000068C0681E4908600DE01D49086806E097
:1081E000C168A14202D1E168C16002E0C068002814
:1081F000F6D100BF00BF0020E06000BF204600F0C5
:10820000A7F91BE0204600F093FD2146114801F03C
:108210006EFA204600F0E0F910E000BF2146094860
:1082200001F065FA01200849087000BF204600F0FF
:108230008FF903E0204600F00FF8B9E700BF0020F7
:10824000B6E70000E0010020E80100201402002051
:10825000D8010020DC01002070B50546287D0328E8
:1082600004D004280AD0072818D10FE0284602F0CD
:1082700031FC04460CB90520287511E0284602F0AF
:1082800029FC04460CB90520287509E0284602F0AF
:1082900021FC04460CB90920287501E0002070BDBE
:1082A00000BF1CB9284600F047FF09E0601C38B940
:1082B00000BF688B40F00800688300BF0020EEE735
:1082C0002046ECE72DE9F05F80460F4691469A463E
:1082D0000A9D05F0010008B1042000E0002005F02F
:1082E000020109B1002100E00021084405F0080165
:1082F00009B1002100E00021084405F0100109B196
:10830000002100E0002146180320FDF781FE041E35
:1083100005D13846FEF7D4FA0020BDE8F09FA572DB
:108320000020206067603889801B20811421384636
:10833000FEF7F0F820B1204602F061FB0020ECE7E8
:1083400060684068E060B8F81600FDF716FCE16868
:108350000880B8F81800FDF710FCE1684880504626
:10836000FDF7FEFBE1684860B346F11706EB91713B
:108370008910491D4FF6FF7202EA013141EA0900F6
:10838000FDF7FBFBE16888810020E1684882204618
:10839000C3E770B50B46164603B970BD998C71B131
:1083A0002822914202DD8D1AADB200E000252C4654
:1083B000A04201DA054600E02546284600BF00BF7E
:1083C000EBE72DE9F84304460D460027B94605F0D2
:1083D000020000B1012707F0010008B1042000E00D
:1083E000002007F0020109B1002100E0002108444B
:1083F00007F0080109B1002100E00021084407F05E
:10840000100109B1002100E0002100EB01094FF447
:10841000207249463620FEF7B5F8B0F1000809D1C0
:1084200000BF608B40F08000608300BF4FF0FF30E2
:10843000BDE8F88300972A4641462046E36DFFF7E2
:1084400041FF061E07D100BF608B40F080006083B3
:1084500000BF701EECE7E06E08B9E66607E0E06E6C
:1084600000E0006801680029FBD1066000BF002021
:10847000A4F8680005F0020010B905F0010010B181
:10848000E06D401CE06505F0010028B100BF608B85
:1084900040F02000608300BF7068FEF75CF9B4F81C
:1084A00066100844A4F866000020C1E708B1C0F8CF
:1084B0009010704770B523480078401C214908701F
:1084C00000BF2148046839E0A07F1E49097888422E
:1084D00033D01C480078A077A07E00F0010078B16E
:1084E00000BF608B40F00200608300BF204600F0B8
:1084F00023FE00BF608B4FF6FC710840608300BF15
:10850000A07E00F0080048B100BF608B4FF6F77105
:108510000840608300BF2046FFF79EFEE568A06F1D
:1085200048B1002009490870204601F0F3FB0748D4
:10853000007800B1C5E72C4600E0E468002CC3D108
:1085400070BD0000EA010020E0010020E8010020E9
:1085500010B5044621460120FDF720FD10BD0000A6
:108560002DE9F04706460C469046994614E025460C
:1085700024686868FEF7EFF80746B6F86600C01B87
:10858000A6F866002889124909880844104908801D
:10859000284602F034FA00BFB4B1E1684868FDF73C
:1085A000DFFA8246E1688889FDF7E7FA00F0030008
:1085B00008B1012000E00020218908445044054909
:1085C0000968401A0028D2DD2046BDE8F087000087
:1085D000080200200402002010B5044621460220B3
:1085E000FDF7DCFC10BD10B50446606F20B1606F74
:1085F00002F012FA0020606710BD00000D480188EB
:108600000088401C0B4A10800B48006818B10B48CA
:108610000088814205DA0A48006800F11402505CC3
:10862000704706480078081AC2B203480068805CA8
:10863000F6E70000FC010020F8010020F601002010
:10864000F001002070B50B48046810E0E568A07EDA
:1086500000F0080048B100BF608B4FF6F77108408A
:10866000608300BF2046FFF7F7FD2C4600BF002CBB
:10867000ECD170BDE001002010B5F7F755FEC0F356
:108680000D0000F540400149088010BDD0010020D8
:108690002DE9FE4F05468B46FC49686808606889ED
:1086A000142800DA6FE2FA4A11685069FCF73EFBC1
:1086B00028B9F748007D00F0F000E02800D162E220
:1086C000F24909688889FDF758FA00138700142FCA
:1086D00002DB2889B84200DA55E2A7F11400ED491F
:1086E00008800020EC4908606889B84208DBE94846
:1086F0000088EA49088039462846FEF7BAF923E09F
:1087000014212846FEF7B5F96889E4490880E14854
:1087100000880988401A1FFA80FAE0480188284634
:10872000FEF7A7F928684089504500DA2BE228684F
:108730004068D949086051462868FEF79AF92889A7
:10874000A0EB0A00288100BFD04909680888FDF71E
:1087500014FACE4909680880CC4909684888FDF7B1
:108760000CFACA4909684880C84909684868FDF791
:10877000F7F9C64909684860C9490860C3490968EA
:108780008868FDF7EDF9C14909688860C549086046
:10879000BE490968C889FDF7F0F9BC490968C88174
:1087A000BA4909688889FDF7E8F900F03F00BE4939
:1087B00008702889BD490880BB48007800F0030094
:1087C00040B108460088401C0880288909888842F2
:1087D00000DDD8E14FF00009B548046831E0207AA7
:1087E00050B1217AAA48406890F83000401CC0B2CD
:1087F000814201D0A14623E0208BA4490968098861
:1088000088421BD1E08AA14909684988884215D16C
:108810009F4960680969884210D19D49206849696B
:1088200088420BD1B9F1000F07D0E068C9F80C00FD
:108830009F480068E0609E48046004E0A14600BFD5
:10884000E468002CCBD100BF002C6AD199480468A1
:108850002BE0207A48B1217A8D48406890F83000AA
:10886000401CC0B2814200D01EE0208B87490968BD
:108870000988884217D1E08A844909684988884272
:1088800011D183496068096988420CD18049206808
:108890004969884207D1204602F010FC2846FEF7BD
:1088A0000FF8BDE8FE8F00BFE468002CD1D1A146CF
:1088B000814806681FE0307A50B1317A74484068C8
:1088C00090F83000401CC0B2814201D0B14611E0A6
:1088D000F08A6E4909684988884209D16C49306834
:1088E0004969884200D108E00EB1306800B904E05F
:1088F000B14600BFF668002EDDD100BF8EB1B9F1E0
:10890000000F07D0F068C9F80C006B480068F060F1
:1089100069480660304600F01DFA2846FDF7D0FF92
:10892000BFE7002C73D000206449086028890881C3
:108930000846456055480068C860002060490860E6
:1089400060490870604908805748007800F00800C6
:1089500018B1687B40F001006873A06F80B12046B9
:1089600001F0D8F90D3028B1A06F48B14F48008808
:10897000002805DD608D10B9204602F059F8D0E0DE
:1089800052480460204600F0E7FE804608F10D00E2
:10899000002816D04B48007800F0080090B100BFC6
:1089A000D4F8900028B16FF00D01D4F89020206920
:1089B000904700BF21463E4800F099FE2046FFF751
:1089C000C7FDADE04FF000083F480088002819DDE2
:1089D0003D48B0F800A000BFD4F8800038B152463E
:1089E0002146D4F8803020699847804601E04FF056
:1089F000000800BF08F10D0000B992E000203249E4
:108A0000088000BF204600F0D3F808B189E098E064
:108A10002B48006860B3A07E00F0100038B12848F1
:108A20000068FDF74DFF2046FFF78AFA79E000BFA6
:108A3000D4F8840048B100232149D4F884C02069C7
:108A40000A682146E047804607E000231C4821468B
:108A50000268184601F066FE804600BF08F10D006E
:108A600000B95EE0B8F1000F02D015480068A067B9
:108A70001448007800F0200050B3A06F48B3A06FF6
:108A8000407B40F02000A16F48733EE0F0010020E1
:108A90003CBF0020F4010020F8010020F601002076
:108AA00000020020040200200C0200200A02002024
:108AB000E0010020E4010020DC01002034F6002069
:108AC000100200200D0200200802002014020020E5
:108AD0001BE0FFE7208DB0F5066F02D0208D401C13
:108AE000208500BFD4F8840040B100231A462146F7
:108AF000D4F884C02069E047804601E04FF00008C8
:108B000000BF08F10D0000B90BE00020204908600B
:108B1000204600F04DF800B103E0204600F00CFBC9
:108B200000BF00201A4908601A4908601A484068C6
:108B300040B319494868FDF7C3FE00201649486054
:108B400020E0164909688889FDF717F800F004004D
:108B5000A8B9124800680088104909684988104A75
:108B6000CDE9002102900F4800680F49098842189A
:108B70000B4B1B1D0D480168002001F0FFFE28462D
:108B8000FDF79EFE8DE62846FDF79AFE00BF88E6BB
:108B9000140200201002002034F60020F001002012
:108BA0004CBF0020000200200A0200200402002026
:108BB00010B504460F48007800F01000B8B1A07E50
:108BC00000F0100050B900BFD4F8900028B16FF049
:108BD0000E01D4F890202069904700BF2146064836
:108BE00000F085FD2046FFF7B3FC012010BD0020FA
:108BF000FCE700000D020020E00100202DE9F0411B
:108C000004460026216D481EFCF7AAFF8046434615
:108C100000223146204600F0BBFB054615B9701E08
:108C2000BDE8F081334600222946204600F033FC9F
:108C3000231D22462946204600F003FC07463846FD
:108C4000EEE700002DE9F04107467F2F01DD7F2090
:108C500000E0384606460EB9BDE8F081701EC6B287
:108C60004FF0000800250F48046813E0607DB04213
:108C700008DB607DB0420CD10B49206A0968081AF4
:108C8000404506D30849206A0968A1EB000825463B
:108C9000667DE468002CE9D115B12846FFF750F94C
:108CA00000BFD9E7E0010020D40100202DE9F04108
:108CB0000546002700260D4804680EE0207DA842E6
:108CC0000AD10B49206A0968081AB84204D3084936
:108CD000206A09680F1A2646E468002CEED11EB1FE
:108CE00000213046FFF7AEF8BDE8F081E00100203A
:108CF000D401002070B5002600250B4804680BE065
:108D00000A49206A0968081AB04204D30749206A50
:108D100009680E1A2546E468002CF1D115B12846E1
:108D2000FFF70EF970BD0000E4010020D40100201F
:108D300070B50546012407E0054951F8241008687C
:108D4000294601F035FD641C042CF5D370BD0000EC
:108D50008CF600082DE9FE4305464D48007800F0EA
:108D6000040008B1BDE8FE834948007800F0100017
:108D7000B0B1484800680088464909684988464AB1
:108D8000CDE900210290454800684549098842180C
:108D9000414B1B1D43480168284601F0EFFD75E07B
:108DA0003B48007800F0020000286FD0687DFFF794
:108DB000E1F8044674B900BFA86938B14FF0FF323A
:108DC0000021AB6928699847804601E06FF00F08E1
:108DD00000BFC7E730481038406920602E4810387F
:108DE00000696060E88AE0822A4800680088208381
:108DF0000320207529480068401C6062606AE062B8
:108E0000204600F041F90646A66526656664E665DB
:108E100022480068401E606528692061E567687A1D
:108E200000F00C006072287A207200BF00BF1E485C
:108E30000068E0601C48046002F024F900BF0120D3
:108E40001A49087000BF204600F09EFB11480068D8
:108E5000C08924F8600F20886080603C201DFCF7EA
:108E6000DDFA8046608E221D4146FFF792FA608649
:108E700012212046FFF7A5FA074627B10021204618
:108E8000FEF7E0FF6EE7204600F056F900BF69E705
:108E90000C020020F00100204CBF00200002002046
:108EA0000A02002004020020E0010020E801002066
:108EB00070B504460D4600222946204600F002F80F
:108EC00070BD00002DE9F041044688461746002594
:108ED00000BF14B96FF00F0656E000BF00BF207D41
:108EE00010B16FF00E064FE000BF207D012803D1C6
:108EF00025466FF0080647E00220FDF789F8054691
:108F000015B94FF0FF363FE020692861E08AE8821A
:108F100001202875607D6875607A6872002028726B
:108F2000E07AE872A07AA87220682860E08AD8B156
:108F300000BF18480068A04205D116480068C06804
:108F4000144908600DE01349086806E0C168A142B1
:108F500002D1E168C16002E0C0680028F6D100BF1C
:108F600000BF0020E06000BF2046FFF7F1FA0A488A
:108F7000A86100BF09480068E8600848056002F081
:108F800081F800BF002600BF07B13E702846BDE84B
:108F9000F0810000D80100205F7F0008DC01002084
:108FA00070B506460D46D6B13068C0B10C480168B0
:108FB000304600F01BF80B480168304600F016F808
:108FC0006DB1286858B10848046806E02068316827
:108FD000884201D128682060E468002CF6D170BD79
:108FE000E0010020D8010020DC0100202DE9F04143
:108FF00005460E4634460AE020682968884205D1B5
:10900000E7682046FEF79CFF3C4600E0E468002C41
:10901000F2D1BDE8F08110B54020FEF7ABFF10BDE6
:1090200010B5002300BF16480088401C144C208057
:10903000204600884FF6FF74A04203D14FF4404011
:109040000F4C2080002116E00E4850F821000268E5
:109050000DE0D08A0A4C2488A04207D1581C83B264
:10906000B3F5804F01DB002010BDDCE7D268002A99
:10907000EFD1481CC1B20429E6DB01480088F3E7C0
:10908000D00100208CF60008014605480068054A1A
:1090900012681044024A10601046006870470000D1
:1090A000EC010020D401002070B505460C46E968AB
:1090B0008889FCF762FD00F0010020B1204601F034
:1090C000ABFC002433E013E0E1688889FCF755FD30
:1090D00000F0010038B10120FCF74FFDE9688989F3
:1090E0000843E968888126462468304601F087FCF9
:1090F0004CB1E06840682189084429890D4A12680A
:109100001144081AE0D594B128890A49096808442D
:10911000E1684968401A002809DDE068808805494F
:109120000988401A288129896868FDF761FC2C604C
:1091300070BD0000000200202DE9F84F044693485E
:109140000068A04202D10020BDE8F88FB4F86000AA
:10915000B4F84810884202DAB4F8600001E0B4F8CC
:1091600048008146E56E45B9A07E00F0020018B1C6
:10917000204601F05DFCE7E7FEE0221D2146204687
:1091800001F0EDFB074617B96FF00300DCE70CB107
:10919000206858B90FB1381D00E00020014611B910
:1091A0006FF00300D0E70868206000BFE9684868F6
:1091B000FCF7D6FC616C401A29890844484519D946
:1091C000B4F8600048450CD1206F50B994F899006C
:1091D00038B9002004F8980F012060700020A070BA
:1091E000983CA07E00F0020018B1204601F020FC5F
:1091F000AAE7C1E0002084F89900266F26B100E0BC
:10920000366830680028FBD1A3E0206FA0B1A07EB3
:1092100000F0440080B9E06E38B1E06E006858B9E3
:10922000E06E0089618E884206DAB4F8640018B1F5
:10923000B4F86600082801DB012000E0002020B916
:10924000A07E00F0A00000B98FE0207D022807D0AA
:109250001020FCF792FCE96889890843E968888155
:109260003A462146284600F01FF90090009838B190
:1092700000BF608B40F08000608300BF009863E710
:109280002868E066207D022806D000BF608B4FF67C
:10929000FC710840608300BFE9684868FCF760FC27
:1092A0008046E9688889FCF768FC00F0030008B193
:1092B000012000E000202989084408EB000A206D05
:1092C000B0EB0A0001D5C4F850A0E9688889FCF722
:1092D00054FC00F0030008B1012000E000202989BF
:1092E000084470B300202860206F10B925672E460F
:1092F0002EE0E9684868FCF733FC8046F16848686E
:10930000FCF72EFCB8EB00001CD504F1700801E05E
:10931000D8F80080D8F8000068B1D8F80010C96803
:109320004868FCF71DFC8346E9684868FCF718FCB0
:10933000BBEB0000ECD4D8F800002860C8F800505F
:1093400006E002E03560366802E0284601F057FB8F
:10935000E56E55B1E9684868FCF702FC616C401A9B
:109360002989084448457FF650AF00BFE06E10B928
:109370000020A4F8680000BF00BF608B4FF67F712B
:109380000840608300BF0020DEE6000014020020D9
:109390002DE9FF4104460E4617469846608D10237E
:1093A000218BE28ACDE901130092039043463A46AD
:1093B0003146606A00F00AF805461DB1618D606AA9
:1093C0000844E062284604B0BDE8F0812DE9F05F72
:1093D00082460D4617469846DDF830B005F1140078
:1093E000384481B24FF420722220FDF7CBF80646B4
:1093F00026B374680A98FCF7C0FB20800B98FCF732
:10940000BCFB6080C4F804805046FCF7A9FBA06058
:10941000A946E91705EB91718910491D4FF6FF72B6
:1094200002EA013141EA0B00FCF7A7FBA0810D988D
:10943000FCF7A3FBE0810020208260823046BDE87B
:10944000F09F2DE9FE4F0446884691469A465246C3
:109450004946204601F083FA8346BBF1000F02D152
:109460006FF0030511E014B1E67AA77A01E0FF2658
:1094700000270620334652464946CDE9010B0097A6
:109480004046FBF74BFE054600BF4046FDF718FA85
:109490002846BDE8FE8FF0B5044615461E4600235B
:1094A000486800F11402F0BD2DE9FE4F04460D4658
:1094B0001646204600F05EF810B10020BDE8FE8F91
:1094C000686AFCF74DFBE1688860688DFCF755FB26
:1094D000E168C881698D686A0844E862E06800F163
:1094E0001408A07A00F0010078B12A1D31464FF42B
:1094F0000670FEF74EFF82464AF00170FCF730FB23
:10950000C8F8000008F1040800BFB5F930000028D1
:1095100001DA00202886686B38B91548006868634E
:10952000E1684868FCF71CFBA863A089616889882A
:10953000401A87B260684089C01B616848816068D2
:109540000089C01B616808816168E068486000208C
:10955000E16808820621A87A8DE84300EB7A2A1D8B
:1095600029466068FBF7DAFD81464846A6E7000019
:10957000D401002001464868807B012801D00120E9
:1095800070470020FCE700002DE9F0410646234823
:109590000088002840D000202149088036E0FFF7ED
:1095A0002DF8074627B1012F04D0022F1FD102E06A
:1095B000BDE8F08128E0FFF721F8042806D118481B
:1095C0000088801C15490988884200DDF0E7FFF714
:1095D00015F80502FFF712F80543B5F5067F00DC24
:1095E00015B94FF4067000E0284670860CE0FFF7CE
:1095F00005F80446022C00DADAE7A01E08490988BB
:1096000008440749088000BF00BF00BF0448008825
:10961000024909888842C2DB00BFC9E7F401002083
:10962000FC0100202DE9FF5F0C4616469846DDE957
:109630000FAB0E9FA146B4421BDA0AF0020050B9EC
:10964000B87E00F04000A0B9BBF1000F03D0F86E67
:1096500008B9386F68B104F21B2020F00300B04253
:1096600001D9304603E004F21B2020F003001FFA6A
:1096700080F94FF4207249460098FCF783FF0546B5
:109680001DB9002004B0BDE8F09F6889001BA8F850
:1096900000002C816C812846F4E710B5044600BF19
:1096A00004B910BD00BF207DF8B1207D0A281CD070
:1096B000207D012819D0A06F20B1A06FFDF700F91F
:1096C0000020A067606F10B12046FEF78CFF4FF0BE
:1096D000FF302086E06E01F09FF9206F01F09CF9C9
:1096E0000020E0662067A4F8680000BFD9E770B5E5
:1096F00005460C4600BF2868A04203D12868C06810
:1097000028600CE0286806E0C168A14202D1E16847
:10971000C16002E0C0680028F6D100BF00BF002091
:10972000E06000BF2046FFF7B8FF207D0A280FD079
:10973000207D01280CD0A07E00F0010040B100BFC8
:10974000608B40F00200608300BF2046FFF7F4FC0E
:1097500000202075E08270BD2DE9FE4304460027FD
:109760000026F848007800F00400A8B3207D022805
:1097700006D1F549206D096888421BD1012719E0FF
:10978000F249606A0968884201D1012712E0EF4975
:10979000606A0968081A0DD4218D606A0844EB4993
:1097A0000968081A002805DC00BF608B40F0020041
:1097B000608300BF8FB1E648007840F00800E449BC
:1097C000087000BF608B4FF6FE710840608300BFD9
:1097D0006FF00D00BDE8FE8301E00020FAE7D948F4
:1097E000007800F0020068B1207D02280AD0207DB8
:1097F000032807D000BF608B40F00200608300BFE9
:109800000020E7E7A07E00F0100010B9D148006802
:109810002062002084F89B0084F89A002046FFF71D
:10982000B3FE207D801E08287CD2DFE800F004B063
:10983000FCFBFAF9F8F7C348007800F010000028A4
:1098400071D0C048007800F0020000287AD0606C27
:10985000401CBD490968884274D1BC480068401C5E
:109860006062606AE062B84800686064BA48006894
:10987000C089A4F86000B4F86000A4F86200B3489E
:109880000068401E606504202075201DFBF7C6FDA2
:109890008046608E221D4146FEF77BFD6086608E0D
:1098A0008100400041F21C12904202D9608E4000BB
:1098B00001E041F21C10814202D2608E80000AE079
:1098C000608E400041F21C11884202D9608E400037
:1098D00001E041F21C1024F8480FE08B401EE083A9
:1098E000A56A483C1DB9E56E2868E06601E0286875
:1098F0002067284601F083F8206F18B94FF0FF3039
:10990000208603E00020208684F8420000BFD4F8BF
:10991000880048B100222146D4F888302069984751
:10992000064602E0E6E10DE0002600BF06F10D006C
:1099300010B96FF00C004DE700BF608B40F00200E3
:10994000608323E07F48007800F01000F0B1824887
:1099500000680088804909684988804ACDE900216B
:1099600002907A4800687E49098842187B4B1B1D8B
:1099700075480168204601F001F894F84200062875
:1099800004DA00202086204600F092FFB3E16D4803
:10999000007800F0100000287DD0606C401C6A49FF
:1099A0000968081A62D46849206D0968081A0028F5
:1099B0005CDC04202075E06F10B96FF005060EE046
:1099C00000BFE06F806938B1E16F206900228B69C8
:1099D00021469847064601E06FF00F0600BF46B1EA
:1099E00006F10D0010B12046FEF7AAFA6FF00C0048
:1099F000F0E6204600F0DEF95A48008820B15948C8
:109A00000088401E57490880608E8100400041F266
:109A10001C12904208D9608E400007E054E114E126
:109A20004CE0D4E05CE04AE041F21C10814202D2FA
:109A3000608E80000AE0608E400041F21C11884276
:109A400002D9608E400001E041F21C10A4F84800E9
:109A50003F48007800F0200000B300BF608B40F06A
:109A60000200608300BF0720207526E03A480068A6
:109A70000088394909684988384ACDE900210290AF
:109A800032480068364909884218344B1B1D2E485D
:109A90000168204600E002E000F070FF0DE0294878
:109AA000007800F0020040B1606A401E2749096852
:109AB000884202D1204600F087FE1CE100BF20460C
:109AC00000F078F92248007800F0200038B100BF9B
:109AD000608B40F00200608300BF072020750AE120
:109AE000204600F067F91A48007800F02000E8B33B
:109AF0001448007800F01000C8B31349206D0968BD
:109B000088424CD1E06E90BB00BF608B40F00200F9
:109B1000608300BF2046FFF7C0FD00BF00BF1248B2
:109B20000068A04205D110480068C0680E4908606E
:109B300023E00D4908681CE0C168A14218D1E16822
:109B4000C16018E00C020020040200200002002086
:109B50000D020020D4010020F00100204CBF0020A5
:109B60000A02002008020020E001002020E016E0A8
:109B7000C0680028E0D100BF00BF0020E06000BF47
:109B800001205E49087000BF0A20207500BF5C48B4
:109B90000068E0605A48046001F074FA16E000BF03
:109BA000608B40F00200608300BF082020750DE04C
:109BB0005448007800F0100040B15349206D096806
:109BC000884203D1E06E08B90620207593E0204654
:109BD00000F0F0F84D48007800F02000A0B300BF7E
:109BE000608B40F00200608300BF2046FFF755FD08
:109BF00000BF00BF46480068A04205D14448006845
:109C0000C068434908600DE04149086806E0C16842
:109C1000A14202D1E168C16002E0C0680028F6D12B
:109C200000BF00BF0020E06000BF01203349087082
:109C300000BF0A20207500BF31480068E06030484E
:109C4000046001F01FFA00BF55E0204600F0B2F8B2
:109C50002C48007800F01000A8B32B49206D09684B
:109C6000884230D1E06E70BB2046FFF716FD00BF82
:109C700000BF27480068A04205D125480068C06899
:109C8000234908600DE02249086806E0C168A14246
:109C900002D1E168C16002E0C0680028F6D100BFCF
:109CA00000BF0020E06000BF01201449087000BF21
:109CB0000A20207500BF12480068E0601048046068
:109CC00001F0E0F900BF16E0204600F073F80D48FF
:109CD000007800F0100060B10B49206D09688842DF
:109CE00007D1E06E28B90948007840F01000074914
:109CF000087000E000BF00BF00206BE5E801002015
:109D0000E40100200C020020040200200D020020CB
:109D1000E00100202DE9F041044600BF1CB96FF0BE
:109D20000F00BDE8F08100BFA06F477BA66F002049
:109D3000A06700BFD4F8840040B10023324621461A
:109D4000D4F884C02069E047054606E00023324687
:109D50002146184600F0E6FC054600BFF5B907F0BD
:109D6000200028B3208DB0F5066F02D0208D401C56
:109D7000208500BFD4F8840040B100231A46214654
:109D8000D4F884C02069E047054600E0002500BF04
:109D900005F10D0060B96FF00C00C2E705F10D0090
:109DA00010B96FF00C00BCE7A6676FF00400B8E7CD
:109DB0000020B6E72DE9F05F04464FF00009FE48A9
:109DC000007800F01000002870D0B4F86000A16D99
:109DD00000EB0108F949606D0968401A15D4F7498C
:109DE000606D0968884204D1F549A06D0968401A80
:109DF0000BD4F349A06D096888421AD1F148006874
:109E0000C089B4F86010884213D9EE480068C08950
:109E100024F8600F608834F86019884203DAB4F8D7
:109E20006000A4F86200E54800686065E4480068E6
:109E3000A065E349606C0968081A00284ADCE2481A
:109E4000008890BBB4F86010A06D084440453AD13A
:109E5000B4F93000002836DBD949606C09688842C3
:109E600031D14FF0010994F84300401CC0B294F87E
:109E70004310884204DD94F84300401C84F84300FA
:109E800094F84300032817DD00BFB4F84800618E42
:109E9000084480B2B4F84810884208DBB4F848009F
:109EA000618E0844A4F8480005E00CE02AE14FF672
:109EB000FF70A4F8480000BF94F84300032802DBB9
:109EC000204600F0BBFCB9F1000F02D1002084F85D
:109ED0004300EBE0606C401CB9490968081A7DD466
:109EE000B749206D0968081A002877DCA07E00F0C9
:109EF000040060B100BF608B4FF6FB7108406083C7
:109F000000BF48346088208000206084483C0020E6
:109F10002434A077608BB4F9181000EBE10000B294
:109F2000A083208CA6490988081A85B20020E07712
:109F3000A3480068206214F8100C243C042865DB58
:109F4000B4F84800B4F84A10884227DA628B02F469
:109F500000620AB1012200E002221146628E4A43E9
:109F600092B2AA4201DD2A4602E0628E4A4392B2D0
:109F7000104600BFB4F84820024492B2B4F848300A
:109F80009A4205DBB4F848200244A4F8482003E0D4
:109F90004FF6FF72A4F8482000BF37E000BFB4F8C6
:109FA0006A00284480B2B4F86A10884205DBB4F82D
:109FB0006A002844A4F86A0003E04FF6FF70A4F892
:109FC0006A0000BFB4F86A00B4F8481088421DDB8C
:109FD0004834608C2188401A608400E063E0483C8B
:109FE00000BFB4F84800618E084480B2B4F848104D
:109FF000884206DBB4F84800618E0844A4F84800A3
:10A0000003E04FF6FF70A4F8480000BF6FA220469F
:10A01000D4E91B31FEF7A4FA20676EA22046D4E9EA
:10A020001B13FEF79DFAE066206F18B94FF0FF3062
:10A03000208601E00020208600202077E06E10B905
:10A040000020A4F86800B4F8640064490988084452
:10A05000A4F86400608B00F4006018B3206F88B926
:10A06000E06E40B1E16EC9684868FBF779FDE16CCC
:10A07000081A002816DC00BF608B4FF2FF71084001
:10A0800060830FE0216FC9684868FBF769FDE16CE8
:10A09000081A002806DC00BF608B4FF2FF710840F1
:10A0A000608300BF02E0204600F0C2FC606B48B352
:10A0B0004349A06B0968401A24D5A08E48490988F5
:10A0C000081A07B2B4F93C00A7EBE00007B2A08F72
:10A0D000384400B2A087002F01DA784207B2B4F901
:10A0E0003E00A7EBA00007B2E08F384400B2E08743
:10A0F000E08FB4F93C1000EBE10000B2A4F840009E
:10A10000002060633048008800286DDD207D07282E
:10A110006ADA2A48616A0068401C081A34D4274861
:10A12000616A0068284A12881044401E081A0028F4
:10A130002ADC2C4845682149606A0968A0EB010ABD
:10A140001FFA8AF627480089801B2649088108469D
:10A1500040680089801B1FFA80FB07E06889301A7D
:10A1600086B2A5F808B0002068812D686889B042E1
:10A17000F4DB31462846FCF77CFC1049606A086035
:10A180001849C96848600AE00C49606A0968081AF9
:10A1900005D500BF608B40F00200608300BF074917
:10A1A000606A0968081A75D4218D606A0844401EE7
:10A1B00002490968081A18E00C0200200002002079
:10A1C00004020020F00100200A020020756E616385
:10A1D0006B656400756E73656E7400000802002084
:10A1E000D401002034F600207CE2002852DCF7493C
:10A1F000606A096888426ED1F549C9688889FBF7A9
:10A20000BCFC00F0030008B1012000E00020F04990
:10A2100009890844EF490880208D0988884240DA7E
:10A22000EB49C9688889FBF7A8FC00F0010098B1E8
:10A23000E749C9688889FBF7A0FC00F03E0528467D
:10A24000FBF79BFCE249C96889894CF2FF02114087
:10A250000843DF49C9688881208DDD490881C968C4
:10A260008889FBF78AFC00F0020020B1D8480089F9
:10A27000401ED7490881D64A11895068FCF7B8FBBF
:10A28000D349C9688889FBF778FC00F0030010B156
:10A29000012001E022E20020CD4909890844CD498E
:10A2A0000880606F002813D0C949C9688889FBF706
:10A2B00064FC00F0010060B107E0656F606F00684A
:10A2C0006067284600F09BFB00BF606F0028F4D158
:10A2D00072E0656F2FE00AE1E9688889FBF74DFCC1
:10A2E00000F0010008B3BA49C9688889FBF745FC4A
:10A2F00000F00200C8B90120FBF73FFCB449C9686F
:10A3000089890843B249C9688881B149C96888897F
:10A31000FBF733FC00F0030008B1012000E000204F
:10A32000AB4909890844AB4908802E462D68304660
:10A3300000F065FB00BF55B1E86840682989084412
:10A34000A2490968A34A12881144081AC4D58DB3DA
:10A350009E4800689F4909880844E9684968401A8E
:10A36000002827DDE868808898490988401A9849BC
:10A370000881C9688889FBF700FC00F0020020B161
:10A3800093480089401E92490881914A118950687A
:10A39000FCF72EFB8E49C9688889FBF7EEFB00F0BD
:10A3A000030008B1012000E0002089490989084420
:10A3B00088490880656700BF844800688549098826
:10A3C00008446062208D83490988401A2085204610
:10A3D00000F0E6FE7E4840680089002806DD7C48E3
:10A3E00040687D4908600020794948607849C9681B
:10A3F0008889FBF7C2FB00F0010028B1774800789C
:10A4000040F020007549087050E0656F606FC068CB
:10A4100040686E490860E9688889FBF7AEFB00F088
:10A42000030008B1012000E0002029890844616A86
:10A4300008446062E9688889FBF79FFB00F003002D
:10A4400008B1012000E0002029890844218D081A64
:10A450002085204600F0A4FE6868008900280DDDF4
:10A460005D48006828B15C4869680068FCF75BF9E2
:10A4700002E059496868086000206860E9688889D6
:10A48000FBF77BFB00F0010050B15448007840F02E
:10A49000200052490870207D042801D10720207532
:10A4A00028686067284600F0AAFA00BF606F28B1EC
:10A4B000606FC0684068616A8842A6D000BFA07E15
:10A4C00000F0010060B100BF608B4FF6FE710840E4
:10A4D000608300BF00BF608B40F00200608305E036
:10A4E00000BF608B40F00100608300BF0EE1606F31
:10A4F00020B9374800F071FA6067EBE00026656F1D
:10A50000E3E0E868406831490968884217D130487B
:10A5100000892989884211DD2D4800F05EFA8246C3
:10A52000BAF1000F09D016B1C6F800A001E0C4F8D6
:10A5300074A029465046FEF7B7FDC9E0C8E0A6B9A9
:10A54000E868406821490968081A0DD5204800F0DC
:10A5500044FA8246BAF1000F05D0C4F874A0294627
:10A560005046FEF7A1FDB3E03BE0F0684068401CB8
:10A5700016490968081A33D4E8684068401E134930
:10A580000968081A00282BDC114800F026FA8246D8
:10A59000BAF1000F18D0F0684068318908440B49BF
:10A5A0000968401A002809DDF06880880749098891
:10A5B000081A308131897068FCF71AFAC6F800A0D1
:10A5C00029465046FEF770FD82E0000000020020A0
:10A5D00034F600200A020020100200200D020020A4
:10A5E00000BF2E462868E8BBE8684068484909680B
:10A5F000081A002868DDE9688889FBF7BEFA00F0D0
:10A60000010000B164E0434800F0E7F928602868E1
:10A6100048B3E8684068298908443D490968401AF8
:10A62000002809DDE868808839490988081A2881E6
:10A6300029896868FCF7DCF9218D606A0144364895
:10A640000088334A12681044401A00283BDD29680C
:10A65000C9688889FBF791FA00F00100B0B1296858
:10A66000C96801E030E02EE08889FBF786FA00F047
:10A670003E0A5046FBF781FA2968C96889894CF27D
:10A68000FF02114008432968C9688881A08C218D88
:10A6900008441F490988401A296808812A681189D5
:10A6A0005068FCF7A5F92968C9688889FBF765FA3D
:10A6B00000F0030008B1012000E0002029680989AA
:10A6C00008441549088003E02D68002D7FF419AF78
:10A6D00000BF00BF204600F0ABF917E0204600F0B5
:10A6E000A7F913E00A49606A0968081A08D4218D9D
:10A6F000606A0844401E06490968081A002805DDFA
:10A7000000BF608B40F00200608300BFBDE8F09F97
:10A710000002002034F600200A02002008B1C0F830
:10A72000841070472DE9F04107460D4614461E4639
:10A7300000BF1DB96FF00F00BDE8F08100BF3CB154
:10A740002189284600F00BF82046FCF7B9F804E010
:10A750001EB92846FDF7CAFCEEE70020ECE72DE91C
:10A76000F04104460F4600BF0CB9BDE8F08100BFC0
:10A77000208D384485B2B5F5066F02DC208DA842E5
:10A7800003DD4FF40660208500E02585204600F0BB
:10A7900007FD0646B6F5067F08D300BF608B40F084
:10A7A0000200608300BF2046FEF7C6FC00BFDCE766
:10A7B0000246104605E0C36F8B4201D10023C367F8
:10A7C000C0680028F7D170472DE9F0410446206F9A
:10A7D00018B96FF00500BDE8F081256F2846FEF737
:10A7E000C9FE10B16FF00500F5E72868206704F195
:10A7F0006C0600E03668306858B13168C96848684E
:10A80000FBF7AEF90746E9684868FBF7A9F9381A7B
:10A81000F0D4306828603560286810B90020A4F8AA
:10A82000680094F84200FF2804DA94F84200401CC3
:10A8300084F842000020606300BFCCE710B50446F6
:10A84000206FA0B3A07E00F0040080BB2046FFF77D
:10A85000BBFF60BBB4F84810B4F86020914202DA44
:10A86000B4F8481001E0B4F86010084601EBD0716C
:10A87000C1F34F01A4F84A10B4F84A00618E4900B0
:10A88000884204D2608E4004000CA4F84A00B4F858
:10A890004A00618E032202FB0100A4F8480000BFB9
:10A8A000608B40F00400608300BF0020208610BD54
:10A8B00010B50446204600F014F810B9204600F008
:10A8C00001F810BD10B5044694F84200FF2804DAE0
:10A8D00094F84200401C84F842002046FEF72CFC0D
:10A8E00010BD70B50446206F10B96FF0050070BD43
:10A8F000256F07E02846FEF73DFE10B16FF005001A
:10A90000F5E72D6828680028F4D12846FEF732FEC6
:10A9100010B16FF00500EAE7E06E2860206FE06696
:10A920000020206700BF608B40F40060608300BFA0
:10A93000E9684868FBF714F90646E9688889FBF777
:10A940001CF900F0030008B1012000E00020298973
:10A9500008443044E0640020606300BFC7E770B57E
:10A9600004460E4615462CB1207A18B1207AFBF722
:10A9700063FC70BD2846FAF751FDFAE72DE9F04F68
:10A9800085B081460C4615461E46DDF838A04FF0CE
:10A99000000846F2080B2046FBF7E2F81422049068
:10A9A000DDE90F018DE80708002241462846049B97
:10A9B000FEF70CFD074617B905B0BDE8F08F43461A
:10A9C000002239464846FEF766FD53463246394670
:10A9D0004846FEF736FD00BFEEE770B5054603209A
:10A9E000FBF716FB04460CB9002070BD95E80F007C
:10A9F00084E80F006068FCF735F82046F5E710B5ED
:10AA0000044644B1606810B16068FBF759FF214605
:10AA10000320FBF7C3FA10BD70B5044605E02568B6
:10AA20002046FFF7ECFF2C4600BF002CF7D170BD8D
:10AA30002DE9F04704460025A9460DB1042000E0A9
:10AA4000002005F0020109B1002100E000210844C6
:10AA500005F0080109B1002100E00021084405F0DB
:10AA6000100109B1002100E0002100EB0108206D78
:10AA7000FBF776F882465346002241462046FEF711
:10AA800087FC06464EB900BF608B40F00300608330
:10AA900000BF6FF00100BDE8F0874B462A46314603
:10AAA0002046FEF7F8FC231D224631462046FEF7DD
:10AAB000C8FC07462FB100BF608B40F003006083E5
:10AAC00006E000BF608B4FF6FC710840608300BF5A
:10AAD0003846E0E770B50446E06EE8B1E56E00E0A8
:10AAE0002D6828680028FBD1E9688889FBF745F8BC
:10AAF00000F0070078B90120FBF73FF8E968898981
:10AB00000843E968888100BF608B40F020006083C3
:10AB100000BF002070BD00BF01212046FDF751FCA1
:10AB2000F8E700002DE9F04F85B04FF00009EA4842
:10AB30000068401CE8490860E8480078401CE74984
:10AB4000087000BF0025E64804689DE1A07FE34946
:10AB50000978884202D12546E46895E1DF4800780B
:10AB6000A0770026B046207D022806D194F8420046
:10AB7000062802DB701CC6B2B5E094F842000C282F
:10AB800002DB701CC6B2AEE094F89900002841DDEB
:10AB900094F89A000C2802DB701CC6B2A3E094F86B
:10ABA0009900401ECF490F5C94F89800B84204DA2F
:10ABB00094F89800401C84F8980094F89800B842E3
:10ABC00027DB4FF0010AB4F8600030B9204600F0EE
:10ABD00048FD70B14FF0000A0BE0B4F86010204659
:10ABE00000F08AF928B92046FEF7A6FA08B94FF016
:10ABF000000ABAF1000F0BD0002084F8980094F8F6
:10AC00009900072804D294F89900401C84F8990010
:10AC100000BF68E0B4F93000002809DBB4F9300067
:10AC200047F6FF71884203DA208E401C00B220866E
:10AC3000B4F93000B4F94010884254DB2046FFF7E5
:10AC400050FE18B1206F70BBE06E60B3207D02280B
:10AC50001ED094F842200C2A02D294F8422000E040
:10AC60000C221146B4F93E20B4F93C3002EBE30269
:10AC70009D4B5B5C02FA03F047F6FF72904201DAEB
:10AC8000024601E047F6FF7212B2A4F8402000BF6E
:10AC900000202086B4F84800B4F86010884203DA37
:10ACA000B4F8480002E01EE0B4F860000490049894
:10ACB0004010A4F84A00B4F84A00618E4FF6FF72C3
:10ACC00002EA4101884205DA608E114601EA40003D
:10ACD000A4F84A00608EA4F848000020A4F86A0096
:10ACE0002046FFF7EFFD207D06280BD1A07E00F067
:10ACF000100038B17849206A0968081A282801D953
:10AD0000701CC6B2607A00F00800D0B3207D042821
:10AD100002D0207D072834D17449D4F89400084427
:10AD20004FF4FA71B0FBF1F06B4A216A1268511AC4
:10AD3000884206D2701CC6B208F1010000F0FF087C
:10AD40001FE094F89B1042F29F4211FB02F1D4F8ED
:10AD5000940000EBC1004FF4FA71B0FBF1F05E4AD1
:10AD6000216A1268511A88420BD22046FDF746FF2D
:10AD70008146B9F1000F04D194F89B00401C84F87F
:10AD80009B00606F68B15449206A0968081AB4F9D9
:10AD9000401001EB4101B0EB410F02D32046FDF71B
:10ADA00022FC207D032807D14B49206A0968081A34
:10ADB000282801D9701CC6B2207D092807D1464930
:10ADC000206A0968081AF02801D9701CC6B29EB31F
:10ADD000D4F890A02046FEF760FC15B1E068E8606A
:10ADE00002E03F49E0680860B8F1000F0BD0208B0B
:10ADF000E18A221DCDE90021029023462046626AA5
:10AE0000216DFFF7BBFDD4F810B0207D03902746DD
:10AE1000E4683846FDF79CFB00203549087000BF08
:10AE2000BAF1000F03D06FF00C015846D04700BFB5
:10AE30002F48007808B185E600E024E02546E46864
:10AE4000287F401C2877287F697F88421BDB0020F1
:10AE500028772749087000BFD5F88C0030B1294603
:10AE6000D5F88C2028699047814601E04FF0000911
:10AE700000BF1F48007800B164E6B9F1000F02D1AD
:10AE80002846FEF759F900BF002C7FF45FAE00257D
:10AE9000184804681BE000260F49206A0968081A50
:10AEA000F02801D9701CC6B27EB12046FEF7F5FB32
:10AEB00015B1E068E86002E00E49E06808602746E6
:10AEC000E4683846FDF744FB01E02546E468002CC1
:10AED000E1D105B0BDE8F08FD4010020EA010020E7
:10AEE000E001002085F6000878F60008B84C0A005A
:10AEF000E8010020E40100202DE9F04F85B005466F
:10AF00000E464FF0000A0024A346EC6E24B94FF021
:10AF1000FF3005B0BDE8F08F16B96FF00500F8E717
:10AF20002089B04201DC0020F3E7A77A07F0010096
:10AF300008B1042000E0002007F0020109B100215F
:10AF400000E00021084407F0080109B1002100E0F9
:10AF50000021084407F0100109B1002100E00021A0
:10AF6000084404902089801B1FFA80F90498484403
:10AF700081B24FF420723620FBF704FB8346BBF10D
:10AF8000000F00D174E0606800892189401A3044C4
:10AF900080B20290DBF80430049A991860684A463F
:10AFA000029BFBF74DFC484500D061E0E1688889D1
:10AFB000FAF7E3FD00F03F080020039008F00800D6
:10AFC00028B128F00808039840F00800039008F022
:10AFD000010028B128F00108039840F00100039017
:10AFE000E1684868FAF7BCFD30440346CDE90070DB
:10AFF00059462846039AFDF765F98246BAF1000FD3
:10B0000000D135E06068FBF7A6FB35F8661F081A2B
:10B01000288062681289A2EB090291B26068FBF78E
:10B02000E7FC2089A0EB090020814046FAF7A5FD46
:10B03000E16889890843E16888816068FBF78BFBD8
:10B04000298808442880DAF80400FBF784FB298863
:10B05000084425F866092068CAF80000C4F800A072
:10B06000DAF8000010B90020A5F86800002050E7C9
:10B07000BBF1000F02D05846FBF722FC4FF0FF3027
:10B0800047E7000010B50948006868B9084800683B
:10B0900010B90848006838B101200449086000224E
:10B0A0000549FA20FCF7C8FD10BD00002002002071
:10B0B000E0010020E401002091B700083EB50446FD
:10B0C0002248007800F0040000B13EBD1F4800781F
:10B0D00000F0020018B31E49606A0968081A26D4F5
:10B0E000218D606A08441A490968081A00281EDC84
:10B0F000184800680088174909684988164ACDE948
:10B100000021029012480068144909884218124B25
:10B110001B1D134801682046FFF730FCD5E70B489C
:10B12000007800F0010010B10E48006820620B4862
:10B130000088002808DD00BF608B40F002006083BB
:10B1400000BF2046FDF7F8FF00BFBEE70C0200205D
:10B1500000020020F00100204CBF00200A02002065
:10B1600004020020D401002010B5FDF7A3F9064821
:10B170000078401CC0B20449087000F0010008B11A
:10B18000FFF7D0FC10BD0000E90100200348007863
:10B1900040F0100001490870704700000D020020C7
:10B1A00010B501460B8D486AC218488ECB6AB0F5BF
:10B1B000866F02DD4FF4866000E0488E1844101A56
:10B1C00004D4088D4885C86A101A10BDCB6A486A35
:10B1D000C01A002802DD0020488504E04C6ACB6AD2
:10B1E000181B488500BF0020EFE72DE9FF4F91B005
:10B1F00004468A4617464FF0000B002500201090A9
:10B200000F900E9000260B900A908146099000BF87
:10B2100024B96FF00F0015B0BDE8F08F00BFB4F88F
:10B22000621001EBD1725210638E9A4201DD628E80
:10B2300004E0B4F8620000EBD072521092B20792B0
:10B24000079A0AB1079800E0608E079000BFBAF134
:10B25000000F02D16FF00F00DDE700BF3946204636
:10B2600000F0D0F90890089808B10898D3E7B4F82E
:10B2700066000D9000200C90E06E00287AD0E56EFC
:10B2800000E02D6828680028FBD1A87A00F00100B2
:10B2900008B1042000E00020A97A01F0020109B100
:10B2A000002100E000210844A97A01F0080109B159
:10B2B000002100E000210844A97A01F0100109B141
:10B2C000002100E0002108440690298906980144E5
:10B2D0000798401A1FFA80F8B4F868000A90BDF881
:10B2E0002800002822DD1095BDF82800B84202DAB7
:10B2F000BDF8280000E03846404501DD404607E043
:10B30000BDF82800B84202DABDF8280000E038464F
:10B31000814606EB090086B2BDF82800A0EB0900C3
:10B3200080B20A90A8EB09001FFA80F8BE4262DAE8
:10B33000B8F1000F5FDD288900285CDDB81B4045AF
:10B3400001DD404600E0B81B80B2059010951498CE
:10B3500000F00100F0B1012114980AAB4246CDE99A
:10B360000040029100200599FEF75CF9B0F1000B56
:10B3700001D133E140E00AEB0601DBF80400059A55
:10B38000F5F7BAF85846FBF7E6F90D99084480B28C
:10B390000D902CE06868049002E004980068049026
:10B3A000049800680028F8D10498007B00F0C000E1
:10B3B00040B90498416840890844504502D1059835
:10B3C000099013E0012200200599FBF7DBF8B0F1AA
:10B3D000000B00D102E10AEB0600CBF8040058464E
:10B3E000FBF7B9F90D99084480B20D9000BF05989C
:10B3F000304486B200BF00BF79E0B81B80B206902F
:10B400000C990798401A80B20590DDE90510884232
:10B4100001DA069800E005980490149800F0010005
:10B42000F8B10E9808B9012100E000211498CDE987
:10B43000004002910C9A0498104481B20AAB362065
:10B44000079AFEF7EFF8B0F1000800D1C6E00AEB6A
:10B450000601D8F804300C9A9818049AF5F74CF8BD
:10B460001DE0012236200499FBF78CF8039000B907
:10B47000B4E00AEB0601039841604FF420723620D5
:10B480000C99FBF77FF8B0F1000803D10398FBF7A4
:10B4900017FAA3E040460399FBF745F900BF404681
:10B4A000FBF759F90D99084480B20D900D980828C2
:10B4B00003D94046FBF704FA90E00B980090E06D4A
:10B4C0008319002241462046FCF7FCFE109000B98B
:10B4D00084E00E9810B910980E9002E0DDE90F108C
:10B4E000086010980F900498304486B200BFBE42A6
:10B4F00083DBB9F1000F21DDD5F8048017E0B8F83F
:10B5000008004844A8F80800D8F8000068B9B8F85E
:10B510000A20D8F8041088184A465146F4F7ECFF80
:10B52000B8F80A004844A8F80A00D8F80080B8F132
:10B53000000FE4D128894844288100BFBDF82800C5
:10B54000A4F86800BBF1000F09D059466868FBF702
:10B55000EAF82889BBF808100844288119E00998FE
:10B56000002816DD686804E0028909991144018108
:10B57000006801680029F7D1028909991144018105
:10B5800042890999114441812A89099911442981E3
:10B5900000BF15B90E98E06601E00E98286054F8D7
:10B5A0005C0F384420602089C01B20810D98608189
:10B5B0005C3C109880B11098C06868B1149800F095
:10B5C000020048B90820FAF7D8FA1099C9688989A1
:10B5D00008431099C968888100201CE600BF608B71
:10B5E00040F08000608300BFBBF1000F02D05846DE
:10B5F000FBF766F90E9810B10E98FFF70DFA4FF0B1
:10B60000FF3008E60246107D04280BD0107D072885
:10B6100008D0107D022805D0107D032802D06FF0DD
:10B620000A00704709B90020FBE7B2F864008842BD
:10B6300008DA00BF508B40F08000508300BF4FF00D
:10B64000FF30EEE7B2F86600082808D300BF508B41
:10B6500040F08000508300BF4FF0FF30E1E7002052
:10B66000DFE72DE9FC5F04464FF0000AE56E15B9EF
:10B670000020BDE8FC9F94F89A00FF2804DA94F8B3
:10B680009A00401C84F89A00E9688889FAF775FAEC
:10B6900000F0010018B1288908B9012000E000205D
:10B6A0008146B9F1000F01D1012000E0002083465E
:10B6B000E86843685A4651462046FDF769FE06464B
:10B6C00016B94FF0FF30D4E77768B9F1000F09D011
:10B6D0001120FAF752FAB9894CF2FF0211400843DF
:10B6E000B8810DE0706814300090696809892A8972
:10B6F000891A8BB2012268680099FBF7A1F800BF94
:10B70000E9684868FAF72CFA00F10108206DB0EBFF
:10B71000080001D5C4F85080534600223146204627
:10B72000FDF7B9FE231D224631462046FDF789FE6E
:10B73000019001989DE7000038B505460C46FAF7E0
:10B7400022FA0A4805600A48046006210948FCF705
:10B7500012FA0948FCF73AFA0820C3010022074907
:10B76000009007A0FCF74CFA38BD000070010020E3
:10B7700074010020780100207C010020C9B7000876
:10B7800074637069705F74687265616400000000C2
:10B7900010B50446FFF7E8FC0748006810B90748F1
:10B7A000006828B100220649FA20FCF745FA02E0B9
:10B7B00000200449086010BDE0010020E4010020E1
:10B7C00091B700082002002008B50C48FCF7F3F9F7
:10B7D0000B48006820B10B48006809490968884790
:10B7E0000AE06946084800F035F8009800B903E01F
:10B7F000009800F00BF800BFF3E700007C01002088
:10B8000070010020740100207801002010B504466A
:10B81000207820B101280ED0022818D113E0201D75
:10B8200007C8904710B16068FBF74AF82146092025
:10B83000FAF7B4FB0CE0D4E9011088472146082050
:10B84000FAF7ACFB04E0D4E90110884700E000BF40
:10B8500000BF10BD2DE9F04106460F4600BFFCF7C2
:10B8600055FA0446601C60B91148FCF7BCF9002287
:10B8700039463046FCF71EF90D48FCF79CF9BDE847
:10B88000F08114B9FCF74CF9E9E70948FCF7ABF98A
:10B89000224639463046FCF70DF905460448FCF7C8
:10B8A0008AF9681C10B9FCF73BF9D8E700BFE6E756
:10B8B0007C01002070B505460E460820FAF7A8FB6B
:10B8C000044614B94FF0FF3070BD01202070656050
:10B8D000A66021460648FCF75EF930B121460820F3
:10B8E000FAF75CFB4FF0FF30EEE70020ECE70000DA
:10B8F0007801002010B50446FBF7BEFE10BD000025
:10B90000B0F1804F02D0044A904203D1026861F343
:10B910008A22026070470000000C0040C16282620F
:10B92000436923F001035B1C43617047026861F3C4
:10B93000092202607047026861F3061202607047D4
:10B94000026861F30002026070470146486A70476E
:10B950004162704710B5044621460B4800F078F864
:10B9600001210948FFF7ECFF01218807FFF7E8FFF5
:10B9700000220A211C20FAF755FD01224021080669
:10B9800000F04AF810BD0000002C014010B584689A
:10B9900061F30D348460846862F3CF34846084681A
:10B9A00063F30B24846010BDF0B504460D461646C3
:10B9B0001F463B46324629462046FFF7E7FFA06870
:10B9C00020F4804000F58040A060F0BDCA430261D1
:10B9D000704700001CB504460020019000902046EE
:10B9E000FFF7B3FF019000236A4601A908480068E9
:10B9F00002F044FF0098012809D1009838B14FF0B7
:10BA0000805004490860BFF34F8FBFF36F8F1CBD98
:10BA10003000002004ED00E0012A03D1C3680B438D
:10BA2000C36003E012B9C3688B43C360704702462A
:10BA3000002013690B4023B1D3680B400BB10120E8
:10BA400000E000207047026861F3C712026070478F
:10BA5000C1627047426861F3061242607047026B30
:10BA600061F3070202637047826861F30202826039
:10BA70007047826861F3C712826070472DED028BB8
:10BA800082B00020019000259FED200AB0EE408A90
:10BA90009FED1E0AF0EE408A0220FFF75BFF33E0C5
:10BAA000322201A91A48006802F0FAFF0446012C6C
:10BAB00022D19DED010AB8EE400ADFED160A20EE14
:10BAC000200ADFED150A80EE201AF0EE418A9FED84
:10BAD000130AC0EE280AB0EE608A9FED110A28EE24
:10BAE000000AB0EE408ABCEEC80A10EE100A0D49FA
:10BAF000C968C881002507E028466D1C642803D961
:10BB000000200849C968C881CAE700000000000099
:10BB1000300000200000C842002474493333134031
:10BB200066666640D0030020826861F30612826078
:10BB30007047F8B504466669002500E06D1C0022D8
:10BB40006946F06802F0ACFF0128F7D02846F8BD3E
:10BB50002DE9F05F804689469246D8F814404FF0B0
:10BB6000000B4FF0010BBAF1450F0ED0BAF14E0F9A
:10BB700003D0BAF14F0F0CD103E0002500260027B7
:10BB80000AE002250026012706E0012500260127FC
:10BB900002E04FF0000B00BF00BFBBF1010F29D145
:10BBA0002B4632463946484601F0CAFD352000286A
:10BBB00007DB00F01F0201219140104A430942F8BF
:10BBC000231000BF002207213520FAF72BFCA068C4
:10BBD00058B903220021012002F06BFCA060002272
:10BBE0000121802002F065FCE06001220449206808
:10BBF00000F004FA0020BDE8F09F000080E200E0C1
:10BC000005000C002DE9F04104460D461646676913
:10BC100032462946F86802F043FF012802D100208D
:10BC2000BDE8F0814FF0FF30FAE72DE9F047064616
:10BC30000C461746994675694FF0000816E000BF9C
:10BC40008021286800F05AF90028F9D02178286866
:10BC500000F042F900BF4021286800F04FF90028A9
:10BC6000F9D0641C08F1010000F0FF08B845E6D3E4
:10BC70000020BDE8F0870000014800787047000010
:10BC8000F002002010B5F4F74FFBC0F30D0000F5F3
:10BC900040400149088010BD240200202DE9FE4FDC
:10BCA00005460E46002001906889082803DA2846D8
:10BCB000FAF706FE9BE0D5F804A04E4A11685069D9
:10BCC000F9F734F88146BAF80000F9F756FF8346D1
:10BCD000BAF80200F9F751FF029000240027A046AD
:10BCE0004548046838E0618A0298814232D14A4668
:10BCF0003146204600F082F860B3207C00F004005A
:10BD0000A8B9B8F1000F01D1A04610E0B9F1000FB9
:10BD10000DD038484069401C48B9D8F80000716817
:10BD2000884204D020687168884200D1A046A08A69
:10BD300058450FD1606820B12E4960680969884272
:10BD400008D137B1E068F8602B480068E0602A4805
:10BD5000046003E02746E468002CC4D100BF04B9A6
:10BD6000444614B10120019008E0224970684969F5
:10BD7000884201D1012000E000200190019888B3A1
:10BD800008212846FAF775FE18B12846FAF798FDFB
:10BD90002DE07CB1A06948B1CDF800B0154B10334F
:10BDA0002A462146D4E906C0E0471FE02846FAF7B4
:10BDB00087FD1CE0B9F1000F10D10E48007D00F0A6
:10BDC000F000E0280AD00B488089083001B22846EC
:10BDD000FAF7CFFD03212846F8F744FE2846FAF784
:10BDE0006FFD03E0FFE72846FAF76AFD00BFBDE8F4
:10BDF000FE8F00003CBF00202802002030B5034623
:10BE0000187A50B11C7A1448406890F83000401CF1
:10BE1000C0B2844201D0002030BD8AB173B118682D
:10BE200060B10D484069401C40B118688C682040E2
:10BE3000094C64698D682C40A0420BD10120EBE7CE
:10BE400033B1186820B1044C18686469A04201D16C
:10BE50000120E1E70020DFE73CBF002010B50246EB
:10BE600082B1136873B169B10B685BB1064B186896
:10BE700006E003681468A34201D10B680360C06840
:10BE80000028F6D110BD00002802002070B502463F
:10BE90000C46FF25FF2309E012F8010B80EA03019D
:10BEA0000648405C80EA05030548455C201EA4F175
:10BEB0000106B4B2F0D143EA052070BDC0F6000817
:10BEC000C0F700080148008870470000AA0300205E
:10BED0000146486880B27047C1F30802426070476B
:10BEE000C26861F34D32C260704701F01F0212B1A7
:10BEF0000268426801E0CA43026070470246106867
:10BF0000084008B1012070470020FCE741B94269B0
:10BF100022F480724261426922F40072426127E099
:10BF200001290AD1426922F4807202F580724261CD
:10BF3000426922F4007242611AE002290AD1426980
:10BF400022F480724261426922F4007202F50072AA
:10BF500042610DE003290BD1426922F4807202F59F
:10BF600080724261426922F4007202F500724261FD
:10BF7000704700002DE9F04385B004460F46904617
:10BF800099466846F5F722FC1848844208D01848BC
:10BF9000844205D01748844202D01748844201D118
:10BFA000029E00E0039E06EB86004000B0FBF7F522
:10BFB0000A20B5FBF0F100FB1150052803D20A203E
:10BFC000B5FBF0F503E00A20B5FBF0F0451CA068D6
:10BFD00065F30F00A060E06868F30C30E060206952
:10BFE00069F30D30206105B0BDE8F08300380140F1
:10BFF00000600140006401400068014030B5012A42
:10C000000BD100EB11431B6801F01F050124AC406C
:10C01000234300EB114423600AE000EB11431B684B
:10C0200001F01F050124AC40A34300EB1144236041
:10C0300030BD41B9C26822F40072C260C26822F405
:10C040008062C2601AE001290AD1C26822F400723B
:10C05000C260C26822F4806202F58062C2600DE0B4
:10C0600002290BD1C26822F4007202F50072C2608C
:10C07000C26822F4806202F58062C2607047C268C2
:10C0800061F38202C2607047C26861F3C302C2609A
:10C09000704701460A69D1E901309860D1E901038E
:10C0A00058605068884201D188685060002008615B
:10C0B0001068401E1060106870470000054909684C
:10C0C000886904490968C96AC1F11001014A126806
:10C0D00091617047FC000020034B0360034B0B6031
:10C0E0008023136070470000640A0020640400206D
:10C0F000034B0360034B0B604FF480731360704776
:10C10000C00A00206406002070B504460D4629468A
:10C11000204601F01AFC70BD00F1080141604FF0AB
:10C12000FF31816000F10801C160016100210160FF
:10C13000704700210161704710B502460B685C1C16
:10C140000CB9106907E002F1080000E0406844689B
:10C1500024689C42FAD944684C604C68A1608860AD
:10C1600041600A611468641C146010BD42684A6032
:10C1700093688B60936859609160086103685B1CE9
:10C180000360704710B520210248006801F0DDFB14
:10C1900010BD00000004002070B504460D46164690
:10C1A0004FF480710248006801F0CFFB70BD0000C1
:10C1B0000004002070B504460D4616468021024852
:10C1C000006801F0C2FB70BD0004002070B5044699
:10C1D0000D46164640210248006801F0B6FB70BDCE
:10C1E00000040020014901607047000035F700207D
:10C1F00010B503220021012002F05BF9014908601B
:10C2000010BD0000FC03002070B505460C4620213F
:10C2100013480068FFF769FE012D09D10220F4F7E9
:10C2200079FD01220F490E480068FFF7E7FE05E09F
:10C2300000220C490A480068FFF7E0FE012C08D1F3
:10C240000220F4F72BFD01210748006801F07DFB77
:10C2500004E001210448006801F03AFB70BD0000D1
:10C260000804002005000C001804002038B5C8247C
:10C27000022000F091F8F4F757FB48B10020094B79
:10C280002246092100900848006803F0F3F808E00E
:10C29000002003462246042100900348006803F072
:10C2A000E9F838BD240400202004002008B5F4F784
:10C2B0003BFB48B100200346024608210090074896
:10C2C000006803F0D7F808E0002003460246032187
:10C2D00000900248006803F0CDF808BD200400205B
:10C2E00038B56424012000F057F8F4F71DFB48B17D
:10C2F0000020094B2246092100900848006803F0FD
:10C30000B9F808E0002003462246042100900348C3
:10C31000006803F0AFF838BD24040020200400209A
:10C3200038B511480088322148434FF47A71B0FB88
:10C33000F1F0441C002000F02FF8F4F7F5FA48B1B2
:10C3400000200A4B2246092100900948006803F0AA
:10C3500091F808E00020034622460421009004489A
:10C36000006803F087F838BD1C0400202404002076
:10C370002004002010B500231A4619460248006820
:10C3800002F0A8F910BD0000FC030020014908706C
:10C3900070470000F102002001490870704700005A
:10C3A000B50300200149087070470000F00200202A
:10C3B0000149087070470000F2020020014908801E
:10C3C00070470000AA03002010B502480068FBF780
:10C3D0002BF910BD2C04002000BF502080F31188E1
:10C3E000BFF34F8FBFF36F8F00BF0E480068401C34
:10C3F0000C49086008460068012812D10A48006804
:10C40000C0B208B9012000E0002050B900BF5020A0
:10C4100080F31188BFF34F8FBFF36F8F00BF00BF52
:10C42000FEE770474C00002004ED00E00D48006876
:10C4300050B900BF502080F31188BFF34F8FBFF376
:10C440006F8F00BF00BFFEE706480068401E054929
:10C4500008600846006820B9002080F3118800BFFA
:10C4600000BF70474C00002070B506463546002ED0
:10C4700044D0083D2C46224960680968084008B14C
:10C48000012000E0002050B900BF502080F3118847
:10C49000BFF34F8FBFF36F8F00BF00BFFEE7206871
:10C4A00008B9012000E0002050B900BF502080F3FF
:10C4B0001188BFF34F8FBFF36F8F00BF00BFFEE740
:10C4C0000F49606809680840C0B12068B0B90C49DC
:10C4D000606809688843606000F06EFA0949606826
:10C4E00009680844074908602046FAF7EFFD064846
:10C4F0000068401C0449086002F0E2FE70BD0000C4
:10C500006C0100205C0100206801002000204FF039
:10C51000E02108618861064800684FF47A71B0FB39
:10C52000F1F0401E4FF0E02148610720086170479C
:10C53000F800002070B5F3F7F3FE0446102C16D374
:10C5400004F1E02090F8F05315480078854201DBB3
:10C55000012000E0002050B900BF502080F3118876
:10C56000BFF34F8FBFF36F8F00BF00BFFEE70D48D3
:10C57000006800F4E0600C490968884201D8012095
:10C5800000E0002050B900BF502080F31188BFF3B5
:10C590004F8FBFF36F8F00BF00BFFEE770BD00007D
:10C5A000500000200CED00E0540000200246002066
:10C5B0000BE0084B53F8303033B9064B43F83010DA
:10C5C00003EBC0035A6002E0401C0828F1D300BF0F
:10C5D00070470000405800202DE9F04105460E4606
:10C5E00017462C46FFF7F8FE94F94400401C10B99A
:10C5F000002084F8440094F94500401C10B9002044
:10C6000084F84500FFF712FFA06B28B93A4631467F
:10C6100004F1240000F062F82046FAF7B5FFBDE807
:10C62000F081000070B504460025D4B112480068BE
:10C6300008B9012000E0002050B900BF502080F36D
:10C640001188BFF34F8FBFF36F8F00BF00BFFEE7AE
:10C6500000F0B2F900212046FAF770FA02F030FE3D
:10C6600005463DB94FF0805004490860BFF34F8F35
:10C67000BFF36F8F70BD00003801002004ED00E0B3
:10C680000349096801600349096841607047000077
:10C69000240100201001002001200149086070479A
:10C6A0002001002070B504460D4654B900BF50204B
:10C6B00080F31188BFF34F8FBFF36F8F00BF00BFB0
:10C6C000FEE70548016818312046FFF735FD0121D6
:10C6D0002846FAF733FA70BDFC00002070B5054615
:10C6E0000E46144655B900BF502080F31188BFF3A1
:10C6F0004F8FBFF36F8F00BF00BFFEE70648016892
:10C7000018312846FFF732FD0CB14FF0FF362146B5
:10C710003046FAF713FA70BDFC00002070B50446ED
:10C720000D46164654B900BF502080F31188BFF360
:10C730004F8FBFF36F8F00BF00BFFEE71048006848
:10C7400008B1012000E0002050B900BF502080F364
:10C750001188BFF34F8FBFF36F8F00BF00BFFEE79D
:10C7600045F00040074909688861064801681831AA
:10C770002046FFF7FBFC01213046FAF7DFF970BDD8
:10C7800038010020FC0000202DE9F04706460F4646
:10C7900034464FF00109002E55D0206D50B900BF2E
:10C7A000502080F31188BFF34F8FBFF36F8F00BF0E
:10C7B00000BFFEE7E06CB84201D23D4600E0E56C08
:10C7C000E06AA8423FD0206D01283CD11F48006894
:10C7D000844201D0012000E0002050B900BF502069
:10C7E00080F31188BFF34F8FBFF36F8F00BF00BF7F
:10C7F000FEE7D4F82C80E562A06900F0004010B993
:10C80000C5F11000A06108EB8801114A02EB81011B
:10C810006069884201D1012000E0002098B1201D0C
:10C82000FFF737FC0B49E06A0968884202D90949D9
:10C83000E06A0860E16A01EB8101054A02EB8100D0
:10C84000211DFFF793FCBDE8F0870000FC000020ED
:10C85000805800201401002070B505460E4621487E
:10C86000006808B1012000E0002050B900BF50204E
:10C8700080F31188BFF34F8FBFF36F8F00BF00BFEE
:10C88000FEE746F000402860EC6854B900BF502035
:10C8900080F31188BFF34F8FBFF36F8F00BF00BFCE
:10C8A000FEE72846FFF7F5FB201DFFF7F2FB0E49D8
:10C8B000E06A0968884202D90B49E06A0860E16AC7
:10C8C00001EB8101094A02EB8100211DFFF74EFCBB
:10C8D0000749E06A0968C96A884202D90120054906
:10C8E000086070BD3801002014010020805800202D
:10C8F000FC0000202001002010B586B0002005902B
:10C90000049003AA04A905A8FFF7E6FB0022DDE9CD
:10C9100004101346CDE9002102901FA12048039A7C
:10C9200002F0C8FA1F4908600846006808B10124EF
:10C9300000E00024012C02D102F060FD0446012C2D
:10C9400015D100BF502080F31188BFF34F8FBFF384
:10C950006F8F00BF4FF0FF3013490860012013496B
:10C96000086000201249086001F096FC10E0601C8D
:10C9700008B1012000E0002050B900BF502080F332
:10C980001188BFF34F8FBFF36F8F00BF00BFFEE76B
:10C990000848006806B010BD49444C45000000003E
:10C9A000DD6E0008300100202C010020180100205D
:10C9B000100100203401002002480068401C014999
:10C9C00008607047380100201E48006818B1012037
:10C9D0001D49086034E000201B4908601B480168BD
:10C9E0000CE051B900BF502080F31188BFF34F8F86
:10C9F000BFF36F8F00BF00BFFEE7491E01EB810050
:10CA0000134A52F8200008B9012000E00020002855
:10CA1000E7D101EB81020E4B03EB820042685268C2
:10CA2000426000F108024368934202D142685268B2
:10CA300042604268D268074B1A600448016000BF38
:10CA40007047000038010020200100201401002060
:10CA500080580020FC0000204AF6AA200149086006
:10CA600070470000003000400349496860F302014C
:10CA7000014A516070470000003000404CF6CC4045
:10CA800001490860704700000030004018B90021DB
:10CA9000034A116003E045F25551014A11607047A5
:10CAA00000300040014988607047000000300040BD
:10CAB00000B58BB009A8F7F747FF02208DF82B00CF
:10CAC00000208DF8280008208DF82A0080010990A8
:10CAD00004208DF8290009A94F48F7F740FF0120ED
:10CAE0008DF82B0000208DF828008DF82A004FF4D7
:10CAF0008070099004208DF8290009A94648F7F7AD
:10CB00002EFF01214548F7F787FF07A8F4F76BFAD6
:10CB100002208DF81C0000208DF81D0001208DF8EA
:10CB20001E008DF81F0000208DF820008DF82100D8
:10CB30008DF8220007A93A48F4F7AEF91E20ADF8A7
:10CB4000140000208DF8160005208DF81700002035
:10CB50008DF8180005A93248F4F7FCF901208DF88A
:10CB600004008DF8050000208DF806008DF8070000
:10CB70008DF8080046F64000ADF80A0048F680003F
:10CB8000ADF80E004FF42250ADF80C0046F6A000B0
:10CB9000ADF8100001A92248F4F72EFA01208DF813
:10CBA00004008DF8050000208DF8060001208DF8A6
:10CBB000070000208DF808004AF2C060ADF80A00B6
:10CBC0004AF6E000ADF80E0049F6C000ADF80C00E2
:10CBD00049F6E020ADF8100001A91148F4F70CFA6D
:10CBE000002209211620F9F71DFC0022092114203A
:10CBF000F9F718FC012202210948F4F765FB01222C
:10CC0000D1020748F4F760FB0122D1030448F4F78E
:10CC10005BFB0BB000BD0000000C01400204002CC7
:10CC20000064004000B58BB009A8F7F78DFE022024
:10CC30008DF82B0000208DF8280008208DF82A00A0
:10CC40004020099004208DF8290009A93948F7F7F8
:10CC500086FE01208DF82B0000208DF828008DF82D
:10CC60002A002020099004208DF8290009A93148C4
:10CC7000F7F775FE01213048F7F7CEFE07A8F4F765
:10CC8000B2F900208DF81C008DF81D0001208DF8F0
:10CC90001E008DF81F0000208DF820008DF8210067
:10CCA0008DF8220007A92548F4F7F6F81E20ADF804
:10CCB000140000208DF8160005208DF817000020C4
:10CCC0008DF8180005A91D48F4F744F901208DF8E6
:10CCD000040000208DF807008DF806008DF808008C
:10CCE0008DF80500ADF80A00ADF80C00ADF80E00A7
:10CCF000ADF8100001A91148F4F77EF900220821CF
:10CD00004720F9F78FFB002208214520F9F78AFB1D
:10CD1000012202210948F4F7D7FA0122D10207487B
:10CD2000F4F7D2FA0122D1030448F4F7CDFA0BB09C
:10CD300000BD0000000C01400104042C006800400C
:10CD400010B501210148F7F767FE10BD020310304E
:10CD500010B504460EE0322C05D94CF2503000F0EC
:10CD60000DF8323C06E04FF47A7104FB01F000F05C
:10CD700005F80024002CEED110BD000030B50246AD
:10CD80000A4D2D6802FB05F3094D296800BF084DC7
:10CD90002868884201D3451A04E04FF6FF756D1AE2
:10CDA00005446D1C2C469C42F1D330BD4800002048
:10CDB000241C004000B587B002208DF81B00002025
:10CDC0008DF8180008208DF81A0002200590042024
:10CDD0008DF8190005A97448F7F7C1FD02208DF8F8
:10CDE0001B0000208DF818008DF81A000220059015
:10CDF00004208DF8190005A96C48F7F7B0FD022052
:10CE00008DF81B0000208DF8180008208DF81A00FE
:10CE1000042005908DF8190005A96448F7F79FFDD7
:10CE200002208DF81B0000208DF818008DF81A00E4
:10CE30008020059004208DF8190005A95B48F7F7BC
:10CE40008EFD02208DF81B0000208DF818008DF853
:10CE50001A001020059004208DF8190005A95248E9
:10CE6000F7F77DFD02208DF81B0000208DF81800DB
:10CE70008DF81A002020059004208DF8190005A9CE
:10CE80004948F7F76CFD02208DF81B0000208DF853
:10CE9000180008208DF81A000002059004208DF873
:10CEA000190005A94248F7F75AFD02208DF81B002A
:10CEB00000208DF8180008208DF81A004002059017
:10CEC00004208DF8190005A93948F7F748FD02201C
:10CED0008DF81B0000208DF8180008208DF81A002E
:10CEE0008002059004208DF8190005A93048F7F755
:10CEF00036FD01212F48F7F78FFDF6F7D7FC00BF6D
:10CF0000F6F7C8FC0128FBD0F6F7E6F92A48F6F751
:10CF10005FFA002028490870012088714872487122
:10CF20000846F6F731FA244B5A7A9979187800F0C6
:10CF300047F8012802D0002007B000BD6846F6F788
:10CF400087FC01208DF809008DF80B008DF810008A
:10CF50008DF800008DF801008DF803008DF80A00AF
:10CF600020208DF802008DF8040001208DF80700C4
:10CF70006846F6F75BFA00201049087048704420B4
:10CF800088704520C87056200871012048710846F5
:10CF9000F6F7CEFC01210620F6F728FB01210E2032
:10CFA000F6F724FB0120C7E700100140000801400C
:10CFB000000C01400101123430580020880000208C
:10CFC0002DE9F84306460F469046002000904FF4A6
:10CFD000004200210320F6F707FD10B90020BDE84C
:10CFE000F883002400E0641C10488442FBD300BF97
:10CFF0006D1C6A4600210320F6F7C0FC08B900202A
:10D00000EDE7BDF8000000F4004010B1074885428C
:10D01000EED3002400E0641C04488442FBD3854224
:10D0200001D10020DBE70120D9E70000FFFF0F005E
:10D03000F8B507460D46164600200090012F70D126
:10D0400000BF641C6A4601210320F6F797FC08B96B
:10D050000020F8BDBDF8000000F0040010B9404801
:10D060008442EED33E48844201D10020F1E70024FF
:10D070004FF4805200210320F6F7B6FC08B90020D7
:10D08000E7E700BF641C6A4601210320F6F776FC3F
:10D0900008B90020DDE7BDF8000000F0200010B95D
:10D0A0002F488442EED32E48844201D10020D0E79D
:10D0B0006A4611210320F6F761FC08B90020C8E791
:10D0C000BDF8000000F4004030B10120F6F702FC8A
:10D0D0000120F6F7F5FB41E0BDF8000000F48040C8
:10D0E00030B10120F6F7F6FB0020F6F7E9FB35E05A
:10D0F000BDF8000000F4005030B10020F6F7EAFB64
:10D100000120F6F7DDFB29E0BDF8000000F48050B7
:10D1100000B30020F6F7DEFB0020F6F7D1FB1DE0A0
:10D12000FFE7280240EA463082B200210320F6F7EA
:10D130005BFC08B900208CE7012E03D10120F6F733
:10D14000C9FB02E00020F6F7C5FB012D03D1012049
:10D15000F6F7B6FB02E00020F6F7B2FB012078E715
:10D16000FFFF0F0010B5FFF737F9F7F725FBF7F7CB
:10D1700041FBFFF75BF9FFF7BFFB10BD00B587B0C0
:10D1800000210846FEF7D8FA794800780006784969
:10D19000497840EA01407649897840EA012074499B
:10D1A000C978084302067248007800067049497839
:10D1B00040EA01406E49897840EA01206C49C9780B
:10D1C000084300F47F4042EA0022694800780006E4
:10D1D0006749497840EA01416548807841EA002082
:10D1E0006349C978084300F47F0042EA102260488E
:10D1F000007801065E48407841EA00415C4880784A
:10D2000041EA00205A49C978084342EA1060069072
:10D210005848007800065749497840EA0140554986
:10D22000897840EA01205349C978084302065148E9
:10D23000007800064F49497840EA01404D49897815
:10D2400040EA01204B49C978084300F47F4042EA94
:10D2500000224848007800064649497840EA0141E2
:10D260004448807841EA00204249C978084300F4E4
:10D270007F0042EA10223F48007801063D4840788E
:10D2800041EA00413B48807841EA00203949C978A9
:10D29000084342EA10600590374800780006364996
:10D2A000497840EA01403449897840EA012032490E
:10D2B000C978084302063048007800062E494978AC
:10D2C00040EA01402C49897840EA01202A49C9787E
:10D2D000084300F47F4042EA002227480078000615
:10D2E0002549497840EA01412348807841EA0020F5
:10D2F0002149C978084300F47F0042EA10221E4801
:10D30000007801061C48407841EA00411A488078BC
:10D3100041EA00201849C978084342EA10600490A5
:10D320001648F8F741FC16481649002204ABCDE92F
:10D330000021029005AA06A91348F8F7B3FE08B920
:10D3400000BFFEE71048F8F7F1FF0F48F9F750F873
:10D350000E490D48F9F70DF800204FF400730A4A02
:10D360000B4900900BA0FAF74BFC07B000BD000082
:10D37000640000206C00002068000020880000206D
:10D3800063620008E94600081C1B00208147000872
:10D39000F93C00086574685F6C696E6B5F74687255
:10D3A0006561640070B50320F9F7A0F8F3F74CFC51
:10D3B000054600221146F3F7F4FA044621466FF0C1
:10D3C0000B00F3F749FCF3F73FFC0546002211463A
:10D3D000F3F7E7FA044621466FF00A00F3F73CFC46
:10D3E000F3F732FC054600221146F3F7DAFA044659
:10D3F00021466FF00900F3F72FFCF3F725FC0546F3
:10D4000000221146F3F7CDFA044621466FF00400DE
:10D41000F3F722FCF3F718FC054600221146F3F758
:10D42000C0FA044621466FF00300F3F715FCF3F74A
:10D430000BFC054600220F21F3F7B3FA0446214600
:10D440006FF00100F3F708FCF3F7FEFB054600223E
:10D450000F21F3F7A6FA044621464FF0FF30F3F709
:10D46000FBFB002205214F20F8F7DCFF70BD000018
:10D4700010B501212148F4F76FFA01211F48401C23
:10D48000F4F76AFA01211D48801CF4F765FA0121BE
:10D490001A480E30F4F760FA01214FF4C010F4F787
:10D4A0005BFA01211648F4F757FA01211448401C91
:10D4B000F4F752FA01211248801CF4F74DFA0121C9
:10D4C0000F48C01CF4F748FA01210D481730F4F753
:10D4D00043FA01210B48F4F73FFA012109480D30C6
:10D4E000F4F73AFA012107481230F4F735FA01212E
:10D4F00004481330F4F730FA10BD00000E00140099
:10D500000200180007001C0010B5F4F785FA01218D
:10D510004FF01C10F4F720FA0120FAF719FA2E4800
:10D52000F4F7EAF948B901210320F4F71FF900BF25
:10D530002948F4F7E1F90028FAD00020FAF708FAB0
:10D5400000214FF01C10F4F707FA01210846F4F708
:10D550000DF900BFF4F7E8F90028FBD00121042001
:10D56000F4F704F900BF1D48F4F7C6F90128FAD111
:10D5700001210020F4F7FAF800BF0120F4F7BCF90C
:10D580000128FAD101221D211046F4F707FA0121E2
:10D590000220F4F7EBF800BF1920F4F7ADF90128E9
:10D5A000FAD10020F4F7B0F80420F4F7C1F8042011
:10D5B000F4F7B4F80120F4F7C5F80220F4F758FAAC
:10D5C00000BFF4F773FA0228FBD10020F4F7BAF891
:10D5D000FAF7BCFB10BD0000010020000100240090
:10D5E00030B585B000246846F4F7F0F8039844009D
:10D5F0000B48B4FBF0F0451E2A464FF6FF71094870
:10D60000FEF78CF901200849086000210548FEF763
:10D6100092F901210348FEF793F905B030BD0000EF
:10D6200040420F00001C0040480000201CB5684626
:10D63000F7F78AF901211F48F4F78EF94FF480506B
:10D64000009000208DF806008DF8040004208DF86D
:10D65000050001208DF8070069461748F7F77FF9A4
:10D6600000211648FEF767F900211448FEF75EF91D
:10D6700000211248FEF7F3F900211048FEF7E3F904
:10D6800000224FF6FF710D48FEF748F900210B48C4
:10D69000FEF75EF901210948FEF7EBF90221074880
:10D6A000FEF7D8F900231A4619460448FEF77CF91C
:10D6B0001CBD00000B00180000080140002C0140B8
:10D6C00010B500241D48006842F21071B0FBF1F063
:10D6D000401E84B201214FF4E010F4F73DF901211E
:10D6E0008807FEF70DF900214FF08040FEF723F97F
:10D6F00000214FF08040FEF719F900214FF08040E3
:10D70000FEF7A1F922464FF0FF314FF08040FEF7BF
:10D7100005F900214FF08040FEF7ABF900214FF0F2
:10D720008040FEF797F906214FF08040FEF79CF904
:10D7300000214FF08040FEF7F7F910BDF8000020FF
:10D740002DE9FC4104460D4616461F466846F7F78C
:10D75000FBF801212648F4F7FFF801212548F4F7EA
:10D76000FBF801212348401EF4F7F6F802208DF85B
:10D77000070000208DF8040008208DF80600400204
:10D78000009004208DF8050069461B48F7F7E7F87C
:10D7900002208DF8070000208DF804008DF80600A7
:10D7A000042000908DF8050069461448F7F7D7F873
:10D7B00033462A4621461248FEF7DCFB0121104879
:10D7C000FEF762FC01210E48FEF759FC39460C4871
:10D7D000FEF72FFC00210A48FEF798FB402108487D
:10D7E000FEF783FB01210648FEF77AFBBDE8FC81CA
:10D7F00014001C0005001800001001400014014036
:10D80000005000402DE9FC4104460D4616461F46D7
:10D810006846F7F799F802208DF8070000208DF888
:10D82000040008208DF806001020009004208DF8D8
:10D83000050069461B48F7F792F802208DF80700AB
:10D8400000208DF804008DF80600082000900420C8
:10D850008DF8050069461348F7F781F80121124851
:10D86000F7F7DAF833462A4621461048FEF782FBDE
:10D8700001210E48FEF708FC01210C48FEF7FFFBD2
:10D8800039460A48FEF7D5FB00210848FEF73EFB63
:10D8900040210648FEF729FB01210448FEF720FB42
:10D8A000BDE8FC81000C0140010418340064014013
:10D8B00010B50120FFF7EAF80220FFF7D5F840F68F
:10D8C000FF10FFF7EFF8FFF7C7F8FFF7D7F810BD25
:10D8D0002DE9F04105460E462C4655B900BF5020B3
:10D8E00080F31188BFF34F8FBFF36F8F00BF00BF6E
:10D8F000FEE706F07F4008B9012000E0002050B9A3
:10D9000000BF502080F31188BFF34F8FBFF36F8F9C
:10D9100000BF00BFFEE7FEF75FFD27682068B04349
:10D920002060FEF783FD3846BDE8F08110B5202069
:10D93000F9F748FF044634B100202060201DFEF7AF
:10D94000EBFB00202077204610BD2DE9FE4F074657
:10D950008846002001903C46009057B900BF5020F7
:10D9600080F31188BFF34F8FBFF36F8F00BF00BFED
:10D97000FEE708F07F4008B9012000E0002050B920
:10D9800000BF502080F31188BFF34F8FBFF36F8F1C
:10D9900000BF00BFFEE704F1040909F1080002908E
:10D9A000FFF70AF8D9F80C60206840EA0800206008
:10D9B00026E0D6F804B035680020009005F07F4AD4
:10D9C00025F07F450AF0806028B92068284040B1E2
:10D9D0000120009005E020682840A84201D10120E4
:10D9E0000090009858B10AF0807010B10198284357
:10D9F0000190206840F000713046FEF72DFF5E4632
:10DA000002988642D5D1206801998843206001F0B0
:10DA100057FC2068BDE8FE8F2DE9F04104460D4615
:10DA2000164633462A462146034801F065FD07465F
:10DA30003846BDE8F081000009C100082DE9FF4F1C
:10DA400083B081460D461746DDF840804C464FF0C6
:10DA5000000A00200190B9F1000F0AD100BF502048
:10DA600080F31188BFF34F8FBFF36F8F00BF00BFEC
:10DA7000FEE705F07F4008B9012000E0002050B922
:10DA800000BF502080F31188BFF34F8FBFF36F8F1B
:10DA900000BF00BFFEE70DB1012000E0002050B93B
:10DAA00000BF502080F31188BFF34F8FBFF36F8FFB
:10DAB00000BF00BFFEE701F05BFA10B9B8F1000F3C
:10DAC00001D1012000E0002050B900BF502080F3B8
:10DAD0001188BFF34F8FBFF36F8F00BF00BFFEE70A
:10DAE000FEF76AFF206800902946069A0098F9F729
:10DAF0002FFD0290029838B1009E4FF00008C7B188
:10DB00002068A843206014E0B8F1000F03D1009E04
:10DB1000012001900DE00FB14AF0807A069808B11B
:10DB20004AF0806A45EA0A014246201DFEF7F6FDEA
:10DB3000002601F0C5FB8346B8F1000F23D0BBF1EE
:10DB4000000F07D14FF0805011490860BFF34F8F8D
:10DB5000BFF36F8FFEF7B2FA064606F0007080B989
:10DB6000FEF73AFC266829463046069AF9F7F0FC9B
:10DB700018B117B12068A843206001200190FEF77A
:10DB800055FC26F07F46304607B0BDE8F08F000018
:10DB900004ED00E038B504464FF0FF3000230122C9
:10DBA0001F21009011480068FFF748FF0546042D2B
:10DBB00010D004DC012D07D0022D14D107E0082D70
:10DBC0000BD0102D0FD10BE0012020800BE00220A4
:10DBD000208008E00420208005E00820208002E06A
:10DBE0001020208000BF00BF012038BD00040020AD
:10DBF00010B5FFF79BFE064908600846006808B1AB
:10DC000000BF03E000BF00BF002010BD0120FCE703
:10DC10000004002038B5044600BF00BF0948006872
:10DC200070B1F2F781FE30B16A46214605480068BE
:10DC3000FFF7F2FE04E0214602480068FFF785FE88
:10DC4000012038BD0004002010B504460122214601
:10DC50000248F2F721FE012010BD00000C04002054
:10DC60002DE9FE4F06460F46904699464FF0000BB1
:10DC70004FF0010B2EB9404850F826003F4908608C
:10DC800001E04FF0000BB9F1000F06D0B9F1010F20
:10DC900006D0B9F1020F09D105E00025002408E003
:10DCA0000225002405E00125002402E04FF0000BCE
:10DCB00000BF00BFB8F1080F06D114B94FF0000A39
:10DCC00001E04FF0000B02E04FF0000B00BF00BF7F
:10DCD000BBF1010F26D12B46224651463846FFF7AD
:10DCE00091FD2648006826490844B8B90022254914
:10DCF00022480068FEF782F94D20002807DB00F07B
:10DD00001F0201219140204A430942F8231000BF1D
:10DD1000002206214D20F8F785FB02E04FF0000BB2
:10DD200000BF00BF19481A4908600020C8808880D9
:10DD3000FFF7FCFD174908600846006808B100BFFE
:10DD400001E000BF00BF0120029000200321034634
:10DD50008022CDE9001010A1124801F079F802905C
:10DD60000298012801D100BF04E000BF00BF0020DD
:10DD7000BDE8FE8F0120FBE704040020080400201A
:10DD8000009CFEBF05000C0080E200E0E2140120D0
:10DD90000C040020180400206D625F74785F6972C3
:10DDA00071000000597A000810B504462046F9F7C2
:10DDB00065FE012010BD000038B504460F48048000
:10DDC0000088322148434FF47A71B0FBF1F0451CD2
:10DDD0000B4801230022294600900AA001F0F2FA24
:10DDE0000C4908600846006818B100BF00BF012058
:10DDF00038BD00BF00BF0020FAE700001C0400206F
:10DE0000F5B800084D61737465722074696D6572B0
:10DE1000000000002004002038B500246846FFF709
:10DE200013FF1E48007830B101280AD002281DD007
:10DE300003282FD102E0FEF773FA2BE0FEF770FA09
:10DE400028E0FEF733FA00201549087015490880CC
:10DE50009DF800200888411C124B198012490A5471
:10DE600002200E490870FEF75BFA13E00D480088A7
:10DE7000FF2809DC9DF800200A490888411C094B4D
:10DE8000198009490A5402E0032004490870FEF78A
:10DE900047FA00BF00BF204638BD0000A90300209C
:10DEA000A8030020B203002031F8002010B50024A0
:10DEB0001F48007820B1022807D0032812D109E0BA
:10DEC0000120FFF7A7FE04460DE00220FFF7A2FEA7
:10DED000044608E00120FEF76BFA1020FFF79AFED7
:10DEE000044600E000BF00BF01201149087011483E
:10DEF000007802280AD11048007830B90020FEF7D7
:10DF000057FA1020FFF786FE044600E000BF00BF6E
:10DF1000002008490870FEF7C9F90848007802286F
:10DF200003D10420FFF776FE0446204610BD000012
:10DF3000A9030020A8030020B4030020B50300209B
:10DF400010B500241D48007810B1012831D104E03B
:10DF500000210120FEF758F92CE01948008878B11B
:10DF6000184909680878FFF71FFF16480068401C29
:10DF70001449086012480088401E1149088017E0C3
:10DF80001148007808B9012000E000200F4908700E
:10DF900000210120FEF738F90220084908700B48DB
:10DFA0000078012802D1FEF761F901E0FEF798F947
:10DFB00000E000BF00BF204610BD0000A803002005
:10DFC000B0030020AC03002034F70020B40300208D
:10DFD0000148007870470000B403002010B50446E3
:10DFE000601C50B94FF0FF310948006800F00CFE8A
:10DFF00008B1012010BD0020FCE72146044800685C
:10E0000000F002FE08B10120F4E70020F2E7000072
:10E01000FC03002038B504464FF0FF3000230122F6
:10E020000F2100900E480068FFF708FD0546012DFE
:10E0300006D0022D07D0042D08D0082D0CD108E001
:10E040000120207008E00220207005E004202070EC
:10E0500002E00820207000BF00BF012038BD000092
:10E06000F803002010B5FFF761FC06490860084678
:10E07000006808B100BF03E000BF00BF002010BD72
:10E080000120FCE7F803002038B5044600BF00BFBC
:10E090000948006870B1F2F747FC30B16A46214682
:10E0A00005480068FFF7B8FC04E021460248006814
:10E0B000FFF74BFC012038BDF8030020024605485D
:10E0C00010600548008808800020034B188001205C
:10E0D00070470000EB150120300400202DE9F041CD
:10E0E00004464FF0000814B94FF4FB7600E02646D2
:10E0F000FAF791FF0746051E01D180461CE0324623
:10E1000010492846F9F79AFF28B13846F9F7EEFF8B
:10E110004FF0000810E0FF212846FAF7C9FE051E5F
:10E1200004D13846F9F7E2FFA84605E0064928463B
:10E13000F9F70DFF054805604FF001084046BDE8BE
:10E14000F0810000B8F60008A97600082804002035
:10E1500070B505460C4600261248006800281ED0FF
:10E1600010480068B0F86400A04200DB05E040F20F
:10E170001F120DA11AA0F2F72FF9012322462946FA
:10E1800008480068FDF731F828B906480068FAF732
:10E19000D3FF012603E003480068F9F745FA30464B
:10E1A00070BD00002C0400202E2E5C2E2E5C6D69AC
:10E1B00064646C6577617265735C467265654D6F0A
:10E1C000646275735C706F72745C467265655254FC
:10E1D0004F535C706F72747463702E6300000000A4
:10E1E0007463705F736E6462756628207078504344
:10E1F00042436C69656E742029203E3D207573543E
:10E2000043504C656E67746800000000F0B503462B
:10E210000C461546E208A4EBC20087B20120A840D4
:10E22000401E86B2995C501C185C41EA00213941BD
:10E230003140C8B2F0BD2DE9F043044615461F46F3
:10E24000C808A1EBC0081FFA88FC07FA0CF81FFAEF
:10E2500088F74FF0010808FA05F8A8F101081FFA3D
:10E2600088F6A1EBC00806FA08F81FFA88F6225CC7
:10E2700000F1010814F8088042EA082222EA0608A0
:10E2800048EA070222544FEA222900F1010804F863
:10E290000890BDE8F08300001CB552480068524960
:10E2A000884201D0012000E0002050B900BF50207A
:10E2B00080F31188BFF34F8FBFF36F8F00BF00BF94
:10E2C000FEE7484800684849491E884201D00120BD
:10E2D00000E0002050B900BF502080F31188BFF348
:10E2E0004F8FBFF36F8F00BF00BFFEE73F49084667
:10E2F00000780190FF200A461070084600780090D0
:10E300009DF8000000F0F0009DF80020904201D13F
:10E31000012000E0002050B900BF502080F3118898
:10E32000BFF34F8FBFF36F8F00BF00BFFEE79DF8B5
:10E33000000000F050002E4A107007202D4A106097
:10E3400009E02C480068401E2A4A10609DF8000031
:10E350004006000E00909DF8000000F0800080282C
:10E36000EFD024480068C0F10700042801D1012043
:10E3700000E0002050B900BF502080F31188BFF3A7
:10E380004F8FBFF36F8F00BF00BFFEE719480068D3
:10E390000002184A10601046008800F4E060106027
:10E3A000124A019810700F482030006840F4700045
:10E3B0000C49203108600846006840F07040086051
:10E3C000FEF7A4F800200C490860F1F771FF0B4834
:10E3D000006840F0404009490860F1F755FF00200F
:10E3E0001CBD000000ED00E071C20F4100E400E040
:10E3F00050000020540000204C00002034EF00E0CA
:10E4000010B500BF502080F31188BFF34F8FBFF3CA
:10E410006F8F00BF00F0C2FD18B14FF0805004496B
:10E42000086000BF002080F3118800BF10BD00000D
:10E4300004ED00E070B505460E460DB1012000E088
:10E44000002050B900BF502080F31188BFF34F8FD8
:10E45000BFF36F8F00BF00BFFEE7AE4201D80120BF
:10E4600000E0002050B900BF502080F31188BFF3B6
:10E470004F8FBFF36F8F00BF00BFFEE70222002166
:10E48000284600F016F8044604B1A663204670BD85
:10E490002DE9F041044601260027224600210120F3
:10E4A00000F007F805462846F8F72CFD2846BDE899
:10E4B000F0812DE9F84306460F4690460EB1012043
:10E4C00000E0002050B900BF502080F31188BFF356
:10E4D0004F8FBFF36F8F00BF00BFFEE706FB07F54E
:10E4E0001FB1B5FBF7F0B04201D1012000E00020E0
:10E4F00050B900BF502080F31188BFF34F8FBFF396
:10E500006F8F00BF00BFFEE705F15000A84201D9A0
:10E51000012000E0002050B900BF502080F3118896
:10E52000BFF34F8FBFF36F8F00BF00BFFEE705F152
:10E530005000F9F747F9044664B1A14609F15009C2
:10E54000002084F8460043464A4639463046009447
:10E55000F8F7E7FC2046BDE8F8832DE9F84380464C
:10E560000E4617461D46DDF82090B8F1000F01D089
:10E57000012000E0002050B900BF502080F3118836
:10E58000BFF34F8FBFF36F8F00BF00BFFEE70DB12A
:10E59000012000E0002050B900BF502080F3118816
:10E5A000BFF34F8FBFF36F8F00BF00BFFEE707B110
:10E5B0000EB1012000E0002050B900BF502080F3D0
:10E5C0001188BFF34F8FBFF36F8F00BF00BFFEE70F
:10E5D00007B90EB9012000E0002050B900BF50205B
:10E5E00080F31188BFF34F8FBFF36F8F00BF00BF61
:10E5F000FEE7502000900098502801D1012000E053
:10E60000002050B900BF502080F31188BFF34F8F16
:10E61000BFF36F8F00BF00BFFEE700BF2C464CB1B9
:10E62000012084F846004B463A4631464046009465
:10E63000F8F777FC2046BDE8F883000070B5054682
:10E640000E462C4654B900BF502080F31188BFF30A
:10E650004F8FBFF36F8F00BF00BFFEE7FDF7BCFE1B
:10E66000D4E90F12206801FB0200A0600020A06323
:10E6700020686060E06B401E226C216800FB021184
:10E68000E160FF2084F8440084F845009EB92069C9
:10E6900008B9012000E00020A8B904F1100000F042
:10E6A000C3FD80B14FF0805009490860BFF34F8F20
:10E6B000BFF36F8F07E004F11000FDF72DFD04F1AB
:10E6C0002400FDF729FDFDF7B1FE012070BD00001B
:10E6D00004ED00E02DE9FF4383B0064688461D4661
:10E6E0004FF00009344654B900BF502080F3118820
:10E6F000BFF34F8FBFF36F8F00BF00BFFEE7B8F1CE
:10E70000000F01D1206C08B9012000E0002050B9B1
:10E7100000BF502080F31188BFF34F8FBFF36F8F7E
:10E7200000BF00BFFEE7022D02D1E06B012801D13E
:10E73000012000E0002050B900BF502080F3118874
:10E74000BFF34F8FBFF36F8F00BF00BFFEE700F036
:10E750000FFC08B9059808B9012000E0002050B965
:10E7600000BF502080F31188BFF34F8FBFF36F8F2E
:10E7700000BF00BFFEE700BFFDF72EFEA06BE16B00
:10E78000884201D3022D28D12A4641462046F8F777
:10E79000E2FA0746606A08B9012000E0002068B983
:10E7A00004F1240000F040FD88B14FF08050324960
:10E7B0000860BFF34F8FBFF36F8F08E03FB14FF09A
:10E7C00080502D490860BFF34F8FBFF36F8FFDF767
:10E7D0002DFE012007B0BDE8F083059818B9FDF7BC
:10E7E00025FE0020F6E7B9F1000F04D101A8FDF7DE
:10E7F00047FF4FF00109FDF719FEFEF7DDF8FDF7C1
:10E80000EBFD94F94400401C10B9002084F844004A
:10E8100094F94500401C10B9002084F84500FDF72C
:10E8200005FE05A901A800F0CBFAF0B92046F8F7DB
:10E83000BAFCA0B104F110000599FDF733FF2046A2
:10E84000F8F7A2FE00F03CFD002895D14FF0805073
:10E8500009490860BFF34F8FBFF36F8F8CE72046E5
:10E86000F8F792FE00F02CFD86E72046F8F78CFEC4
:10E8700000F026FD0020ADE704ED00E02DE9F84FA3
:10E8800007468B4690461E463C4654B900BF502072
:10E8900080F31188BFF34F8FBFF36F8F00BF00BFAE
:10E8A000FEE7BBF1000F01D1206C08B9012000E0A8
:10E8B000002050B900BF502080F31188BFF34F8F64
:10E8C000BFF36F8F00BF00BFFEE7022E02D1E06BE7
:10E8D000012801D1012000E0002050B900BF5020E4
:10E8E00080F31188BFF34F8FBFF36F8F00BF00BF5E
:10E8F000FEE7FDF71FFE00BF5021EFF3118081F30B
:10E900001188BFF34F8FBFF36F8F00BF0546A06B19
:10E91000E16B884201D3022E37D194F945A0A06B58
:10E920000090324659462046F8F715FA0AF10100E0
:10E9300088B9606A08B9012000E0002050B904F1EC
:10E94000240000F071FC28B1B8F1000F02D00120C2
:10E95000C8F8000016E0BAF17F0F01D0012000E0F6
:10E96000002050B900BF502080F31188BFF34F8FB3
:10E97000BFF36F8F00BF00BFFEE70AF1010040B296
:10E9800084F845004FF0010901E04FF0000900BF95
:10E9900085F3118800BF4846BDE8F88F2DE9F047A0
:10E9A00006460F46344654B900BF502080F3118804
:10E9B000BFF34F8FBFF36F8F00BF00BFFEE7206C28
:10E9C00008B9012000E0002050B900BF502080F3BA
:10E9D0001188BFF34F8FBFF36F8F00BF00BFFEE7FB
:10E9E000206808B9A06808B9012000E0002050B9EB
:10E9F00000BF502080F31188BFF34F8FBFF36F8F9C
:10EA000000BF00BFFEE7FDF795FD00BF5021EFF30B
:10EA1000118081F31188BFF34F8FBFF36F8F00BF59
:10EA20000546D4F838A0E06B504530D994F94590AC
:10EA30000AF10100A06309F1010070B9606A08B928
:10EA4000012000E00020F8B904F1240000F0ECFB04
:10EA5000D0B1CFB10120386016E0B9F17F0F01D0FD
:10EA6000012000E0002050B900BF502080F3118841
:10EA7000BFF34F8FBFF36F8F00BF00BFFEE709F1F9
:10EA8000010040B284F845004FF0010801E04FF06A
:10EA9000000800BF85F3118800BF4046BDE8F0873D
:10EAA0002DE9F74183B005460E464FF000082C468D
:10EAB00054B900BF502080F31188BFF34F8FBFF3CC
:10EAC0006F8F00BF00BFFEE70EB9206C08B90120B0
:10EAD00000E0002050B900BF502080F31188BFF340
:10EAE0004F8FBFF36F8F00BF00BFFEE700F040FA0B
:10EAF00008B9059808B9012000E0002050B900BF0E
:10EB0000502080F31188BFF34F8FBFF36F8F00BF8A
:10EB100000BFFEE700BFFDF75FFCA76BF7B1314612
:10EB20002046F8F703F9781EA063206908B9012090
:10EB300000E0002060B904F1100000F075FB38B16E
:10EB40004FF080502F490860BFF34F8FBFF36F8F96
:10EB5000FDF76CFC012006B0BDE8F081059818B9FE
:10EB6000FDF764FC0020F6E7B8F1000F04D101A81E
:10EB7000FDF786FD4FF00108FDF758FCFDF71CFF7F
:10EB8000FDF72AFC94F94400401C10B9002084F8D9
:10EB9000440094F94500401C10B9002084F8450059
:10EBA000FDF744FC05A901A800F00AF9F0B92046D8
:10EBB000F8F7ECFAA0B104F124000599FDF772FD15
:10EBC0002046F8F7E1FC00F07BFB0028A3D14FF0D2
:10EBD00080500C490860BFF34F8FBFF36F8F9AE7E7
:10EBE0002046F8F7D1FC00F06BFB94E72046F8F7DD
:10EBF000CBFC00F065FB2046F8F7C8FA00288AD065
:10EC00000020A8E704ED00E02DE9F34182B00546BD
:10EC10004FF000082C46002654B900BF502080F366
:10EC20001188BFF34F8FBFF36F8F00BF00BFFEE7A8
:10EC3000206C08B9012000E0002050B900BF50202E
:10EC400080F31188BFF34F8FBFF36F8F00BF00BFFA
:10EC5000FEE700F08DF908B9039808B9012000E03B
:10EC6000002050B900BF502080F31188BFF34F8FB0
:10EC7000BFF36F8F00BF00BFFEE700BFFDF7ACFB27
:10EC8000A76BFFB1781EA063206810B9F8F750FE9B
:10EC9000A060206908B9012000E0002060B904F1FB
:10ECA000100000F0C1FA38B14FF0805043490860BD
:10ECB000BFF34F8FBFF36F8FFDF7B8FB012004B098
:10ECC000BDE8F081039898B90EB9012000E000205A
:10ECD00050B900BF502080F31188BFF34F8FBFF3AE
:10ECE0006F8F00BF00BFFEE7FDF7A0FB0020E6E747
:10ECF000B8F1000F04D16846FDF7C2FC4FF00108DF
:10ED0000FDF794FBFDF758FEFDF766FB94F9440010
:10ED1000401C10B9002084F8440094F94500401CC0
:10ED200010B9002084F84500FDF780FB03A9684670
:10ED300000F046F840BB2046F8F728FAF0B120680A
:10ED400038B9FDF749FBA06800F01CFA0646FDF74C
:10ED50006DFB04F124000399FDF7A4FC2046F8F7AD
:10ED600013FC00F0ADFA002888D14FF08050134911
:10ED70000860BFF34F8FBFF36F8F7FE72046F8F730
:10ED800003FC00F09DFA79E72046F8F7FDFB00F060
:10ED900097FA2046F8F7FAF90028EED05EB1FDF7B1
:10EDA0001BFB2046F8F73EF807463946A068FDF7FA
:10EDB000EBFCFDF73BFB002081E7000004ED00E0E9
:10EDC00070B505460C4655B900BF502080F3118838
:10EDD000BFF34F8FBFF36F8F00BF00BFFEE754B983
:10EDE00000BF502080F31188BFF34F8FBFF36F8FA8
:10EDF00000BF00BFFEE7FDF7EFFA1348026868683E
:10EE0000131A2068401C08B9002619E00F49286829
:10EE10000968884206D06868904203D8012600201D
:10EE200020600DE02068984207D92068C01A206051
:10EE30002846FDF725FC002602E000202060012680
:10EE4000FDF7F4FA304670BD1001002024010020C7
:10EE50002DE9FF4F85B0804689461746DDE912ABA4
:10EE6000B800F8F7AFFC064656B15C20F8F7AAFCEC
:10EE700004460CB1266304E03046FDF7F5FA00E0E5
:10EE800000248CB1002084F85900CDE900ABCDE915
:10EE900002403A4649464046089BF8F757F8204654
:10EEA000F7F78AFE012501E04FF0FF35284609B04B
:10EEB000BDE8F08F2DE9F04F85B0074688469146B2
:10EEC0009A46DDE90EB6109C0EB1012000E000204C
:10EED00050B900BF502080F31188BFF34F8FBFF3AC
:10EEE0006F8F00BF00BFFEE70CB1012000E00020E3
:10EEF00050B900BF502080F31188BFF34F8FBFF38C
:10EF00006F8F00BF00BFFEE75C20039003985C2872
:10EF100001D1012000E0002050B900BF502080F353
:10EF20001188BFF34F8FBFF36F8F00BF00BFFEE7A5
:10EF300000BFB4B1AEB125462C462E63022085F841
:10EF40005900002004A953464A46CDE900B1CDE955
:10EF5000025041463846F7F7F9FF2846F7F72CFEEE
:10EF600001E000200490049805B0BDE8F08F000097
:10EF70000549096809B9012005E00449096809B98A
:10EF8000022000E000207047180100203801002016
:10EF90000149086870470000100100202DE9F04188
:10EFA0004FF000084348006800287BD142480068C1
:10EFB000451C4148056015BB40480068006808B919
:10EFC000012000E0002050B900BF502080F31188DC
:10EFD000BFF34F8FBFF36F8F00BF00BFFEE737480F
:10EFE0000768374800683549086035480760354884
:10EFF0000068401C33490860F8F70AFA00BF32483D
:10F00000006885423BD300BF2C480068006808B9FF
:10F01000012000E0002020B14FF0FF302A490860B5
:10F020002CE026480068C068C4686668B54202D211
:10F030002548066022E0201DFDF72BF8A06A18B1D4
:10F0400004F11800FDF725F82049E06A09688842B4
:10F0500002D91E49E06A0860E16A01EB81011C4A9D
:10F0600002EB8100211DFDF781F81A49E06A096869
:10F07000C96A8842C8D34FF00108C5E700BF1548E8
:10F080000068C06A00EB8000114951F82000012897
:10F0900001D94FF001081048006808B14FF001088D
:10F0A00005E0FFE70D480068401C0C490860404639
:10F0B000BDE8F0813801002010010020000100208F
:10F0C00004010020240100202C0100201401002054
:10F0D00080580020FC000020200100201C0100209E
:10F0E00070B505462C460026002D43D02248006806
:10F0F000844201D1012000E0002050B900BF50201F
:10F1000080F31188BFF34F8FBFF36F8F00BF00BF35
:10F11000FEE7206D50B900BF502080F31188BFF387
:10F120004F8FBFF36F8F00BF00BFFEE7206D401E03
:10F130002065E16CE06A88421CD0206DD0B9201DAA
:10F14000FCF7A7FFE06CE062E06AC0F11000A0618C
:10F150000A49E06A0968884202D90849E06A0860F9
:10F16000E16A01EB8101064A02EB8100211DFCF7F7
:10F17000FDFF0126304670BDFC0000201401002078
:10F180008058002070B505462C460026002D42D040
:10F190002249E06A0968C96A884235D2A06900F04C
:10F1A000004028B91D480068C06AC0F11000A06185
:10F1B000E16A01EB81011A4A02EB81016069884230
:10F1C00001D1012000E00020C0B1201DFCF761FF4B
:10F1D00012480068C06AE0621249E06A0968884221
:10F1E00002D91049E06A0860E16A01EB81010C4A2A
:10F1F00002EB8100211DFCF7B9FF03E0074800681E
:10F20000C06AE062012606E00449E06C0968C96A48
:10F21000884200D20126304670BD0000FC0000206C
:10F22000805800201401002070B50646F068C468BC
:10F2300054B900BF502080F31188BFF34F8FBFF344
:10F240006F8F00BF00BFFEE704F11800FCF721FF3D
:10F2500015480068A0B9201DFCF71BFF1349E06AA0
:10F260000968884202D91149E06A0860E16A01EB45
:10F2700081010F4A02EB8100211DFCF777FF04E0BA
:10F2800004F118010B48FCF771FF0B49E06A0968AB
:10F29000C96A884204D9012501200849086000E0B4
:10F2A0000025284670BD0000380100201401002010
:10F2B00080580020E8590020FC0000202001002098
:10F2C00070B5002400263648006850B900BF5020B1
:10F2D00080F31188BFF34F8FBFF36F8F00BF00BF64
:10F2E000FEE7FDF779F82E480068401E2C490860BB
:10F2F0000846006800284ED12A48006800284AD0F5
:10F3000023E02948C068C46804F11800FCF7C1FE76
:10F31000201DFCF7BEFE2549E06A0968884202D933
:10F320002249E06A0860E16A01EB8101204A02EBB0
:10F330008100211DFCF71AFF1E49E06A0968C96AAD
:10F34000884202D301201C4908601748006808B9A8
:10F35000012000E000200028D3D00CB1F8F758F8C5
:10F360001648056865B100BFFFF718FE10B101200F
:10F37000114908606D1E002DF6D100200F4908606C
:10F380000D48006838B1012630070D490860BFF309
:10F390004F8FBFF36F8FFDF749F8304670BD000007
:10F3A000380100200C010020E85900201401002041
:10F3B00080580020FC000020200100201C010020BB
:10F3C00004ED00E02DE9FC4705460E461746984639
:10F3D000DDF828902C20F8F7F5F9044654B1002008
:10F3E00084F8280043463A4631462846CDE9009441
:10F3F000F7F70BFE2046BDE8FC87000010B586B08D
:10F400000024F7F735FC16480068D0B100200590BD
:10F41000049003AA04A905A8FCF76AFE0222DDE90C
:10F4200004100023CDE9002102900EA10F48039A99
:10F43000FFF740FD0E4908600846006800B101244E
:10F4400000BF54B900BF502080F31188BFF34F8F25
:10F45000BFF36F8F00BF00BFFEE7204606B010BDB0
:10F4600044010020546D7220537663006F750008CC
:10F47000480100202DE9FF4704460D4616461F4669
:10F48000DDF830804FF0000954B900BF502080F300
:10F490001188BFF34F8FBFF36F8F00BF00BFFEE730
:10F4A0001448006810B3009501960294062D15DAF1
:10F4B000FFF75EFD022808D10023424669460D4849
:10F4C0000068FFF707F9814610E000231A466946F5
:10F4D00008480068FFF7FEF8814607E000233A4637
:10F4E000694604480068FFF7C9F98146484604B0F8
:10F4F000BDE8F087440100202DE9FF4104460D4698
:10F5000016461F466FF00100009001940295039685
:10F5100000233A46694604480068FFF7AFF9804681
:10F52000404604B0BDE8F081440100204FF0407037
:10F53000E1EE100A70470000000000000000010228
:10F54000030406070809000000000102030400008C
:10F5500000000102030402040608020C0810000067
:10F560000000000000000102030406070809FFFF75
:10F57000FFFFFFFF0000000000000000200004006B
:10F58000A7C50020900100209C0005002AC600208D
:10F59000940100201C00080039C9002098010020B7
:10F5A000100010001CCA00209C0100202000050053
:10F5B0001FCB0020A001002018000F00C2CB0020AC
:10F5C000A4010020100002002DCD0020A801002081
:10F5D0002800040050CD0020AC01002010000800DD
:10F5E000F3CD0020B00100201000080076CE0020EE
:10F5F000B401002010000300F9CE0020B801002063
:10F60000100010002CCF0020BC0100206002100070
:10F610002FD00020C00100207CF5000888F50008EC
:10F6200094F50008A0F50008ACF50008B8F500084E
:10F63000C4F50008D0F50008DCF50008E8F500087E
:10F64000F4F5000800F600080CF60008E4F80008DD
:10F650000CF900082CF90008ECF80008D8F80008AC
:10F66000C0F80008CCF8000820F90008F8F80008F5
:10F6700000F9000814F90008010203040506070751
:10F68000070707070703060C18306078DC01002025
:10F69000D8010020E0010020E4010020FA00000071
:10F6A00069B10008E8030000D1570008E803000032
:10F6B000394400080300000000000000FFFFFFFFC6
:10F6C00000C1814001C0804101C0804100C1814032
:10F6D00001C0804100C1814000C1814001C0804122
:10F6E00001C0804100C1814000C1814001C0804112
:10F6F00000C1814001C0804101C0804100C1814002
:10F7000001C0804100C1814000C1814001C08041F1
:10F7100000C1814001C0804101C0804100C18140E1
:10F7200000C1814001C0804101C0804100C18140D1
:10F7300001C0804100C1814000C1814001C08041C1
:10F7400001C0804100C1814000C1814001C08041B1
:10F7500000C1814001C0804101C0804100C18140A1
:10F7600000C1814001C0804101C0804100C1814091
:10F7700001C0804100C1814000C1814001C0804181
:10F7800000C1814001C0804101C0804100C1814071
:10F7900001C0804100C1814000C1814001C0804161
:10F7A00001C0804100C1814000C1814001C0804151
:10F7B00000C1814001C0804101C0804100C1814041
:10F7C00000C0C101C30302C2C60607C705C5C40401
:10F7D000CC0C0DCD0FCFCE0E0ACACB0BC90908C871
:10F7E000D81819D91BDBDA1A1EDEDF1FDD1D1CDC61
:10F7F00014D4D515D71716D6D21213D311D1D010D1
:10F80000F03031F133F3F23236F6F737F53534F4C0
:10F810003CFCFD3DFF3F3EFEFA3A3BFB39F9F83830
:10F8200028E8E929EB2B2AEAEE2E2FEF2DEDEC2C20
:10F83000E42425E527E7E62622E2E323E12120E090
:10F84000A06061A163A3A26266A6A767A56564A480
:10F850006CACAD6DAF6F6EAEAA6A6BAB69A9A868F0
:10F8600078B8B979BB7B7ABABE7E7FBF7DBDBC7CE0
:10F87000B47475B577B7B67672B2B373B17170B050
:10F880005090915193535292965657975595945440
:10F890009C5C5D9D5F9F9E5E5A9A9B5B99595898B0
:10F8A000884849894B8B8A4A4E8E8F4F8D4D4C8CA0
:10F8B0004484854587474686824243834181804010
:10F8C00046494E5F574149545F31000046494E5FFB
:10F8D000574149545F32000045535441424C49530B
:10F8E00048454400434C4F534544000053594E5F34
:10F8F0005243564400000000434C4F53494E4700CA
:10F900004C4153545F41434B000000004C49535459
:10F91000454E000054494D455F5741495400000091
:10F92000434C4F53455F57414954000053594E5F74
:10F9300053454E540000000075617274350000009C
:10F9400060F900080000002064040000C001000805
:10F950005CFA0008640400205C2201001C0200081C
:10F96000014C1AAA0101141DC0A801250405220199
:10F97000FFFFFF140801404A10041240120832042D
:10F9800012021A18084904391C320129085A023097
:10F99000291029086910293529084A0808291F0152
:10F9A000110339127A029C0F021AC00B4A6E1954C5
:10F9B000022902321113511E33080413F11C3308BB
:10F9C000031A6308321013BB1F3308061AE92032EA
:10F9D00017137D1D33080113091B3308051A791805
:10F9E000320F1A2B2829721AB718013F0927B9A913
:10F9F000B84BA722B81A330829B84B0525B84B2DA8
:10FA000024B84B1923B84B0521B81ABD1029B81AD0
:10FA10006F2029711A9D18016413BA031B20C404B6
:10FA20001352F914201AFA82201AE20C1362FB1BFB
:10FA300020E2047C6208011851042D640140125038
:10FA4000B9301338F9140851BB1C082BBCFC19043D
:0CFA50001A330C1334041B204404410042
:040000050800018569
:00000001FF
